:020000040800F2
:1000000000500020DD1000088D1100087954000810
:100010008D1100088D1100088D11000800000000EE
:100020000000000000000000000000008D1100082A
:100030008D110008000000008D110008556A0008AD
:100040008D1100088D1100088D1100088D11000818
:100050008D1100088D1100088D110008512D000828
:100060008D1100088D1100088D1100088D110008F8
:100070008D1100088D110008253B00088D11000826
:100080008D1100088D1100088D1100088D110008D8
:100090008D1100088D1100088D110008552D0008E4
:1000A0008D1100088D1100088D110008253E0008F3
:1000B000313E0008393E0008453E0008CD250008C5
:1000C0004D290008D1250008492900088D11000894
:1000D0008D110008593B0008953B00088D11000860
:1000E000811C00088D1100088D110008000000001F
:1000F0000000000000000000000000000000000000
:0C01000000000000000000005FF808F1A3
:1001100010B5054C237833B9044810B10448AFF347
:1001200000800121217010BDD405002000000000D6
:10013000BC4B010808B5064B1BB106480649AFF396
:1001400000800648016811B1054A02B1904708BD18
:1001500000000000BC4B0108D8050020D405002099
:100160000000000081F0004102E000BF83F0004386
:1001700030B54FEA41044FEA430594EA050F08BF42
:1001800090EA020F1FBF54EA000C55EA020C7FEA06
:10019000645C7FEA655C00F0E2804FEA5454D4EB83
:1001A0005555B8BF6D420CDD2C4480EA020281EA4D
:1001B000030382EA000083EA010180EA020281EA85
:1001C0000303362D88BF30BD11F0004F4FEA0131D7
:1001D0004FF4801C4CEA113102D0404261EB4101E6
:1001E00013F0004F4FEA03334CEA133302D052426C
:1001F00063EB430394EA050F00F0A780A4F1010428
:10020000D5F1200E0DDB02FA0EFC22FA05F2801861
:1002100041F1000103FA0EF2801843FA05F3594147
:100220000EE0A5F120050EF1200E012A03FA0EFCC6
:1002300028BF4CF0020C43FA05F3C01851EBE371F0
:1002400001F0004507D54FF0000EDCF1000C7EEB0D
:1002500000006EEB0101B1F5801F1BD3B1F5001F4B
:100260000CD349085FEA30004FEA3C0C04F101046A
:100270004FEA445212F5800F80F09A80BCF1004F93
:1002800008BF5FEA500C50F1000041EB045141EA15
:10029000050130BD5FEA4C0C404141EB010111F416
:1002A000801FA4F10104E9D191F0000F04BF0146C1
:1002B0000020B1FA81F308BF2033A3F10B03B3F19F
:1002C00020020CDA0C3208DD02F1140CC2F10C022F
:1002D00001FA0CF021FA02F10CE002F11402D8BF8D
:1002E000C2F1200C01FA02F120FA0CFCDCBF41EA59
:1002F0000C019040E41AA2BF01EB0451294330BD28
:100300006FEA04041F3C1CDA0C340EDC04F1140404
:10031000C4F1200220FA04F001FA02F340EA0300DB
:1003200021FA04F345EA030130BDC4F10C04C4F121
:10033000200220FA02F001FA04F340EA0300294601
:1003400030BD21FA04F0294630BD94F0000F83F44B
:10035000801306BF81F480110134013D4EE77FEA2E
:10036000645C18BF7FEA655C29D094EA050F08BF7A
:1003700090EA020F05D054EA000C04BF194610465B
:1003800030BD91EA030F1EBF0021002030BD5FEA9F
:10039000545C05D14000494128BF41F0004130BDC7
:1003A00014F580043CBF01F5801130BD01F000451B
:1003B00045F0FE4141F470014FF0000030BD7FEA8E
:1003C000645C1ABF194610467FEA655C1CBF0B4689
:1003D000024650EA013406BF52EA033591EA030FA0
:1003E00041F4002130BD00BF90F0000F04BF002198
:1003F000704730B54FF4806404F132044FF00005CB
:100400004FF0000150E700BF90F0000F04BF002143
:10041000704730B54FF4806404F1320410F00045A9
:1004200048BF40424FF000013EE700BF42004FEAA4
:10043000E2014FEA31014FEA02701FBF12F07F4321
:1004400093F07F4F81F06051704792F0000F14BF1E
:1004500093F07F4F704730B54FF4607401F0004562
:1004600021F0004120E700BF50EA010208BF7047B9
:1004700030B54FF000050AE050EA010208BF7047AE
:1004800030B511F0004502D5404261EB41014FF417
:10049000806404F132045FEA915C3FF4DCAE4FF01B
:1004A00003025FEADC0C18BF03325FEADC0C18BF02
:1004B000033202EBDC02C2F1200300FA03FC20FA53
:1004C00002F001FA03FE40EA0E0021FA02F11444A0
:1004D000C1E600BF70B54FF0FF0C4CF4E06C1CEAB5
:1004E00011541DBF1CEA135594EA0C0F95EA0C0F2A
:1004F00000F0DEF82C4481EA030621EA4C5123EA9D
:100500004C5350EA013518BF52EA033541F48011CB
:1005100043F4801338D0A0FB02CE4FF00005E1FB7E
:1005200002E506F00042E0FB03E54FF00006E1FBC8
:1005300003569CF0000F18BF4EF0010EA4F1FF040B
:10054000B6F5007F64F5407404D25FEA4E0E6D414B
:1005500046EB060642EAC62141EA55514FEAC5205C
:1005600040EA5E504FEACE2EB4F1FD0C88BFBCF5D8
:10057000E06F1ED8BEF1004F08BF5FEA500E50F189
:10058000000041EB045170BD06F0004646EA01014F
:1005900040EA020081EA0301B4EB5C04C2BFD4EB81
:1005A0000C0541EA045170BD41F480114FF0000E7A
:1005B000013C00F3AB8014F1360FDEBF002001F0E8
:1005C000004170BDC4F10004203C35DA0C341BDC62
:1005D00004F11404C4F1200500FA05F320FA04F034
:1005E00001FA05F240EA020001F0004221F0004168
:1005F00010EBD37021FA04F642EB06015EEA430EDB
:1006000008BF20EAD37070BDC4F10C04C4F120050A
:1006100000FA04F320FA05F001FA04F240EA0200BD
:1006200001F0004110EBD37041F100015EEA430E8E
:1006300008BF20EAD37070BDC4F1200500FA05F2AE
:100640004EEA020E20FA04F301FA05F243EA02032D
:1006500021FA04F001F0004121FA04F220EA02003C
:1006600000EBD3705EEA430E08BF20EAD37070BD82
:1006700094F0000F0FD101F00046400041EB010162
:1006800011F4801F08BF013CF7D041EA060195F044
:10069000000F18BF704703F00046520043EB0303FE
:1006A00013F4801F08BF013DF7D043EA06037047EB
:1006B00094EA0C0F0CEA135518BF95EA0C0F0CD0F6
:1006C00050EA410618BF52EA4306D1D181EA03013C
:1006D00001F000414FF0000070BD50EA410606BF36
:1006E0001046194652EA430619D094EA0C0F02D17B
:1006F00050EA013613D195EA0C0F05D152EA0336C0
:100700001CBF104619460AD181EA030101F00041DD
:1007100041F0FE4141F470014FF0000070BD41F026
:10072000FE4141F4780170BD70B54FF0FF0C4CF400
:10073000E06C1CEA11541DBF1CEA135594EA0C0F1F
:1007400095EA0C0F00F0A7F8A4EB050481EA030E6C
:1007500052EA03354FEA013100F088804FEA033353
:100760004FF0805545EA131343EA12634FEA022221
:1007700045EA111545EA10654FEA00260EF00041E2
:100780009D4208BF964244F1FD0404F5407402D234
:100790005B084FEA3202B61A65EB03055B084FEAC5
:1007A00032024FF480104FF4002CB6EB020E75EBC2
:1007B000030E22BFB61A754640EA0C005B084FEAEA
:1007C0003202B6EB020E75EB030E22BFB61A754667
:1007D00040EA5C005B084FEA3202B6EB020E75EBB2
:1007E000030E22BFB61A754640EA9C005B084FEA2A
:1007F0003202B6EB020E75EB030E22BFB61A754637
:1008000040EADC0055EA060E18D04FEA051545EA25
:1008100016754FEA06164FEAC30343EA52734FEACE
:10082000C2025FEA1C1CC0D111F4801F0BD141EA47
:1008300000014FF000004FF0004CB6E711F4801FAC
:1008400004BF01430020B4F1FD0C88BFBCF5E06F8C
:100850003FF6AFAEB5EB030C04BFB6EB020C5FEA9C
:10086000500C50F1000041EB045170BD0EF0004EF1
:100870004EEA113114EB5C04C2BFD4EB0C0541EA23
:10088000045170BD41F480114FF0000E013C90E620
:1008900045EA060E8DE60CEA135594EA0C0F08BFE4
:1008A00095EA0C0F3FF43BAF94EA0C0F0AD150EAE3
:1008B00001347FF434AF95EA0C0F7FF425AF104676
:1008C00019462CE795EA0C0F06D152EA03353FF49E
:1008D000FDAE1046194622E750EA410618BF52EA1B
:1008E00043067FF4C5AE50EA41047FF40DAF52EAEF
:1008F00043057FF4EBAE12E74FF0FF3C06E000BF8C
:100900004FF0010C02E000BF4FF0010C4DF804CD98
:100910004FEA410C7FEA6C5C4FEA430C18BF7FEA58
:100920006C5C1BD001B050EA410C0CBF52EA430C86
:1009300091EA030F02BF90EA020F0020704710F106
:10094000000F91EA030F58BF994208BF90422CBF95
:10095000D8176FEAE37040F0010070474FEA410C8E
:100960007FEA6C5C02D150EA013C07D14FEA430CAC
:100970007FEA6C5CD6D152EA033CD3D05DF8040B1D
:10098000704700BF8446104662468C46194663464F
:1009900000E000BF01B5FFF7B7FF002848BF10F126
:1009A000000F01BD4DF808EDFFF7F4FF0CBF01206B
:1009B00000205DF808FB00BF4DF808EDFFF7EAFFE7
:1009C00034BF012000205DF808FB00BF4DF808EDA2
:1009D000FFF7E0FF94BF012000205DF808FB00BF97
:1009E0004DF808EDFFF7CEFF94BF012000205DF821
:1009F00008FB00BF4DF808EDFFF7C4FF34BF01202E
:100A000000205DF808FB00BF4FEA4102B2F1E0436D
:100A100024BFB3F5001CDCF1FE5C0DD901F0004CE5
:100A20004FEAC0024CEA5070B2F1004F40EB830035
:100A300008BF20F00100704711F0804F21D113F161
:100A40003872BCBF01F00040704741F480114FEA9A
:100A50005252C2F11802C2F1200C10FA0CF320FA23
:100A600002F018BF40F001004FEAC1234FEAD32340
:100A700003FA0CFC40EA0C0023FA02F34FEA4303AA
:100A8000CCE77FEA625307D150EA01331EBF4FF033
:100A9000FE4040F44000704701F0004040F0FE404E
:100AA00040F40000704700BF80F0004002E000BF4B
:100AB00081F0004142001FBF5FEA410392EA030F49
:100AC0007FEA226C7FEA236C6AD04FEA1262D2EB93
:100AD0001363C1BFD218414048404140B8BF5B4298
:100AE000192B88BF704710F0004F40F4000020F031
:100AF0007F4018BF404211F0004F41F4000121F047
:100B00007F4118BF494292EA030F3FD0A2F1010290
:100B100041FA03FC10EB0C00C3F1200301FA03F1CE
:100B200000F0004302D5494260EB4000B0F5000FF1
:100B300013D3B0F1807F06D340084FEA310102F1B0
:100B40000102FE2A51D2B1F1004F40EBC25008BF62
:100B500020F0010040EA03007047490040EB00002C
:100B600010F4000FA2F10102EDD1B0FA80FCACF15B
:100B7000080CB2EB0C0200FA0CF0AABF00EBC2505A
:100B800052421843BCBFD0401843704792F0000F48
:100B900081F4000106BF80F400000132013BB5E79B
:100BA0004FEA41037FEA226C18BF7FEA236C21D011
:100BB00092EA030F04D092F0000F08BF0846704776
:100BC00090EA010F1CBF0020704712F07F4F04D144
:100BD000400028BF40F00040704712F100723CBF57
:100BE00000F50000704700F0004343F0FE4040F481
:100BF000000070477FEA226216BF08467FEA23633F
:100C00000146420206BF5FEA412390EA010F40F429
:100C1000800070474FF0000304E000BF10F0004375
:100C200048BF40425FEA000C08BF704743F096435C
:100C300001464FF000001CE050EA010208BF704777
:100C40004FF000030AE000BF50EA010208BF7047FE
:100C500011F0004302D5404261EB41015FEA010C13
:100C600002BF84460146002043F0B64308BFA3F10B
:100C70008053A3F50003BCFA8CF2083AA3EBC253ED
:100C800010DB01FA02FC634400FA02FCC2F120020C
:100C9000BCF1004F20FA02F243EB020008BF20F043
:100CA0000100704702F1200201FA02FCC2F12002A9
:100CB00050EA4C0021FA02F243EB020008BF20EA9E
:100CC000DC7070474FF0FF0C1CEAD0521EBF1CEACC
:100CD000D15392EA0C0F93EA0C0F6FD01A4480EABA
:100CE000010C400218BF5FEA41211ED04FF00063A3
:100CF00043EA501043EA5111A0FB01310CF00040CF
:100D0000B1F5000F3EBF490041EAD3715B0040EAF4
:100D1000010062F17F02FD2A1DD8B3F1004F40EBC4
:100D2000C25008BF20F00100704790F0000F0CF097
:100D3000004C08BF49024CEA502040EA51207F3A5B
:100D4000C2BFD2F1FF0340EAC250704740F4000036
:100D50004FF00003013A5DDC12F1190FDCBF00F027
:100D600000407047C2F10002410021FA02F1C2F1D5
:100D7000200200FA02FC5FEA310040F1000053EA71
:100D80004C0308BF20EADC70704792F0000F00F0BF
:100D9000004C02BF400010F4000F013AF9D040EAC5
:100DA0000C0093F0000F01F0004C02BF490011F459
:100DB000000F013BF9D041EA0C018FE70CEAD15357
:100DC00092EA0C0F18BF93EA0C0F0AD030F0004CD7
:100DD00018BF31F0004CD8D180EA010000F000408B
:100DE000704790F0000F17BF90F0004F084691F049
:100DF000000F91F0004F14D092EA0C0F01D1420283
:100E00000FD193EA0C0F03D14B0218BF084608D14B
:100E100080EA010000F0004040F0FE4040F4000095
:100E2000704740F0FE4040F4400070474FF0FF0C28
:100E30001CEAD0521EBF1CEAD15392EA0C0F93EA6F
:100E40000C0F69D0A2EB030280EA010C49024FEAC1
:100E5000402037D04FF0805343EA111143EA10137A
:100E60000CF000408B4238BF5B0042F17D024FF432
:100E7000000C8B4224BF5B1A40EA0C00B3EB510F0D
:100E800024BFA3EB510340EA5C00B3EB910F24BFF6
:100E9000A3EB910340EA9C00B3EBD10F24BFA3EB7B
:100EA000D10340EADC001B0118BF5FEA1C1CE0D143
:100EB000FD2A3FF650AF8B4240EBC25008BF20F0F6
:100EC000010070470CF0004C4CEA50207F32C2BF4A
:100ED000D2F1FF0340EAC250704740F400004FF0E7
:100EE0000003013A37E792F0000F00F0004C02BF18
:100EF000400010F4000F013AF9D040EA0C0093F0E2
:100F0000000F01F0004C02BF490011F4000F013B3B
:100F1000F9D041EA0C0195E70CEAD15392EA0C0FA3
:100F200008D142027FF47DAF93EA0C0F7FF470AFDB
:100F3000084676E793EA0C0F04D14B023FF44CAF1E
:100F400008466EE730F0004C18BF31F0004CCAD1B3
:100F500030F000427FF45CAF31F000437FF43CAFEF
:100F60005FE700BF4FF0FF3C06E000BF4FF0010C11
:100F700002E000BF4FF0010C4DF804CD4FEA4002F3
:100F80004FEA41037FEA226C18BF7FEA236C11D03D
:100F900001B052EA530C18BF90EA010F58BFB2EBF0
:100FA000030088BFC81738BF6FEAE17018BF40F070
:100FB000010070477FEA226C02D15FEA402C05D124
:100FC0007FEA236CE4D15FEA412CE1D05DF8040BA9
:100FD000704700BF844608466146FFE70FB5FFF73C
:100FE000C9FF002848BF10F1000F0FBD4DF808EDF4
:100FF000FFF7F4FF0CBF012000205DF808FB00BFE5
:101000004DF808EDFFF7EAFF34BF012000205DF83E
:1010100008FB00BF4DF808EDFFF7E0FF94BF01208B
:1010200000205DF808FB00BF4DF808EDFFF7D2FF88
:1010300094BF012000205DF808FB00BF4DF808EDCB
:10104000FFF7C8FF34BF012000205DF808FB00BF98
:101050004FEA4002B2F1FE4F0FD34FF09E03B3EBC5
:1010600012620DD94FEA002343F0004310F0004F05
:1010700023FA02F018BF404270474FF0000070475B
:1010800012F1610F01D1420205D110F0004008BFFA
:101090006FF0004070474FF00000704742000ED2E2
:1010A000B2F1FE4F0BD34FF09E03B3EB126209D4A3
:1010B0004FEA002343F0004323FA02F070474FF059
:1010C0000000704712F1610F01D1420202D14FF0CE
:1010D000FF3070474FF00000704700BF1D481E49A9
:1010E000026800608A4200F01F80002100F004B80E
:1010F0001A4B5B584350043119481A4B42189A4214
:10110000FFF4F6AF184A00F003B8002342F8043B9E
:10111000164B9A42FFF4F9AF0BF0D4FB0FF050FAE4
:1011200004F0A4F9FFF7FEBF114E124830601248D8
:10113000016821F070610160410201600F4C1820CC
:1011400020600F490F4808600F48D0F800D0406871
:1011500000470000F04F0020EFBEADDEE04B01087D
:1011600000000020D4050020D40500205C200020D1
:10117000181002400900000004000140140C014056
:10118000000C01404434434400F0FF1FFFF7FEBF52
:101190002E4B2DE9F34105461878002838D000245D
:1011A00026462746A0463221082253206B4601F0EE
:1011B000A9FA9DF801109DF80000013400EB01230D
:1011C0009DF803109DF802001AB200EB01239DF870
:1011D00005109DF80400E4B290441AB200EB01231C
:1011E0009DF80710BF18202C1AB2164401F07F009A
:1011F00001D00028D7D1164B98FBF4F897FBF4F7F1
:1012000096FBF4F6A5F800806F80AE801C701AE0A3
:10121000322106226B46532001F074FA9DF801201A
:101220009DF800109DF8030001EB02239DF80220B9
:101230002B8002EB00219DF804309DF805006980A9
:1012400003EB0022AA80BDE8FC8100BFF00500206E
:10125000F105002008B5134B53201B782D210822DF
:101260007BB101F013FB31210A22532001F00EFB68
:101270002C210C22532001F009FB5320382190220D
:1012800009E001F003FB31210A22532001F0FEFAAC
:1012900053202C210A2201F0F9FA034840F20912E6
:1012A000028008BDF00500201200002037B5104B69
:1012B00005461A680F480C46002182428DF8071037
:1012C00001D1002013E0532001220DF1070301F0AA
:1012D00019FA0028F5D09DF80710E529F1D12A78F0
:1012E0000548064B064920601A70616001203EBD2A
:1012F00084010020001BB70055120008F0050020F3
:101300009111000813B50622044602216B461820ED
:1013100001F0F8F99DF800309DF8012098089DF83B
:10132000023000EB02219DF8032098089DF804305C
:10133000218000EB02219DF805209808618000EBD8
:101340000221A1801CBD000008B50F210822182031
:1013500001F09CFA0E221820102101F097FA024B9E
:101360004FF480521A8008BD1200002037B50024C7
:1013700002AB054603F8014D18202146012201F079
:10138000C1F950B19DF80730FB2B05D10348044942
:1013900028606960012000E020463EBD4913000836
:1013A0000513000813B506220446A8216B466820E1
:1013B00001F0A8F99DF800209DF8013043EA0220D1
:1013C00001B2042391FBF3F29DF802009DF8031093
:1013D000228041EA002210B290FBF3F19DF8052033
:1013E0009DF80400618042EA002108B290FBF3F30B
:1013F000A3801CBD08B5642005F05FFB6820232195
:10140000F02201F043FA10B9032005F0F5FB0520A6
:1014100005F053FB044B68201A78202142F00F029C
:10142000BDE8084001F032BAF205002037B50546A4
:1014300019200C4605F041FB68200F2101220DF117
:10144000070301F05FF99DF80730D32B16D10C4844
:101450000C490D4A4E2C28606960EA600B4B07D09E
:101460005D2C09D0362C01D0002002E0402000E0A5
:1014700080201870012002E0C020FAE700203EBD65
:10148000F5130008A5130008DDE9A731F2050020D7
:1014900013B50622044601216B461C2001F032F9E7
:1014A0009DF800209DF8013043EA022040F38D01B1
:1014B000042391FBF3F29DF802009DF803102280B3
:1014C00041EA002242F38D0090FBF3F19DF80520E4
:1014D0009DF80400618042EA002141F38D0090FBF9
:1014E000F3F3A3801CBD000013B5042120230224C4
:1014F0008DF806101A486944ADF804308DF807409D
:1015000001F054FB2A2100221C2001F0BFF90E211A
:101510001C20224601F0BAF90F2103221C2001F001
:10152000B5F92B2112221C2001F0B0F92C211C202E
:10153000224601F0ABF92D2101221C2001F0A6F971
:101540002E2100221C2001F0A1F905221C202A21B5
:1015500001F09CF903484FF4807202801CBD00BF6B
:10156000000801401200002013B50446104811493C
:10157000026800238A428DF8073001D1002015E06F
:101580001C200D2101220DF1070301F0BBF80028FA
:10159000F4D09DF807302A2B01D01A2BEED1064843
:1015A000064A0749206062600B7001201CBD00BF25
:1015B00084010020001BB700E91400089114000802
:1015C000F305002013B5022204461B2101AB68205D
:1015D00001F098F89DF804209DF8053043EA0220B8
:1015E00000F54E5110314FF48C7291FBF2F323331E
:1015F00023801CBD13B5062204461D216B466820BE
:1016000001F080F89DF800209DF8013043EA0220A7
:1016100001B2042391FBF3F29DF802009DF8031040
:10162000228041EA002210B290FBF3F19DF80520E0
:101630009DF80400618042EA002108B290FBF3F3B8
:10164000A3801CBD08B5192005F037FA68201521C4
:10165000002201F01BF910B9032005F0CDFA0C4B64
:1016600016211A78682042F0180201F00FF91721AC
:101670000022682001F00AF93D210122682001F0D2
:1016800005F968203E210122BDE8084001F0FEB8BE
:101690000000002038B5054619200C4605F00DFA6B
:1016A00068201521002201F0F1F818B3124B1348FD
:1016B0001349144A622C2B606860A960EA60124BDF
:1016C0000FD004D80A2C12D0142C0CD10DE0BC2C55
:1016D00004D0B4F5807F06D1002009E00120187005
:1016E00038BD022004E0032002E0042000E00520D1
:1016F0001870012038BD00BF45160008F515000818
:10170000C51500081844923100000020064B1878D7
:1017100020B1012806D14FF4805201E04FF400625D
:1017200002490A80704700BFF40500201200002023
:1017300007B5232005F0C1F96820752101220DF1BC
:10174000070300F0DFFF30B19DF80700B0F1680338
:10175000594251EB03000EBD13B506220446432146
:101760006B46682000F0CEFF9DF800209DF8013008
:1017700043EA022001B2042391FBF3F29DF8020038
:101780009DF80310228041EA002210B290FBF3F191
:101790009DF805209DF80400618042EA002108B20E
:1017A00090FBF3F3A3801CBD13B5062204463B2136
:1017B0006B46682000F0A6FF9DF800209DF80130E0
:1017C0009DF8021043EA02209DF80320208042EA9F
:1017D00001239DF804009DF80510638041EA002272
:1017E000A2801CBD07B5204A02204FF40053ADF87B
:1017F00004308DF8070013681C48042183428DF8DB
:10180000061001D11A4803E01A498B4203D11A4845
:1018100001A901F0CBF96B218022682001F036F894
:10182000052005F04AF919210022682001F02EF860
:101830006B210322682001F029F837210222682059
:1018400001F024F80D4A1A216820127801F01EF8E0
:101850001B211822682001F019F868201C21102291
:1018600001F014F80EBD00BF8401002000127A00C0
:10187000000C0140001BB7000010014001000020D7
:1018800030B585B00446FFF753FF002841D006214C
:101890000A46682002AB00F035FF9DF80B309DF83A
:1018A0000D5003F0010105F001004A0042EA8005F5
:1018B0009DF8090000F001031D4307D0012D1648D3
:1018C00001D1002318E0022D0CD114E00C21682076
:1018D00001220DF1070300F015FF9DF8071011F02C
:1018E0000F0203D1052005F087F906E0042A0A4813
:1018F00001D1057001E0012303700748074903780F
:10190000074A2160002B14BF6E216F216260217293
:10191000012005B030BD00BFF40500200D17000800
:10192000A917000838B505460C46FFF701FF28B394
:10193000134B14481449142C2B606860E960134B56
:1019400015D004D8052C16D00A2C0ED111E0BC2CD1
:1019500008D0B4F5807F03D0622C06D102220BE0C0
:10196000002209E00120187038BD032204E004229F
:1019700002E0052200E006221A70012038BD00BFF7
:10198000E51700085917000819449231010000209A
:10199000044B054903EB4000427831F8123098B20D
:1019A000704700BF7E1500207815002070B5424BAF
:1019B00004221A70414A424D11782E68414D4C1C48
:1019C000E4B2AE4290B05970147004D105259D70F8
:1019D000DC708B1C1370007830B1384C364922789B
:1019E0000871551C4A712570344D37480BF0A4FF1F
:1019F000297836480024364B01298CBF80222246A4
:101A0000069008914FF48060202105930A924FF4CC
:101A100080734FF400520C900D912B4805A90B9345
:101A20000E92079409940F940BF0FEFF26480121B3
:101A30000CF027F82B784FF46022012B94BF002084
:101A4000012001218DF804008DF805102148694618
:101A50000094029203948DF810300BF00BF9174BA1
:101A60001878A0420AD914491A4811F81410013400
:101A7000E4B2224603230BF04EF9F0E715480121AA
:101A80000BF025F9134801210BF018F911480BF060
:101A900027F910480BF029F90028FAD10D480BF06E
:101AA00028F90C480BF02AF90028FAD1094801213D
:101AB0000BF028F910B070BD7E150020F505002050
:101AC00084010020001BB7000800024078150020A8
:101AD0004C24014000240140334B2DE9F0411C8887
:101AE000324B5A891E89A51A7543B3F91240B3F9CE
:101AF0001420EF13BE18E50295FBF6F43F19A7F585
:101B00007A6202FB02F4B3F90480B3F902C00A2539
:101B10007D43DF6102FB0CFCB3F90E7002FB08F29F
:101B2000B3F90C802413674304FB08F4241404EB7A
:101B30006232941CA210DC88083502F50042624330
:101B40002E114FEAEC24B3F92050B3F9003004EB26
:101B5000E72404EB830303FA05F39C1C144BD20B1C
:101B60001B68A3EBA4044CF2503343FA05F3634320
:101B700003D45C00B4FBF2F302E0B3FBF2F25300D7
:101B80001A12524340F6DE3462430A4C5C4324147A
:101B900004EB224202F6CF6203EB221300B1036092
:101BA00001B10E60BDE8F08126060020FC05002092
:101BB0002006002043E3FFFF104B07B5187818B943
:101BC0000F490A88531C0B80F621032201AB7720B2
:101BD00000F098FD9DF805109DF804000A020949DF
:101BE00042EA00409DF80630B1F920201843C2F1C6
:101BF000080320FA03F0044908600EBDF605002032
:101C0000F8050020FC050020200600200B4B07B53E
:101C1000187818B90A490A88531C0B80F621022249
:101C200001AB772000F06EFD9DF804009DF80510D3
:101C3000044B41EA00221A800EBD00BFF6050020C9
:101C4000F805002026060020064B074893F82020C0
:101C5000002192013432017002F0FC027720F4215D
:101C600000F014BEFC050020F6050020034B002206
:101C70001A707720F4212E2200F008BEF60500200D
:101C800010B54FF480400AF077FF0128044605D1D3
:101C90004FF480400AF080FF014B1C7010BD00BF64
:101CA000F60500202DE9F0476B4B05461A686B4896
:101CB0008CB0824200F0CA80DFF8C0A19AF80080A0
:101CC000B8F1000F40F0C480654F102102264FF498
:101CD00000598DF80A10384602A94FF480448DF857
:101CE0000B60ADF8089000F061FF0423384602A9AC
:101CF0008DF80A30ADF8084000F058FF0E2130464C
:101D0000C7F8109000F08EFF0126082204A88DF875
:101D1000152004948DF814808DF816600AF0F0FEFA
:101D200028200F218DF80C0003A88DF80D108DF8D8
:101D30000E108DF80F600BF045F8142004F0BDFE76
:101D40007720D02132460DF1070300F0DBFC9DF82F
:101D50000730444C0322552BE375228418BFC7F883
:101D6000149073D1D12132460DF10703772000F092
:101D7000C9FC9DF80700162200F00F010309217627
:101D80006376AA2106AB772000F0BCFC9DF81820F2
:101D90009DF819009DF81B3040EA02219DF81A2099
:101DA000218043EA02209DF81C109DF81D206080D0
:101DB00042EA01239DF81E009DF81F10A38041EA0E
:101DC00000229DF821309DF82000E28043EA0021A6
:101DD0009DF822209DF82300218140EA02239DF8EE
:101DE00024109DF82520638142EA01209DF82730C8
:101DF0009DF82610A08143EA01229DF828009DF855
:101E00002910E28141EA00239DF82A209DF82B0049
:101E1000238240EA02219DF82D309DF82C2061821A
:101E200043EA0220104B41F2707146F67812A0820C
:101E30008AF800600D4829806A806B600C490D4A61
:101E40000D4BA860E9602A616B6101E0002000E0B1
:101E500001200CB0BDE8F08784010020001BB70012
:101E600000100140FC0500206D1C00080D1C00083E
:101E7000491C0008B91B0008D91A000824060020D4
:101E80002DE9F04F4E4E4F4B85B07789039119687D
:101E90003289844638020F1A87FB0201C00940EAE2
:101EA0004162CB11F188B48887FB0101240400252D
:101EB00014EB020845EB0309000A40EA01620B1229
:101EC000B189748887FB0101E403002514EB020A41
:101ED00045EB030BC00D40EA41224FF4FA60CB15ED
:101EE0000021801841EB0301CDE90001B0F5FA6F44
:101EF00071F1000147DAA2FB024502FB03F605EB94
:101F00004607B80040EA9471A0002646241847EB23
:101F1000010569104FEA3400A408B8EB000869EB2A
:101F20000109A91044EA8570BAEB000A6BEB010BBA
:101F300025484FF0FF31DDE9004584428D4122DA2A
:101F400040F6AC500021801841EB03014143A0FB57
:101F500000236FF0060003EB4103544200FB0344EF
:101F6000A2FB000118EB0008214449EB01090B24F6
:101F7000A2FB040104FB031149104FEA3000BAEB45
:101F8000000A6BEB010B114A1368A3FB0A0103FB68
:101F90000B11400D40EAC1224B15B2EB080263EB76
:101FA0000903D20B42EA4343BCF1000F01D0CCF845
:101FB0000030039808B10099016005B0BDE8F08FCA
:101FC000300600202C06002024FAFFFF28060020FF
:101FD00007B50021032201AB772000F093FB9DF8A9
:101FE00005009DF8043001029DF8062041EA0340F7
:101FF00010430EBD08B5FFF7EBFF014B186008BD9D
:102000002806002008B5FFF7E3FF014B186008BD64
:102010002C06002077204821012200F037BC7720D1
:102020005821012200F032BC454B73B51A680446B2
:10203000444882420FD010258DF80650424D0221AF
:102040004FF400568DF80710284601A9ADF804603A
:1020500000F0ACFD6E610A2004F02FFD7720A02176
:1020600001220DF1030300F04DFB002866D01E2174
:102070000122772000F00AFC4FF42F6004F012FDDB
:102080000025A5F160030026D9B20222772001AB1A
:102090008DF804608DF8056000F034FB9DF8042095
:1020A0009DF80500294B40EA0221E9520235102D26
:1020B000E7D1DA8902F47F4502F00F00DD81324674
:1020C00001232249515A0232002918BF0023102A45
:1020D000F7D113BB1A4612F0010F1C494FEA6206F2
:1020E00004D011F816104B40082104E031F8161006
:1020F00083EA1123F8E713F4004F18BF83F4C053A9
:102100005B000139F7D10132102AE4D10F49C3F342
:10211000033305439842CD8101D000200EE00C4AE4
:1021200042F210702080608062600A480A490B4BBE
:102130000B4A2061A160E360626101207CBD00BFA9
:1021400084010020001BB700001001403006002071
:102150001F200008F51F00080520000815200008B2
:10216000811E0008F8B5134B05469B890E461446A0
:10217000ECB116B116F8017B00E0FF270D480221F3
:102180000AF072FD0028F9D00A4839460AF067FDC6
:10219000084801210AF068FD0028F9D005480AF036
:1021A00060FDC0B20DB105F8010B013CE0E7012074
:1021B000F8BD00BF003800402DE9F047012188B08C
:1021C0004FF480400BF0B4FA374C01214FF48040BB
:1021D0000BF0C6FA03214FF420401823ADF800009D
:1021E0008DF80310204669468DF802304FF0040840
:1021F00000F0DCFC2D4E4FF4804220466946ADF8DD
:1022000000204FF480554FF0100A8DF8028000F046
:10221000CDFC69462046ADF800508DF802A000F0D4
:10222000C5FC30460AF0BEFC07214FF400700023C5
:102230000222ADF81600ADF81C104FF0010930462F
:1022400003A94FF48277ADF80C30ADF81030ADF83B
:102250001A30ADF81220ADF80E70ADF814901F468C
:10226000ADF818A00AF0D0FC304649460AF0EBFC65
:102270009F238DF804308DF805708DF806708DF869
:1022800007700DEB08014246656102A8FFF76AFF7F
:1022900025619DF80900B0F1EF014A4252EB0100BF
:1022A00008B0BDE8F08700BF000C014000380040D6
:1022B0002DE9F84F9C4C2068838A9BB213F00102F1
:1022C00039D0018821F400631A04110C0180012126
:1022D0000BF010FB954A964B117800201870D9B17D
:1022E000944803781BB9944A1178FF2914D101232B
:1022F000037092480278022A06D18B490B6818882D
:1023000082B242F4006119808D4B874819780068C9
:1023100001220BF009FB2FE18948834B0178002251
:1023200018680BF001FB844A1178FF2900F0248122
:10233000FF207F4BDEE003F00201C9B200293DD04F
:10234000BFF35F8F7D4D2E78012E354616D177492C
:102350000B789BB177490B7883B111460BF0CAFA21
:10236000BFF35F8F20683146038B0BF0B7FA754AD5
:10237000206816704FF480613246FBE0038BBFF398
:102380005F8F6E490A78022A09D1684B1A7832B1F8
:10239000684B1A781AB100210BF0ACFAE5E0097825
:1023A000032907D1614B1A7822B162490B78002BBF
:1023B00040F0DD804FF480610122DBE003F0040691
:1023C000F6B2002E71D0594BDFF878811A780126C9
:1023D00088F80060574B002A4DD01A78002A4AD05E
:1023E000564D2F78524D022F574F29D90BF082FAB4
:1023F000206895F80090D7F800A00BF092FA4FFAF9
:1024000089FB0AF80B0009EB0600314628702068AA
:102410000BF064FA206888F800603F6895F8008047
:102420000BF07FFA4FFA88F907F80900B0442068EA
:102430004FF48061324685F800800BF067FA2BE09C
:1024400031460BF04BFA20682E78D7F800800BF05D
:1024500068FA4FFA86F9731C08F80900D9B22068A7
:102460004FFA81F83F6829700BF05BFA033607F8E2
:1024700008002E7010E01B78012113B9334A13783D
:102480002BB10BF02BFA2A480278511C03E00BF019
:1024900019FA284801210170234A11680B8803F4B6
:1024A000807082B2002AF9D166E003F040010F4645
:1024B0001F4D09B3244B2F78D3F800800BF031FA6D
:1024C0004FFA87F908F80900781CC1B229701B4D32
:1024D0004FB22A780337BA4205D120684FF48061A1
:1024E00032460BF013FA124B28781A7851B2884210
:1024F00042D1501C18703FE01B063DD52B785EB2D0
:10250000721C27D0124901330A682B70915D0BF0C1
:1025100006FA0A4895F90020017891422CD12068EA
:102520004FF480613A4625E0580600205506002009
:10253000540600204C0600204406002045060020DA
:102540005D060020430600204806002042060020C9
:1025500050060020154A297011780BF0E0F9144854
:10256000017811B9134B1A7832B9134800684FF447
:10257000806100220BF0CAF90E4A104B117893F9D2
:1025800000004A1C90420ED10D4B0E4918780022D3
:102590000A7028B1084908684FF440710BF0B6F989
:1025A000094B00221A70BDE8F88F00BF44060020D6
:1025B000550600204506002058060020540600203D
:1025C000430600204C0600205C060020FFF770BE8A
:1025D000FFF76EBEF0B5484C89B04FF440651C2340
:1025E00007460226204602A9ADF808508DF80A30A9
:1025F0008DF80B6000F0DAFA4048142107608DF87E
:102600000E10204603A9ADF80C508DF80F6000F0B5
:10261000CDFA25610825384CA268520503D40A205A
:1026200004F040FAF7E74FF480660A20666104F090
:1026300039FA6F1E0A20266104F034FA17F0FF05FC
:10264000E9D14FF4006767610A2004F02BFA666154
:102650000A2004F027FA26610A2004F023FA022057
:1026600027611C218DF80F002046244C4FF4406355
:102670008DF80E1003A9ADF80C3000F097FA206821
:102680000BF082F804A80BF003F920682A464FF4F7
:1026900040710BF03BF91A484FF480434BF6FF7240
:1026A000049001212068ADF81C30ADF81620ADF87B
:1026B00014500BF0FBF804A920680BF07FF84FF4DE
:1026C000A0600AF075FB2221012201A88DF80410F8
:1026D0008DF805508DF806508DF807200AF072FB32
:1026E000212301A82E468DF804308DF805500AF0FC
:1026F00069FB09B0F0BD00BF000C01405806002086
:10270000801A060010B54000244CC0B22070244846
:10271000244C017000212170234C01202070234C97
:102720002360234C2360234B1A70234A10702348E4
:10273000017023490868838803F4007291B2A1B93B
:10274000038803F4807291B241B9038803F40072E4
:1027500091B20029F9D101210BF0B4F818484FF4D7
:102760004071006801220BF0D1F847F23053124A51
:10277000117811B1013BFAD100E053B911490A882F
:10278000501C83B20B800E490868FFF723FF00201E
:1027900010BD0A4B187880F0010010BD5D060020C6
:1027A000440600204206002055060020480600206E
:1027B00050060020450600205C0600204D06002043
:1027C000580600204006002010B54000244CC0B23E
:1027D00020702448244C01702449012008700021F5
:1027E0002170234C2360234C2360234B1A70234A0F
:1027F00010702348017023490868838803F400722D
:1028000091B2A1B9038803F4807291B241B90388EF
:1028100003F4007291B20029F9D101210BF052F8B2
:1028200018484FF44071006801220BF06FF847F22E
:102830003053124A117811B1013BFAD100E053B97B
:1028400011490A88501C83B20B800E490868FFF7B3
:10285000C1FE002010BD0A4B187880F0010010BDA9
:102860005D06002044060020550600204206002098
:102870005006002048060020450600205C06002087
:102880004D060020580600204006002007B502AB88
:1028900003F8012D0122FFF797FF0EBD274B37B537
:1028A0001868818A8AB20192019B13F4706F02D07A
:1028B000234A01211170019B13F4E06F31D04FF4D2
:1028C00080610022038B0BF021F80198810528D448
:1028D0001A4D2868018801F4007293B20BBB04887A
:1028E00004F480718CB29CB1028802F4807399B2B6
:1028F0000029F9D101210AF0F1FF1048006802888F
:1029000002F4007399B20029F9D1FFF763FE08E0E1
:1029100001210AF0E3FF28684FF4407122460AF0D3
:10292000F5FF06480268938A23F470610804030CDB
:102930000449938200220A703EBD00BF5806002061
:102940004D0600205C060020FFF7A8BFFFF7A6BFDA
:10295000014B188880B270474006002007B500225E
:1029600002AB03F8012D1E200A210122FFF7CAFE47
:1029700030B19DF80700B0F14803594251EB030014
:102980000EBD000037B50622044603216B461E200B
:10299000FFF7B8FE9DF801309DF80000154D43EAA1
:1029A000002108B2FEF73AF92968FEF78BF9FEF725
:1029B0004FFB9DF8022020809DF8030040EA02238F
:1029C00018B2FEF72BF9A968FEF77CF9FEF740FB79
:1029D0009DF805209DF80410A08042EA012000B275
:1029E000FEF71CF96968FEF76DF9FEF731FB6080B0
:1029F0003EBD00BF040000202DE9FF41634B644A47
:102A0000186890420DD104274FF480550226ADF886
:102A100004508DF807608DF806705E480DEB0701D5
:102A200008E05D49884207D104A94FF480445B481F
:102A300021F80C4D00F0BAF8322004F03EF80021E5
:102A400011221E20FFF722FF012160221E20FFF726
:102A50001DFF642004F031F802A8FFF793FF002463
:102A60000A2527462646012202211E20FFF70EFFD7
:102A7000322004F022F802A8FFF784FFBDF9080015
:102A8000BDF90A20BDF90C3024188242B8BF1046A7
:102A9000F6189842B8BF034613F5805F174409DD66
:102AA0003C49013DC86880F01002CA60DBD14FF09C
:102AB000010801E04FF000081E2000211222FFF75C
:102AC000E5FE0A25022101221E20FFF7DFFE32204B
:102AD00003F0F3FF02A8FFF755FFBDF90800BDF9A9
:102AE0000A10BDF90C30241A8142B8BF0846F61A04
:102AF0009842B8BF034613F5805FC1EB070707DDB7
:102B00002448013DC26882F01001C160DAD101E0C1
:102B10004FF000082046FEF781F801462048FEF7F6
:102B200085F9204D20F000432B603846FEF776F8FB
:102B300001461B48FEF77AF920F0004068603046F5
:102B4000FEF76CF801461848FEF770F920F00042D5
:102B5000AA60002170221E20FFF798FE012120228A
:102B60001E20FFF793FE1E2002210022FFF78EFE9B
:102B7000642003F0A2FFB8F1000F04D14FF07E51A2
:102B800029606960A960BDE8FF8100BF8401002061
:102B900000127A00000C0140001BB7000010014039
:102BA00000406F460400002001C05E462DE9F04160
:102BB0000F88002347FA03F2D2072DD58A7803F055
:102BC0000705DC08AD0012F0100F18BF91F803C024
:102BD00002F00F0618BF46EA0C064FF00F0C0CFA75
:102BE00005FC06FA05F550F82480282A28EA0C0C82
:102BF00045EA0C0540F8245006D1012202FA03F2FE
:102C0000C46824EA020206E0482A05D1012202FA39
:102C100003F2C4682243C2600133102BCAD1BDE85D
:102C2000F081000001F0030230B592000F2404FA95
:102C300002F400FA02F0074B8908023153F82150E0
:102C400025EA040443F8214053F82140044343F8A3
:102C5000214030BD000001407FB5274C0E4623784F
:102C60009BB9264A7A21B2F900000222C0F1B403CE
:102C70008DF8041093FBF2F18DF8051001AB6D2077
:102C8000FF21FFF7A1FD012334E0012B1DD17925A0
:102C90008DF804500A2592FBF5F00021B4225A3039
:102CA00001F0ECFE8DF8050096FBF5F00021B42252
:102CB0005A3001F0E3FE01AB8DF80600FF216D20D4
:102CC0000322FFF781FD022314E0022B13D101221E
:102CD000002814BF1046002064218DF804108DF8E0
:102CE00005208DF8060001AB6D20FF210322FFF7C0
:102CF0006BFD002323707FBD5E060020021F0020B5
:102D00000E4B0F4A9868118810B501420D4C03D044
:102D100003F0A8FE20600BE003F0A4FE23689842B5
:102D200006D9094AC01A12683B2190FBF1F31360DF
:102D3000064A1068BDE8104009F02EBF000C0140A3
:102D400064060020740600206C060020680600203F
:102D5000FFF7D6BFFFF7D4BF30B52F4B85B02F4A52
:102D600050B1012816D12E4C2E4D0221188028700A
:102D70001180216007200BE04FF4807119804FF41F
:102D800000731380274D264A092413602C701720E6
:102D9000254908702048214D038802221024234829
:102DA00001A98DF80720ADF804308DF80640FFF733
:102DB000FDFE29880423ADF804101C480DEB030127
:102DC0008DF80630FFF7F2FE164A154D11780120F6
:102DD000FFF728FF286809F0DFFE2868002102902D
:102DE0008DF80D4002A801248DF80C108DF80E40CE
:102DF00009F086FE0C4B1A7802F01F0304FA03F464
:102E000050B20B4A410942F8214003F045FE0949FE
:102E10003C38086005B030BD700600206406002014
:102E2000680600206706002066060020000C0140AE
:102E300000E100E06006002038B5044603F02CFEF7
:102E4000084B19683C3188420BD31860064D07487F
:102E50002A880460064C0B20226103F023FE2B8895
:102E6000636138BD60060020700600206C060020FB
:102E7000000C01402DE9F843044683796278002B69
:102E800014BF0220002002B101303A49002551F858
:102E90002090A8462F462E4619F80620FF2A02F059
:102EA0000F0002F0F00363D0A17811B1811E012957
:102EB0005BD9E17811B1011F032956D9E17909B134
:102EC000814252D002F02002D1B219B12278002AF8
:102ED00008BF002303F01001CAB21AB161780029BB
:102EE00008BF0023227932B1A17921B9A0F10802EB
:102EF000012A98BF8023617929B1A2791AB9011FEB
:102F0000032998BF802303F01002D1B211B100F061
:102F1000CDF92AE003F02002D1B221B1F9B200F0DC
:102F20008FF9013721E003F04002D1B281B122894B
:102F3000114B4FEA0010B2F5FA7F1844E9B2A389A9
:102F400002D900F0E3F801E000F0F6F801350CE0FA
:102F50001B060AD5084B5FFA88F103EB0010628963
:102F6000E38900F0FFF808F1010801360E2E93D135
:102F7000BDE8F8831823010878230108074BA1F561
:102F80007A7153F82000838802684B434FF47A70BB
:102F900093FBF0F18BB21380704700BF7C060020DA
:102FA000024B53F820000268118070477C06002015
:102FB0002DE9F04F044647488E46057889B0691CD4
:102FC0000170914611462068724601930C2600F06C
:102FD00077FEA268182303A96E4360684FF0020AC7
:102FE000ADF80C208DF80E308DF80FA0FFF7DEFD48
:102FF00004A8394F256894F80CB00AF0D8F870206E
:10300000019BADF81000012100224FF4807007EB06
:103010000608ADF81210ADF81420ADF81630ADF872
:1030200018A0ADF81C00BBF10C0F2BD8DFE80BF09B
:10303000072A2A2A102A2A2A192A2A2A2200284656
:1030400004A909F0ADFF284608210AF0E5F819E0C7
:10305000284604A909F0E8FF284608210AF0E4F808
:1030600010E0284604A90AF023F8284608210AF0AF
:10307000E5F807E0284604A90AF05CF8284608218C
:103080000AF0E4F8A17B19B1206801210AF0ADF83B
:10309000206801210AF09DF8237B0C2B14D8DFE86F
:1030A00003F0071313130A1313130D131313100054
:1030B0002268343207E02268383204E022683C3269
:1030C00001E022684032BA51A8F80490404609B0A5
:1030D000BDE8F08F78060020CC06002008B5044B30
:1030E00053F820301BB10B2801D89A68904708BDCF
:1030F0007C060020044B53F820201AB107289CBFFF
:1031000012681180704700BFAC06002010B50C4655
:103110000649B1FBF2F292B20821FFF749FF044BD6
:10312000044943F82400816010BD00BF00127A00FA
:103130007C0600207D2F000810B50C460649B1FB27
:10314000F2F292B20121FFF733FF044B044943F836
:103150002400816010BD00BF40420F007C060020AB
:10316000A12F000810B50C46054991FBF2F292B26E
:103170000121FFF71DFF034B43F8240010BD00BFE2
:1031800040420F00AC0600200A4A0B481368116049
:10319000C91A40F68C2291420360084B01DD0020E1
:1031A00006E01A78072A9CBF054820F81210501C28
:1031B0001870704714080020700700205C0700207A
:1031C0005E0700207FB5044601A80D46164609F0AB
:1031D000F8FF002003210123ADF80A00ADF80C1020
:1031E000204601A9ADF80450ADF80660ADF80830EE
:1031F0000AF068F87FBD00000F4B142210B502FBE7
:1032000000308278036932B9416001218170186809
:10321000197B02220BE044688160084A091B44784C
:10322000C16022F81410002282701868197BBDE872
:103230001040FFF7C7BF00BF740700205E070020E3
:103240002DE9F34114220D466A43154F4FEA001849
:10325000144908EB070401268B188E54E17BA26801
:103260005D701C61606802238DF8061001A98DF85D
:103270000730ADF80420FFF799FC58F80700217BD0
:103280000022FFF79FFF204632464FF6FF7100F005
:1032900039FD20462946044A00F0F4FCBDE8FC81D3
:1032A0007823010874070020F9310008F7B5124EA1
:1032B0000701BC19A168114B0025E27B1D701C6140
:1032C00060680223ADF8041001A98DF807308DF86D
:1032D0000620FFF76BFCB859217B2A46FFF772FFE7
:1032E000204601224FF6FF7100F00CFD20462946D2
:1032F000034A00F0C7FCFEBD7823010874070020D4
:1033000089310008014B33F8100070475E07002038
:1033100041717047426A806A131A594251EB0300A7
:1033200070477FB5044601A80D46164609F049FFCF
:1033300000200123ADF80A00ADF80C0001A92046D9
:10334000ADF80450ADF80660ADF8083009F0BAFFEA
:103350007FBD437913F001010BD0026AC3699A4221
:1033600005D09CBFC0681218D01AC0B270470020A8
:10337000704708467047437910B513F001010446C1
:103380000ED0FFF7E6FF60B1E3696269E168D05CE7
:103390004A1E934201D2013300E00023E36110BDD5
:1033A000084610BD43799A070AD5436A8269D15409
:1033B000416A03694A1CB2FBF3F103FB112242622A
:1033C00070478379012B03D1D1F1010138BF00216E
:1033D000D0F834014268836809B1136170475361C2
:1033E000704707B5034699684822ADF804100223D8
:1033F000406801A98DF806208DF80730FFF7D6FB4D
:103400000EBD00002DE9F74391464FF4127242437E
:103410001F463B4B0646D41808B93A4802E001283B
:1034200004D1394820631030C4F83401374D0020EE
:10343000D55003224FF001086271D4F8342184F88A
:10344000388284F83C0284F8390284F84662E162EA
:103450004FF48071E1602161916804F1340304F557
:103460009C75636120621023E061A561A0626062C7
:10347000A4F84202A4F84402ADF80410506801A96F
:10348000C4F80890A77102258DF806308DF8075012
:10349000FFF78CFB206BFFF7A4FF41462046FFF7A8
:1034A00090FF322003F009FB1948D4F834810368F7
:1034B0001846B0FBF9F1B1F5803F03D30128F8D9E4
:1034C0004008F6E7134A4046B3FBF2F5EAB289B288
:1034D00000F018FC404631460F4A00F0D3FB256B44
:1034E000012F14BF022200222868297BFFF719FF51
:1034F00028463146094A00F0C5FB2046BDE8FE8358
:1035000084150020B8230108D823010848230108A6
:103510008801002040420F0049370008D1350008DB
:1035200003460A4690F84602D96A9B79FFF76ABFBC
:10353000C268036A511E8B4201D3002300E00133AD
:103540000362704710B590F83C220446AAB9836A1A
:10355000416A994225D080692169C05C01338B4260
:10356000A36228BFA26242000A2342F4007084F8DA
:103570003D32A4F83E02012311E090F93D3273B1CF
:10358000B0F83E124A08A0F83E2201F00101FFF710
:1035900018FF94F83D02431E84F83D3210BD84F8B4
:1035A0003C3210BD90F83B3210B583B990F83A32F6
:1035B00090F8392293420AD2012101FA03F1B0F8BE
:1035C000404201332143A0F84012DBB2F2E710BDC4
:1035D0002C4B10B54FF4127404FB00346079C10712
:1035E0004ED594F8381219B3236B0021186809F0EE
:1035F00037FE94F83C1221B1B4F84202421CA4F800
:103600004222236BA2791868197B012A0CBF02227F
:103610000022FFF786FE0020012184F83B1284F887
:10362000390284F83A02A4F8400284F8380210BD46
:1036300094F83B222046012A04BF94F8392284F8EA
:103640003A22FFF7AFFF94F83B02236B50B90120F9
:10365000A27984F83B021868197B012A0CBF022268
:10366000002209E0002184F83B12A2791868197B36
:10367000012A14BF02220022BDE81040FFF751BE0C
:1036800010BD00BF8415002090F83B1200230122DA
:10369000012980F8393280F838220BD180F83B328A
:1036A000036B8279197B1868012A14BF0222002259
:1036B000FFF737BE7047427908B5D20703461BD5DE
:1036C000B0F8402202F4007189B209B9D10705D4DB
:1036D000B3F84402421CA3F8442208BDC16AC2F3F5
:1036E000470211B11046884708BD4169036ACA54B0
:1036F000BDE80840FFF71CBF08BD10B590F8383290
:103700000446002B1ED190F839124A1CD3B2092B63
:1037100080F8393203D1BDE81040FFF743BF0A2BD0
:1037200010D190F83B0228B9B4F8401241F00102E0
:10373000A4F840222046FFF7BEFF2046BDE8104017
:10374000FFF7A2BF10BD0000064B10B54FF4127476
:1037500004FB00342046FFF7F5FE2046BDE810408C
:10376000FFF7CBBF84150020036B13B15A68006CC0
:1037700001E0026AC069101A18BF01207047436B4C
:1037800013B190F844007047826A406A111A4B42A4
:1037900053EB010070471FB5836800210093437904
:1037A000ADF8041003F0040101F0FF0231B14FF451
:1037B0000051ADF806104FF4806201E0ADF806202C
:1037C000ADF80820002213F0010118BF0421ADF864
:1037D0000C209A07ADF80A1005D5BDF80A3043F061
:1037E0000802ADF80A20006D694609F023FE05B015
:1037F00000BD4171FFF7CFBF8160FFF7CCBF026B07
:10380000034610B5406942B11A6CD9688C1A013A66
:1038100018BF1146005D196410BD196ADA68405C72
:103820000131B1FBF2F402FB1411196210BD00006A
:103830002DE9F0411E464B4B8CB098428846174606
:1038400004D11046314600F0C7F807E046498842E7
:1038500040F083801046314600F014F9002587605F
:103860000562C56185624562C0F82C80467185712C
:103870000446FFF790FF01A80AF0F6F8E06C8027F5
:1038800001904FF48052F0070A920B950595079529
:103890000697089527D5206BD0B1E3680395656935
:1038A00020210493099102950AF046F8206B01A9A2
:1038B0000AF0BAF8206B01210AF0E3F8206D4021EC
:1038C000012209F035FE206B0AF0F0F820640AE0CE
:1038D000206D40F2255109F034FE206D40F2255153
:1038E000012209F00BFE01A80AF0BEF8A06C002529
:1038F00080274FF48052B10701900A920B950595ED
:1039000007950697089523D5606BD8B123691021D8
:103910000493039109950AF00FF8606B01A90AF06E
:1039200083F80122606B02210AF0B6F8606B294629
:103930000AF0BAF8606B394645600122206D09F043
:10394000F7FD05E0206D40F22771012209F0D6FD58
:10395000206D012109F0C6FD00E0002420460CB0D6
:10396000BDE8F0810038014000440040836A81696D
:10397000426BC918D160416A994203D9CB1A53608E
:10398000816204E00169CB1A536000228262002147
:1039900080F84410406B01210AF073B810B5426AF8
:1039A0008469A154416A02690131B1FBF2F402FB5E
:1039B0001411426B416232B11368DB070BD4BDE8CE
:1039C0001040FFF7D3BF006D40F227710122BDE820
:1039D000104009F093BD10BD234B13B5234A9860E6
:1039E00023481A6058614FF4807222480C462249DD
:1039F000DA601A61214A9961011D18659964D964D8
:103A00001A630121143A4FF480405A6309F084FE8E
:103A1000022318214FF40070A2078DF80330ADF88F
:103A200000008DF8021003D515486946FFF7BEF86F
:103A300048234FF480628DF80230E307ADF8002090
:103A400003D50F486946FFF7B1F80E2001218DF824
:103A5000040001A88DF805108DF806108DF80710E8
:103A600009F0B0F900481CBDD80A00206023010805
:103A70001808002000380140580900205800024072
:103A800000080140214B224A13B598600C46802063
:103A900040211A60D86019611E4A1F491F485A61A7
:103AA00098610A1D19654FF4003001219A64DA64A7
:103AB00009F03EFE042002231821ADF80000A00703
:103AC0008DF803308DF8021003D515486946FFF7CD
:103AD0006DF808224823E107ADF800208DF8023088
:103AE00003D50F486946FFF761F8262001218DF8BC
:103AF0000400022201A88DF805108DF806208DF82B
:103B0000071009F05FF901481CBD00BF2C0B002015
:103B100060230108580A00200044004018090020D2
:103B20000008014010B50B4C4FF4005009F0C2FFE3
:103B30000021606B09F0A5FF626AA36A9A4204D073
:103B40002046BDE81040FFF711BF012084F8440073
:103B500010BD00BFD80A00200D4B186D028802F07E
:103B600080018AB29AB19A6A596A8A420AD09969DE
:103B7000895C013281801969B2FBF1F001FB1022EE
:103B80009A62704740F22771002209F0B7BC704773
:103B9000D80A00201C4B10B51A6D1488A4B204F08A
:103BA000200188B290B1D96A19B1938898B2884738
:103BB0000CE09288D9695869D2B24254D869DA685F
:103BC000411CB1FBF2F002FB1011D96104F080043A
:103BD000A4B2C4B10C4B9A6A586A82420BD098695D
:103BE000196D805C013288801969B2FBF1F001FB2C
:103BF00010229A6210BD186D40F227710022BDE8B4
:103C0000104009F07BBC10BD2C0B002030B5002407
:103C10000E4D55F82450854202D00134E4B2F7E746
:103C200000200B4D35F810508D4202D0451CE8B2F3
:103C3000F7E704EB8000C0B20F2805D8054C04EB71
:103C4000001083600171027330BD00BF5824010869
:103C500068240108800B00200C2912D8DFE801F04D
:103C600007111111091111110B1111110D00022170
:103C700004E0042102E0082100E01021012209F003
:103C8000C2BA704738B504460D461346217B00681A
:103C90002A46FFF7BBFF2068217BBDE83840FFF7CD
:103CA000DBBF07B58DF80400012000238DF8060066
:103CB0008DF8070001A88DF8053009F083F80EBDD6
:103CC0007FB5044601A80D46164609F067FA0B4B6E
:103CD0000B485E4301680023B1FBF6F2013D561E1E
:103CE000204601A9ADF80850ADF80460ADF80A30DF
:103CF000ADF8063009F00AF97FBD00BF40420F0061
:103D00008801002010B504460068FFF7D9FF20683D
:103D1000012109F05EFA607BBDE81040FFF7C1BFEA
:103D200000230C4A52F82320824202D00133DBB236
:103D3000F7E70022084830F81200884202D0501CF1
:103D4000C2B2F7E703EB82030449DAB201EB0210D7
:103D5000704700BF5824010868240108800B002028
:103D600070B5044600262E4B9D5D95B90221204674
:103D700009F051FB01284FD12046022109F056FBE2
:103D800029462046FFF7CCFF0546204609F036FBC2
:103D90003DE0042D12D12046294609F03CFB0128C4
:103DA0003AD12046294609F041FB29462046FFF733
:103DB000B7FF0546204609F024FB28E0082D12D164
:103DC0002046294609F027FB012825D1204629460F
:103DD00009F02CFB29462046FFF7A2FF05462046A6
:103DE00009F012FB13E00C2D16D11021204609F02A
:103DF00012FB012810D12046102109F017FB29469B
:103E00002046FFF78DFF0546204609F000FBAA6813
:103E100001460AB1287B90470236082EA3D170BD17
:103E2000682401080148FFF79BBF00BF002C014038
:103E30004FF08040FFF794BF0148FFF791BF00BFEC
:103E4000000400400148FFF78BBF00BF000800409E
:103E5000024800214FF480720CF0AABC800B0020B5
:103E600010B5FCF7DBFE0A49FCF72CFF0949FCF70B
:103E7000DDFF094B044618680078FCF7CFFE0146C9
:103E80002046FCF71FFFFDF709F980B210BD00BF07
:103E90003333534000F07F45940C002038B50D4C6F
:103EA00000202578FDF774FD0B4A05F0070322F882
:103EB00013000135002325701846D15A02334018EB
:103EC000102B80B2F9D1C008FFF7CAFF034A107067
:103ED00038BD00BF800C0020820C0020141A002086
:103EE000074B084A19781088884207D3064B1A688E
:103EF000907888428CBF00200120704700207047D6
:103F0000141A0020161A0020940C002038B5114B0A
:103F10002024186000250020FDF73AFD2D180A2006
:103F200002F0CBFD013CF6D1C5F34F10FFF798FF2F
:103F3000084901230A6851786418A04202D301336A
:103F4000062BF9D1044892780370534303490B8040
:103F500038BD00BF940C002010000020161A00206D
:103F60002DE9F04F0446008885B048B9B4F9023015
:103F700043B9B4F90420D2F1010138BF002102E0B5
:103F8000002100E0014611F0010377D13D4D00B260
:103F90002B7000F0C9FD0646B4F9020000F0C4FD24
:103FA0000546B4F9040000F0BFFD0446304609F0B0
:103FB0008BFD0746304609F0FBFD8046284609F098
:103FC00083FD0646284609F0F3FD0546204609F024
:103FD0007BFD8246204609F0EBFD3946814650467E
:103FE000FCF770FE394683464846FCF76BFE5146A7
:103FF00001904046FCF766FE494602904046FCF7B9
:1040000061FE314603905046FCF75CFE1E4C49466B
:10401000206006F10040FCF755FE29466060A5606F
:104020000298FCF74FFE01460198FCF743FD294634
:10403000E0600398FCF746FE01465846FCF738FD61
:104040003146206108F10040FCF73CFE29466061E2
:104050005846FCF737FE01460398FCF729FD294630
:10406000A0610198FCF72EFE01460298FCF722FDA4
:104070003946E0613046FCF725FE206205B0BDE818
:10408000F08F00BF11000020980C00202DE9F843AC
:104090004D4B0C460168013A196080889880072AC8
:1040A00030D8DFE802F004080F14191E2226188801
:1040B00020805A8803E0598821801A885242628001
:1040C0009A881EE01988484220805A88F6E7598865
:1040D000484220801A88F2E7198848422080588890
:1040E0000CE05A882280188808E0198821805A88B4
:1040F00003E05988484220801A88504260809B889B
:104100005A42A280314B1A78002A5AD1B4F90000E1
:10411000FCF784FD8046B4F90200FCF77FFD0746FA
:10412000B4F90400FCF77AFD294D0646296840469B
:10413000FCF7C8FDE96881463846FCF7C3FD014637
:104140004846FCF7B7FCA96981463046FCF7BAFD42
:1041500001464846FCF7AEFC09F0EAFC696820809D
:104160004046FCF7AFFD296981463846FCF7AAFDB9
:1041700001464846FCF79EFCE96981463046FCF75B
:10418000A1FD01464846FCF795FC09F0D1FCA96861
:1041900060804046FCF796FD696980463846FCF72A
:1041A00091FD01464046FCF785FC296A07463046EA
:1041B000FCF788FD01463846FCF77CFC09F0B8FCAA
:1041C000A080BDE8F88300BFBC0C002011000020D7
:1041D000980C002070B5144D06462B78134CABB1EB
:1041E00002F05AFC2268B31898421CD300202870B1
:1041F00002F012FC02F050FC20600D48017809B179
:104200004A1E02700B4B0120187070BD02F044FC76
:1042100021683231884206D30120287002F0FCFB6D
:1042200002F03AFC206070BDC30C0020D00C0020CE
:10423000C60C0020C50C002037B58DF805102249AA
:104240008DF807300B788DF8040002A88DF8062051
:10425000C21812F8044C0D46443CE0B20A282CD88F
:104260001A49022B31F8104003D814B12046FFF749
:10427000B1FF2B78022B0BD9154D2D6802F00CFCE9
:10428000021B954204D21049124B0020087018708E
:10429000114802780146012A00D094B90A4B1878D7
:1042A000022801D8421C1A70002008700B490870BF
:1042B00003B0BDE8304002F0AFBB3224022BD5D9A9
:1042C000D7E703B030BD00BFC40C00207024010844
:1042D000D00C0020C60C0020C50C0020C30C002010
:1042E000014B1860704700BFC80C002070B53F4BF1
:1042F00004465A7B3E4802B1012202704FF400701E
:1043000000F076F9002828D03A4E3B4B31685878B7
:104310000D68003018BF01206A68904748B13368C3
:10432000364D18680121C2682970904708B10221F2
:104330002970304D2B6818688268904728B12E4943
:104340004B7813B92D4A0220107029680B689869C0
:10435000804710B1294900220A70202005F0DAFABE
:1043600060B12248264B827A0AB9C17A21B122482B
:10437000C27A0AB9012100E0002119701F4B187898
:10438000022802D14C204E211DE0012807D14D21E9
:1043900053204C220B46BDE87040FFF74DBF184A32
:1043A0001178012903D1532001464E2206E0104B1B
:1043B0001878012804D15320014602464D23EAE72C
:1043C00024B153204D210A464423E4E70D4A1178D5
:1043D00021B13220BDE87040FFF7FCBE0A4B2046F9
:1043E0001C70BDE8704002F017BB00BFF01F00203A
:1043F000C70C0020C80C0020DF1F0020C20C0020CA
:10440000CC0C0020C60C0020C30C0020014B1870FF
:10441000704700BFC60C00200E4B1A78422A16D1F6
:104420005888B0F56C7F12D11979BE290FD193F855
:10443000AD230020EF2A0CD113F8011B064A484097
:104440009342F9D1D0F1010038BF0020704700201D
:104450007047704700F80108B0FB0108C823142119
:104460001E22038001238170C270037164214FF406
:1044700096722823C18002814381704710B504469B
:10448000272006F097FA2070102006F093FA60704B
:10449000002006F08FFAA070002006F08BFA4FF48F
:1044A000E133E07052206360A360E360207510BDCB
:1044B0007FB51E4D1E4C284605F062FA214628465F
:1044C00005F078FA1F3D04F1240002F0D3F82E46DF
:1044D00004F1680005F006FE16F8C20B02F09AFD22
:1044E000304604F05DF9681C04F018FA05F1B800D4
:1044F00000F01EFE04F1280001F024FF04F149033E
:1045000004F1380005F1C00100930190029105F11A
:104510007800A11D224605F1BE0303F09BFB05F1C7
:10452000340004B0BDE8704001F012BFE71D002068
:10453000E81A002008B5054BD02202FB00300449E0
:1045400000F59E700CF086F808BD00BF181A002018
:10455000C81D0020224A38B5422313704FF46C70F6
:104560000023BE21EF245080117182F8AD4382F800
:10457000AE331D461A4A985C0133B3F56C7F85EA69
:104580000005F7D182F8AE5308F0E4FF04250024BB
:10459000691E11F0FF0516D0342008F0EFFF114816
:1045A00009F042F80F4C04280BD10F4A2046A158BD
:1045B00009F010F80D4B04349C42F4D10428044651
:1045C00001D00446E4E708F0D1FF042C02D1FFF744
:1045D00023FF20B90A20BDE8384002F00DBB38BDEA
:1045E000181A002000F801081822FE17B0FB010875
:1045F000034B996808420CBF00200120704700BFA0
:10460000181A0020024B9A6810439860704700BF48
:10461000181A00202DE9F04FA84AA94D85B010685E
:104620005168A84C02AB03C34FF46C7200212846BA
:104630000CF0BEF8D022002120460CF0B9F8422040
:104640000321287002206971FFF7DCFF2A23202153
:10465000A5F8EE304FF4FA702B2385F8F41040F2F1
:104660004C41FA22A5F8F60085F80531212001F524
:104670004873A5F8F22085F806016E2240F27E40CC
:10468000A5F816314FF47A7300274FF001094FF463
:10469000167685F80421A5F8141140F2DC5200F5D5
:1046A0002F71A5F8D00003F5CB70A5F81221A5F85D
:1046B000F060A5F8D21085F8AC73A5F8FA70A5F8EB
:1046C000F870A5F8FC7085F8E27085F8E37085F85D
:1046D000E470A5F8E670A5F8E870A5F8EA7085F82A
:1046E000ED7085F8EC9085F8077185F8387185F8DC
:1046F0003A7185F8397185F8107185F8187185F867
:10470000197185F81A91A5F8D430A5F8D6006C3047
:10471000A5F8D8004FF4C870322340F2B451A5F880
:10472000DE0005F590709B46A5F8DA10A5F8DC30A0
:10473000A5F8E030019285F81C7185F81D71FFF72E
:104740009DFE1E211723552040F6AC52E172637581
:104750002173A3750B211423AA81E0702D22082058
:104760006171A3710E21637450234FF028086273A6
:104770002074A2766420E171E3765A2178234FF009
:104780000A0A22754122A37221722077E177AF7362
:1047900085F81B71277084F8018084F80280E77522
:1047A00084F804B0A7732776E773677684F812A0BD
:1047B00084F8098084F81E9084F8202084F82370FF
:1047C00084F8247084F82570019904F12A00E184AA
:1047D00084F821B084F8227002F008FC04203A4AE0
:1047E00084F82E0039493A48152384F83430A263FE
:1047F000E163206405F584713648278584F82F80AD
:1048000084F8308084F8449005F014FA4FF448732B
:10481000C8224FF4966140F2D9303E4684F8707059
:1048200084F8717084F8728084F8739084F87670DC
:10483000A4F8743084F8B8A084F8B920A4F8BA10A9
:10484000A4F8BC004FF47F734FF4FA62A4F87830F8
:1048500007F108006B46A2F5FA71A4F87A20C25C51
:10486000A4F87C100137FF2184F87E2084F87F10A3
:104870000834082FE6D11348012480F8BE4080F8A0
:10488000BF4080F8C040C230FFF7E8FD00200C4B6D
:104890000021C2181030C0281161F8D100240E4840
:1048A000D02220180749D0340BF0D4FEB4F51C7F79
:1048B000F5D105B0BDE8F04FFFF74CBEE02201088E
:1048C000181A0020C81D00209A99193FF6287C3F2D
:1048D0003D0A773F86240108541B002008B5FFF7E6
:1048E0009BFD18B9BDE80840FFF794BE08BD000065
:1048F000024B9A6822EA000098607047181A00205C
:10490000364B10B599680A0409D4CC0707D40807B8
:1049100005D4C90303D44FF40040FFF773FE2F4AB8
:104920009068144610F4803F12D0020702D5082088
:10493000FFF7DEFFA3681B0403D54FF40040FFF729
:10494000D7FF26498A68D40702D50120FFF7D0FF98
:1049500022488368044613F0080F0BD0180403D5CF
:104960004FF40040FFF7C4FFA168C90702D501203A
:10497000FFF7BEFF194A48F20103906848F20104AC
:104980000340A342144603D14FF40040FFF7B0FFA9
:10499000A1684A0505D50B0403D44FF48060FFF7E6
:1049A000A7FF0E4A48F24003906848F240010340D6
:1049B0008B4202D14020FFF79BFF094805F03AF8EF
:1049C000084806F009F9074806F082F820B90548BA
:1049D000BDE81040FFF752BD10BD00BF181A0020FF
:1049E000201B0020381B002010B5FFF715FD10B963
:1049F0000A2002F001F90F4C0F4920464FF46C7267
:104A00000BF028FE94F8AC33022B02D9002084F876
:104A1000AC0394F8AC13D02202FB0143074803F522
:104A20009E710BF017FEFFF76BFFBDE81040FFF71C
:104A30003FBD00BF181A002000F80108C81D002063
:104A400008B5FFF7D1FF0F2014210122BDE808406F
:104A500007F012BF08B5054B93F8AC03FFF76AFDEA
:104A6000FFF778FDBDE80840FFF7EABF181A0020FD
:104A7000014B9868704700BF181A0020884203DB7A
:104A80008242B4BF114601460846704700230361C5
:104A900070472DE9F041066904460136012E0D46A6
:104AA000066105D10023616021608360BDE8F0816B
:104AB000D0F8008008464146FBF7FAFF074630462B
:104AC000FCF7ACF801463846FCF7B0F90146404621
:104AD000FBF7F0FF0646606031462846FBF7E8FF2B
:104AE00001463846FCF7EEF8A168FBF7E3FF2660C5
:104AF000E060A060BDE8F08110B5044600690128BF
:104B000007DD0138FCF78AF80146E068FCF78EF90A
:104B100010BD002010BD08B5FFF7EEFFBDE808404E
:104B200009F068BA0000000008B5FBF76DFC04A3AB
:104B3000D3E90023FBF7CEFCFBF766FF08BD00BFFF
:104B4000399D52A246DF913F2DE9F041069C064671
:104B50000F46002B0CBF4FF020084FF030082046C6
:104B600010F8013B0BB9154603E0002AFBDD013AC2
:104B7000F6E7002D04DD30464146B847013DF8E731
:104B800014F8011B11B13046B847F9E7BDE8F081D0
:104B9000014B186801F002BFDC0C00202DE9F04346
:104BA00089B006460F4603921C46039A134613F833
:104BB000011B0393002900F08A80252901D030468B
:104BC00083E0002004905578911C302D039105D18D
:104BD0009578033203924FF0010800E08046A5F17A
:104BE0003003D8B2092806D8284603A90A2204AB04
:104BF00000F02AF905466C2D05D10399012211F820
:104C0000015B039100E00022642D2FD010D8582DB5
:104C10003AD006D8002D5AD0252DC6D13046294687
:104C200053E0632DC1D130462178251DB8474AE0B5
:104C3000752D0DD0782D27D0732DB6D1251D246864
:104C4000304600943946049A0023FFF77DFF3AE08E
:104C5000251D20680A2122B1002205AB00F07EF854
:104C600002E005AB00F0AAF82C4623E005AD04F104
:104C700004092068294612B100F095F801E000F01F
:104C8000C2F84C46009517E004F104092068102191
:104C900042B1B5F15804634253EB040205AB00F096
:104CA0005DF806E0B5F158035A425A4105AB00F0F1
:104CB00085F84C4605A8009030463946049A43468C
:104CC000FFF742FF71E72C466FE7B8476DE709B081
:104CD000BDE8F0830FB407B5094904AB086809497A
:104CE00053F8042B09680193FFF758FF064B186827
:104CF00001F073FE0028F9D0BDE80E4004B0704703
:104D0000D80C0020D40C0020DC0C0020034A044BFB
:104D1000044900201A600860704700BF914B0008EA
:104D2000D40C0020D80C0020014B1860704700BF45
:104D3000DC0C002070B50646B6FBF2F408461546BA
:104D400014B12046FFF7F6FF05FB1464024B195D12
:104D500000F8011B70BD00BF8F240108F0B50124CD
:104D6000B0FBF4F58D4201D34C43F9E70026C4B102
:104D7000B0FBF4F504FB1500B4FBF1F41EB9002DF3
:104D800001DC002CF4D1092DEFB204DD002A0CBFA8
:104D90005725372500E03025ED1903F8015B013672
:104DA000E5E71C70F0BD00280B4603DA2D224042D7
:104DB00003F8012B0A210022FFF7D0BFF0B5012430
:104DC000B0FBF4F58D4201D34C43F9E70026C4B1A2
:104DD000B0FBF4F504FB1500B4FBF1F41EB9002D93
:104DE00001DC002CF4D1092DEFB204DD002A0CBF48
:104DF0005725372500E03025ED1903F8015B013612
:104E0000E5E71C70F0BD00280B4603DA2D22404276
:104E100003F8012B0A210022FFF7D0BFA0F13003D5
:104E2000DAB2092A01D818467047A0F161010529B4
:104E300001D857387047A0F14103052B01D8373806
:104E400070474FF0FF3070472DE9F8430D68044676
:104E50000F469046994600262046FFF7DFFF0028C0
:104E600006DB404504DC08FB060615F8014BF3E7BA
:104E70003D602046C9F80060BDE8F883931E222BF0
:104E800088BF0A22031E10B50C4603DA2D2001F854
:104E9000010B5842FFF74EFF00210170204610BD64
:104EA00030B587B005460C4603A800210C220BF054
:104EB0007FFC28460021FCF7C1F820B1284629498B
:104EC000FBF7F8FD03E028462649FBF7F1FD2649EC
:104ED000FBF7F8FEFCF7BCF8054685EAE570A0EBA9
:104EE000E5700A226946FFF7C9FF002D01DB202388
:104EF00000E02D2368468DF80C300CF08DFB012866
:104F000007D130228DF80D208DF80E208DF80F205E
:104F10000CE0022805D130218DF80D108DF80E100F
:104F200004E0032802D130208DF80D00694603A863
:104F30000CF070FA03A80CF06FFBC51EEDB22A4608
:104F400003A920460CF006FC0023635520460749C0
:104F50000CF060FA03A9204649190CF05BFA2046D0
:104F600007B030BD6F12033A00007A44002F0108E9
:104F70002DE9F041027803460130202AFAD0092AAF
:104F8000F8D02D2A02D10346414D04E02B2A08BF58
:104F900003464FF07E551E460024334616F8010B9B
:104FA000A0F13007F9B209290DD83A492046FBF79C
:104FB00089FE04463846FBF731FE01462046FBF7E2
:104FC00079FD0446E9E72E2817D1324F334616F80B
:104FD000010B3038C2B2092A0FD8FBF71FFE394641
:104FE000FBF724FF01462046FBF764FD29490446F0
:104FF0003846FBF767FE0746E8E71878652801D0D2
:10500000452839D15E782D2E02D19F1C012605E05E
:105010002B2E01D05F1C00E09F1C00267B1E00276A
:1050200013F8012F303AD1B2092903D80A2000FB26
:105030000727F5E7B7F59A7F28BF4FF49A77B84668
:105040004FF07E51B8F1070F07D908461249FBF718
:1050500039FEA8F108080146F4E707F0070737B161
:1050600008460C49FBF72EFE013F0146F7E72EB13B
:105070002046FBF7DBFE04E04FF07E512046FBF7B5
:1050800021FE01462846FBF71DFEBDE8F08100BF6A
:10509000000080BF0000204120BCBE4C014B00221C
:1050A0009A807047E40C0020034BB3F90400D0F160
:1050B000010038BF00207047E40C00200649074B70
:1050C0000A68B3F90400137805214B439842D4BF12
:1050D00000200120704700BFEC0C0020E40C0020F1
:1050E00010B50446FFF7EAFF002814BF2046002051
:1050F00000F0010010BD0000074B084A1968B2F922
:1051000004004B780A78D118052251438842D4BF55
:1051100000200120704700BFEC0C0020E40C0020B0
:10512000024B9A88501C9880704700BFE40C002006
:10513000024B00221860024882807047EC0C00206D
:10514000E40C0020034B044918600448002201606D
:10515000C2807047F00C0020B4240108E40C002049
:1051600008B501F03BFF024B00221A7008BD00BFDA
:10517000DF1F002010B5FFF7A1FF00281ED0104B45
:105180005C78201C18BF0120FFF7AAFF70B10D4802
:105190000D4B01680D484A8901681A805A809A802F
:1051A0004A88DA800A4BD888411CD980FFF7A4FFCF
:1051B00000B91CB9BDE81040FFF7D2BF10BD00BF59
:1051C000DF1F0020F00C002036200020EC0C002017
:1051D000E40C0020044B9A8811B2142901DD143A22
:1051E00000E000229A807047E40C002003280B4B5B
:1051F0000AD80B4A126892888A4205D2012101FA24
:1052000000F01A78104318701B780F2B04D1034854
:1052100000210170FFF7DEBF704700BFE00C0020E7
:10522000EC0C002030B5864C89B0FFF76FFDFFF71E
:1052300055FBFFF7D9FBA07B003018BF012001F020
:1052400047FC94F8073133B1012B01D0092B02D16F
:105250008DF80C3004E000218DF80C1084F8071153
:1052600003A8FCF7A3FB0220FFF7C2F910B17548B1
:10527000FEF74CFE7448FEF773FE0E2004F054FB5C
:10528000724D6F4AB5F9283002F1E200B2F8EE1023
:1052900092F8ED2001F0C0FA10B9032001F0ACFC47
:1052A0006B4C1020082360610A252361684C013D86
:1052B000E16881F01002E260E06880F00803E360DA
:1052C000192001F0FAFB012001F0A6FB192001F0E2
:1052D000F4FB002001F0A0FB15F0FF05E6D1102241
:1052E000082121612261564C01F01EFF607904F112
:1052F000100102F00FFDFEF7ABFD04F5907005F014
:10530000E1FC60790E2801D0082803D101238DF833
:10531000163001E08DF816504E4C0121204605F064
:105320001DFC8DF812004020FFF762F98DF8130084
:105330004FF40040FFF75CF98DF810000120FFF7F3
:1053400057F98DF8110003F00BF940498DF814005E
:1053500091F8C02034F8423CC2F3800034F8401C7D
:105360008DF815004FF47A724FF48040ADF8183084
:10537000ADF81A10ADF81C20FFF73AF918B134F85F
:10538000464CADF81C40BDF81800B0F5FA7F02D9C4
:105390000023ADF81C302A4991F80741B1F81221D9
:1053A000012CADF81E2004D0092C01D1072400E007
:1053B000002404A88DF81740FDF75CFD2648FFF790
:1053C000C1FE264C2060FEF78BFF2348216804F0C5
:1053D0006BFB4FF48070FFF70BF958B11848204B66
:1053E00090F81D1190F81C21009300F59070C133C6
:1053F00003F0E4FA4FF48060FFF7FAF808B101F027
:10540000B9FA4FF40060FFF7F3F808B104F0EEFECC
:1054100001F028FB0A49134B4A791860052A03D189
:105420004FF4C87000F07CFE4FF47A7001F028F958
:10543000C82000F09DFF0C4B0120587309B030BD0F
:10544000181A00201C1B0020FE1A0020C81D002076
:10545000000C0140381B0020201B0020981E00205B
:10546000C91D0020280D0020DF1F002008B5FFF710
:10547000D9FE00F001FAFCE708B5034BB3F9D400FC
:1054800002F05EFDFEE700BF181A002008B501F02B
:10549000FDF80B4B50B19A7842B1597879B9012295
:1054A0005A70084B08491888088008BD587830B9E8
:1054B0000220FF210122BDE8084007F0DDB908BD48
:1054C000DF1F0020021F0020A81E00202DE9F04F42
:1054D000A24BA34AB3F90600D18C85B088420FDBFA
:1054E000B0F5FA6F92F8254007DA451A6C43A1F53A
:1054F000FA6694FBF6F4643403E0C4F1640400E05B
:105500006424984A964BB2F8127192F9EC2093F801
:1055100023100097574293F87050019193F87160EF
:10552000B9B293F824300291002103930A468B4FBD
:10553000DDF8008031F907C040F2E637C8EB0C0314
:1055400003F2F31EBE4503D8002BB8BF5B4201E057
:105550004FF4FA73022ADFF818822CD025B1AB423F
:10556000CCBFC5EB030300236427DFF824A293FB21
:10557000F7FE6FF0630B3AF81E900BFB0E3B0EF13B
:10558000010E3AF91EA00FFA89FECEEB0A0E0EFBB1
:105590000BFE9EFBF7FEF14428F80190DDF8048035
:1055A00003FB08FE704B9EFBF3F3DB199BB26343D6
:1055B00093FBF7F712E026B1B342CCBFC6EB03036F
:1055C0000023029F5F43A8F80470039F002BB8BF1D
:1055D0005B427B43644F93FBF7F76437604B02EB0E
:1055E000030E9EF80190642307FB09F898FBF3F97A
:1055F000DFF8A08102F808909EF80B909EF815E065
:1056000007FB09F807FB0EF798FBF3F9DFF8888131
:1056100097FBF3F302F80890DDF80080534FC44580
:10562000D35503DA524BCF5A7F42CF520132023167
:10563000032A7FF47CAF4B4C4FF4FA62B4F8141198
:10564000FFF71CFAB4F814614FF47A75801B4543D8
:10565000C6F5FA63B5FBF3F56421464895FBF1F313
:105660006FF0630630F8132006FB0355013330F961
:10567000130013B2C01A45433F4B3D4C95FBF1F16B
:10568000587A8A18E280002838D03C4F3C4D3E883A
:105690002988721A10B2FFF747FA074608F014FA81
:1056A0000646384608F084FA0546B4F90200FBF7CE
:1056B000B5FA0746B4F90000FBF7B0FA3146804668
:1056C000FBF700FB294681463846FBF7FBFA01460B
:1056D0004846FBF7EDF9FBF7BBFC31462080384626
:1056E000FBF7F0FA294606464046FBF7EBFA01467F
:1056F0003046FBF7DFF9FBF7ABFC60800220FEF7DA
:1057000077FF90B11F4806220378591CCBB2037073
:10571000B3FBF2F002FB103111F0FF0F05D1FEF7E1
:10572000BDFBFEF7DDFB184B1870174A10780030F0
:1057300018BF0120FEF7DAFD00F0F8FC18B100F008
:10574000A5FF58BB04E0022004F0E4F80028F6D0DE
:105750000E4BDA6882F00801D9602CE03620002078
:10576000C81D0020181A00200CFEFFFFFB1E0020A1
:10577000062000200E200020DF1F0020021F002036
:10578000A81E0020F50C0020240D0020000C014074
:1057900026200020FE1E0020F81E00202D4B9978A8
:1057A00011B12D4A082010615B7813B12A480821F5
:1057B000416104F0F5FC8020FEF71AFFB0B12748E4
:1057C000274B02681968501A00280FDB02F5434284
:1057D00050321A601F4B234A5978081C18BF012009
:1057E000B2F90210B2F90020FDF736FA1B481E4A42
:1057F00001681368C81A002810DB164B587B58B98B
:105800009870154B01F5F421D86880F00800D86035
:1058100001F59073136001E00121997005F062FABF
:10582000124A107830B94FF40060FEF7E1FE08B17B
:1058300004F0F0FC202004F06DF818B10749086866
:1058400004F04EF80A4B9A680AB10A48904705B02E
:10585000BDE8F08FDF1F0020000C0140F80C002095
:10586000FC0C0020200F0020080D0020D814002080
:10587000DC1E00209C1E002070B50820FEF7B8FE3C
:1058800010B1A14804F04AF904464FF48030FEF705
:10589000AFFE10B104F0EEF904469C4B9C4A186828
:1058A0001168431A002B02DA002C00F09D8200F5EB
:1058B0009C44203494489749146004F03FF94FF415
:1058C0008040FEF795FE20B1934D2B780BB901F087
:1058D00085FB924890F81B21B2B1914CD11C34F950
:1058E00011504FF47A720021A5F57A70FFF7C6F8CF
:1058F000FBF794F98B49FBF799FA8B49FBF7E2F92F
:10590000FBF7CCFB894B18804FF40070FEF770FE5C
:1059100020B18748026811684C69A0477F4D00227A
:10592000B5F81401B5F8164113467D499B08555E3C
:105930008542C4BF63F07F03DBB2A542B8BF43F02A
:1059400040030232082AF0D17A487B4A047805469F
:105950009C4204D11078F92803D8411C00E00021B2
:1059600011704FF480402B70FEF742FE68B16B4D12
:105970006B4BB5F81211B5F8DC20B3F90640881A64
:10598000844202DD8B189C420CDB4FF48040FEF712
:105990002FFED8B9624C6149B4F90650B1F8142110
:1059A000954213DA01F026FB01F02CFB6348B0F8B6
:1059B00046305BB1584C62492578002D00F0848355
:1059C0000A78002A00F08083FFF760FD5A4B1C78AC
:1059D000142C40F0D1805A4D6C78ECB1574BB3F891
:1059E00046502DB953490C785F2C01D101F0F6FADD
:1059F0004A4A92F81801002800F0BE804F4BB3F8D5
:105A00004650002D40F0B8804A490C787D2C40F07B
:105A1000B38001F0E3FAAFE0464D2978572918D159
:105A20004FF47A7000F02CFE4FF48070FEF7E0FD2A
:105A300008B102F021FF042003F06CFF10B10A202E
:105A400000F096FC082003F065FFE0B93D4B18809C
:105A500019E00420FEF7CCFDA8B12A785A2A12D109
:105A60003948037823B104703848012202700AE0F3
:105A7000374C257885F00101217009B1022000E042
:105A80000320FEF7C3FC2B4C25785D2D00F023830B
:105A90005B2D00F022835E2D00F02183274BB3F8AD
:105AA000465035B923490C786F2C02D1FFF7EEFC34
:105AB00015E01A4A1F4B92F8180118B115B91D7854
:105AC0007E2DF3D01978972904D14FF4C87000F0D7
:105AD00027FB04E0A72902D1194A01249473154831
:105AE0000378BB2B03D11548818D8D1C04E0B72BA7
:105AF00004D11248838D9D1E858531E0BE2B29D1AE
:105B00000E4D6A8D941C2AE0201B0020F80C00200A
:105B1000000D002034200020F01F0020181A002063
:105B20003620002000007A4400C07F44A61E0020DA
:105B3000981E0020100D0020180D0020C81D002008
:105B4000DF1F0020021F0020040D0020250D002073
:105B50000D0D0020BD2B0FD18C4D698D8C1E6C85D9
:105B60008B4C94F8AC03FEF7E5FCFEF7F3FCFEF774
:105B700067FF8848002202700420FEF739FD0028E4
:105B80002CD0854B1A788AB18448457875B1844900
:105B90007F4AB1F90640B2F81401844206DD814D16
:105BA0002C781CB9804932220A801C707D4B587CAD
:105BB00050B17E4B1D782DB97D4C227812B97A48B0
:105BC00032210180012008E0794D2C7834B1734AEC
:105BD000517819B9774B2970012018700023764C41
:105BE0001A4634F8020F40F2135501B2A942CCBF55
:105BF0000025012505FA03F5A0F21550B0F5C77F81
:105C00008CBF002001202A435D1C00FA05F00243EE
:105C100040F2A4608142D4BF00210121981C01FA06
:105C200000F103330A430C2B92B2DAD10023574917
:105C30005C4C01EB4300B0F846100A420CBF002058
:105C4000012018550133152BF1D1627822B10220C1
:105C500003F060FE68B914E04FF40070FEF7C8FC72
:105C600078B1564C21680868836898470028EED1BF
:105C700007E04A4CE17839B901F0BCF90120E07045
:105C800002E0464C0022E270464B444C987830B11A
:105C900021790022E27019B901F0ACF901202071DC
:105CA000404B3E491A780AB901200870CA78444B23
:105CB00012B93A49087910B11021596101E0102256
:105CC0001A61042003F026FE10B3364BD878334B0C
:105CD00080B19A797AB93B480121997101683A4BB0
:105CE0003A481960C1883A4B3A4819803A490260EB
:105CF0000A6000E098714FF40050FEF779FC38B16B
:105D0000284A264B117911B1D87B08B90121D973E2
:105D1000022003F0FFFD20B1224A204B507930B918
:105D20000EE0082003F0F6FD0028F5D118E05979BF
:105D300039B92A4801225A710188294B198000E09B
:105D400058711848154B8279014612B15A7A0AB92E
:105D500001225A72C87918B12049224B0A881A8048
:105D6000202003F0D7FD08B103F05CFD0D480B497E
:105D7000027B02B10122064B8A725879082801D0B1
:105D80000E2875D1054A0021517271E0C81D00200E
:105D9000181A0020180D00200D0D0020DF1F002014
:105DA00036200020F01F0020220D00200C0D0020C6
:105DB000040D0020250D00203C200020981E00200E
:105DC000000C0140241F0020281F00200620002076
:105DD000060D0020640F0020600F0020021F00202D
:105DE000F01E0020A81E002088480268042A3FD820
:105DF000DFE802F0030D1A253100012101600820BF
:105E000003F088FD18B1824800F0AAFB80BB7F4BED
:105E10001868421C04201A6003F07CFD20B17D4903
:105E2000086800F0ABFA18BB784B1868421C0420D5
:105E30001A6003F06FFD10B101F008FEC0B973499C
:105E40000B68581C08604FF48070FEF7D1FB10B14E
:105E500002F0E2FE0CE06D49002210200A6003F01F
:105E600059FD08B100F094FD4FF40050FEF7C0FB5F
:105E700000F0F8FD6849674B8A891860674B22B1CA
:105E80001968411A0029C0F23A8184181C6001F097
:105E900057FBFFF71BFB00F0E5FD614B5D4A1968FE
:105EA0001060604A441A18600820148003F032FD24
:105EB000002833D05C485D4A818801F145039CB2DB
:105EC0008A2C5B4B28D85B4844792CB318881388FC
:105ED000C21A94B2A3B218B2B330BCBF04F5B47303
:105EE0009BB24D4C53481AB2B32A94F8EC20447B31
:105EF000C4BFA3F5B4739BB284B152B250424343C2
:105F00004D4C1BB2627A6FF01D005343464C93FB1D
:105F1000F0F3C918A18001E019881180042003F072
:105F2000F9FC002800F0A18042488279002A00F0A4
:105F30009C80007C3C4B002840F08E803E493F4DC9
:105F400091F8732052B3DE88B5F9003034B291F87D
:105F50007210E21A002AB8BF52428A42384A0CDD57
:105F6000384DB6B2286001209C42107001DD4942D4
:105F700089B22D4A8C19D48077E0117821B1324C46
:105F80003249246810700C603148234A0468B2F822
:105F9000D01018196431B2F8D22031E0DC882D8895
:105FA00026B228B2361A91F87230002EB8BF764267
:105FB0009E4212DD274B1A88A618711B0CB24FF4B3
:105FC000FA6194FBF1F2214D01FB12442E681C8012
:105FD000B6182E6001221A4B08E0194B197831B11E
:105FE000194C1A4924680C601A4C22801A70184BFC
:105FF000094C1A68B4F8D0108018B4F8D220643173
:10600000FEF73CFD084BD8802FE000BF1C0D0020A0
:10601000161B0020F80C0020181A0020140D002078
:10602000280D0020200D002006200020F01E00205A
:10603000021F0020DF1F0020C81D0020060D0020C9
:10604000F40C0020640F0020241F0020281F0020D3
:10605000600F00200E0D002029492A4A91F91A41AB
:106060001068598800FB04145C80274B93F8760075
:1060700050B12649CC780CB90A792AB1244B25486D
:10608000DC8801880A19DA80202003F043FC40B143
:106090001E4BD87908B9197A19B11C7B0CB103F0E1
:1060A00037FB1D481D4A164B00F11E011468B3F85A
:1060B000F62000F12903A04701F054FF01F0D0FEC3
:1060C000BDE8704001F028BF487800283FF47EAC5E
:1060D00000F084FF7AE4012102E0022100E00321C4
:1060E000CCB20748621E80F8AC23FEF733FAFEF705
:1060F0007BFC02202821224606F0BEFBCEE470BDC8
:10610000181A0020600F0020C81D0020DF1F00208B
:1061100006200020480F0020C91D00201400002088
:10612000014B1880704700BF480D0020034B1888B2
:10613000D0F1010038BF0020704700BF480D00209B
:10614000F8B51E4B0022196813461D4C2588B5F57D
:10615000C87F1C4D01D10026EE501B4EEF5832F97E
:1061600006C0184C6744EF500025043395538D52F8
:1061700002320C2BE9D1124B1A88012A18D123685C
:1061800003F1C8024FF4C87392FBF3F20A8062680D
:10619000C83292FBF3F24A80A268C83292FBF3F352
:1061A0000A4A12889B1A8B8000F020FFFEF752FCEF
:1061B000034801884A1E0280F8BD00BF4C0D002034
:1061C000480D00203C0D00201C1F00201200002064
:1061D000F8B5354B0446188832280ED13349344D72
:1061E0000A683448168857889388218862882E80E8
:1061F0006F80AB800180428001E0002834D02B4DBD
:1062000000222E681346284F2B493888322801D1A6
:106210000025CD502948CD58175EED19CD500021ED
:1062200004331152B15202320C2B0D46EBD11E48F1
:106230000188012914D1224B224A022011701D70BD
:10624000FEF7E4F81A4A19481188036850889288C2
:10625000198058809A80174B19885888218060804F
:10626000114B1A88511E198017480378DBB10F496A
:1062700000220B68104902700868322290FBF2F08D
:106280001880486890FBF2F0588089680F4891FBAD
:10629000F2F201882046521A9A8000F0A7FEBDE86B
:1062A000F840FEF7D7BBF8BD220D00204C0D0020B2
:1062B000500D0020580D0020300D00201C1F002024
:1062C0000C0D0020040D0020250D002012000020E0
:1062D000064B02881988891A198042885988891AB8
:1062E0005980808899880A1A9A8070471C1F00205C
:1062F0000F4B10B5596804460E4888470D480E4AA2
:1063000001461278FDF7C2FE0C48038813B12046FF
:10631000FFF716FF0420FEF76BF910B12046FFF7D8
:1063200057FF07490868BDE81040FFF7D1BF00BF1D
:10633000AC1E00201C1F00202C0D0020480D00204A
:106340004C0D0020014B1860704700BF4C0D002021
:10635000014B1860704700BFD01E0020034B188807
:10636000D0F1010038BF0020704700BF640D00204D
:10637000014B1880704700BF640D00202DE9F041EB
:10638000224D2B68C11A00293CDB214E2860307851
:10639000204C012810D120698047626890472188ED
:1063A0002B686269C81828601B491C489047002167
:1063B00031700220BDE8F081A2689047E768B847D5
:1063C0001748184A0768D2F8008014493878D1F87D
:1063D00000C008F10101814208BF0021124B13489F
:1063E0001F6840F828C050F82100BC44C0EB0C07DF
:1063F00011601F6062882B680120D11830702960FD
:10640000BDE8F0810020BDE8F08100BF400E002013
:106410005C0D0020B81E0020680D0020600D0020DB
:10642000D01E00203C0E0020740D00207C0D0020AA
:10643000F8B51E4C1E4A236815681878411EB5FB36
:10644000F1F0FAF7E7FB1B49FAF7F0FC1A4907F0FD
:106450003DFC01464FF07E50FAF72AFB1749FAF748
:1064600031FC07F065FB2668154D746807462868FF
:10647000FAF7D4FB2146FAF725FC124B06461868BA
:10648000381AFAF7CBFB214607464FF07E50FAF751
:106490000FFB01463846FAF715FC01463046FAF77D
:1064A00009FB07F045FB2860F8BD00BFD01E0020A7
:1064B000740D002080E6C547B1DC423ED048874AD3
:1064C000700D00206C0D002010B5154B154A186892
:1064D000154B04781168601E1C680823B4FBF0F0AB
:1064E00091FBF3F4091B4018106090FBF3F0FAF7EE
:1064F00095FB0E49FAF79AFC0D4907F0E7FB0146B8
:106500004FF07E50FAF7D4FA0A49FAF7DBFBFAF7B4
:106510009FFD094B094A19881060481E188010BD5C
:10652000D01E0020780D0020740D002080E6C547A5
:10653000B1DC423ED048874A640D00206C0D00203B
:1065400038B5054C10256561FCF756FA034B01225E
:1065500025611A7038BD00BF000C0140500E0020AC
:10656000F8B5394B394E044632681868811A00294B
:1065700067DB00F5C335A0353560354D2846FCF79F
:1065800001FA344B28461A782946FDF77FFD324838
:10659000827B9AB100233668304F23803049314ADC
:1065A0003E602E881F460E80168063806E884E8067
:1065B0005680A380AB8887738B8093802A480178AC
:1065C00061B1234B22881888811A19806288588803
:1065D000811A59809888A288811A99801F48036877
:1065E000002B2CD0194A1168204ACB1A934216D896
:1065F0001F4C0023E26882F00801E160144818494A
:106600001A5A5C5E10B28442C8BF5A5215495C5E89
:106610008442B8BF5A520233062BEFD10FE0002359
:1066200003600F480F4A195E985E0A18022192FB18
:10663000F1F0E0525B18062BF3D1FEF70BFA0120C4
:10664000F8BD0020F8BD00BFF80C00204C0E002063
:10665000D41E0020440E0020DF1F0020580E002012
:10666000460E0020520E0020500E00207FC3C901AC
:10667000000C0140014B1860704700BF680E0020FD
:10668000014B1880704700BF6C0E0020034B188828
:10669000D0F1010038BF0020704700BF6C0E002011
:1066A0002DE9F8433C4B3D48596888473B483C4AF4
:1066B00001461278FDF7EAFC3A480388002B42D0E5
:1066C000394C256800242F782646254635490A8806
:1066D000B2F57A7F08D1354B354A00201421E850B5
:1066E00001FB0620FEF7D2F9DFF8B0802F4B38F916
:1066F0000400E9584FF014090A18EA502C4B09FB22
:106700000639FAF78BFA01464846FEF7C2F900202F
:1067100024F80800DFF88C802649B8F80020605281
:10672000012A2FD14846FEF7F6F98146DFB13846F7
:10673000FAF774FA01464846FAF780FC98B14FF42C
:106740007A73A8F80030154B1A4A18881188401A35
:106750001880518858889288401A99885880881AD9
:106760009880BDE8F883114B4FF47A72E858114BCA
:1067700000F5FA7191FBF2F0E0520F210A2001229C
:1067800006F07AF8013604350234032E9ED105490D
:106790000A88501E0880D6E7DC1E0020041F002057
:1067A000AC0E00206C0E0020680E00205C0E002055
:1067B000700E0020380F002038B505460A4C002323
:1067C0000A4829462370FBF7ADF848B9074829461F
:1067D000FAF72CFE20B905482946FAF75BFF08B105
:1067E0000120207038BD00BFAC0E0020DC1E002050
:1067F00003780BB1054A1370417809B1044B197045
:10680000807808B1034A1070704700BFAC0E0020BA
:106810002C0D0020440E00202DE9F34106460846C9
:1068200014461D46FFF7C8FF002800F08F80484A35
:1068300000231370072C3ED8DFE804F008081B275C
:10684000333D3D04022003F077F834E04FF4487004
:10685000ADF806003F4901A88DF80430FAF726FD8F
:1068600028B13D4B3A480121042219700270012CD5
:1068700021D03848FBF704F838B1374B34480221AF
:106880000122022C1970027015D03248FAF76CFE02
:1068900038B1314B2E4803210222032C19700270AB
:1068A00009D02C48FAF762FD28B12B4B2848042167
:1068B00001221970027028490B782BB90CB11C46C3
:1068C000B5E7022003F038F82448FBF7ADFB30B9F8
:1068D0002248FBF7E7F910B9042003F02DF8304601
:1068E000FFF786FF022003F015F810B1194C22685B
:1068F00090471B4801688847FCF730F818B1194BDE
:1069000003241C7002E0082003F016F8082003F0AE
:1069100001F8154CB8B1642795FBF7F63046FAF745
:106920007DF9804607FB165000B2FAF777F90F4958
:10693000FAF7C8F901464046FAF7BCF80C49FAF7ED
:10694000C1F9206001E0002222600120BDE8FC8145
:106950002C0D0020AC1E0020560D0020B81E00207B
:10696000DC1E0020440E0020740F00208988883C23
:106970000000204108B50120FCF7EEF9102002F0DC
:10698000D3FF024B00221A6008BD00BFEC1E00209E
:106990000148FCF751BA00BFEC1E002008B503689F
:1069A0001A68904708BD38B505460C4614F8011B17
:1069B00019B12846FFF7F2FFF8E738BD08B50368BC
:1069C0005968884708BD08B503689968884708BDB5
:1069D00008B50368DA68904708BD08B50368196907
:1069E000884708BD08B503685A69904708BD00008C
:1069F000034B4FF4805208B15A6170471A617047D7
:106A000000080140034B4FF4805208B11A617047EF
:106A10005A6170470008014008B5024B1968884761
:106A200008BD00BFB00E0020054B06481A68064995
:106A300082420CBF054A064A00200A60FFF7ECBFFD
:106A400084010020001BB700B00E0020056A00087A
:106A5000F1690008024B1A68501C1860704700BFAB
:106A6000B40E002010B5094A094913688C681068F3
:106A70008342F8D1074A106811684FF47A72504384
:106A8000001BB0FBF1F102FB031010BDB40E00209F
:106A900010E000E0B80E0020014B1868704700BFFE
:106AA000B40E002038B50446FFF7DCFF0546FFF7BB
:106AB000D9FF401BA042FAD338BD10B504462CB113
:106AC0004FF47A70FFF7EEFF013CF8E710BD0000CD
:106AD00070B53B4D8CB006AC06460FCD0FC495E8A3
:106AE000030084E80300304605F04CFF35480121DF
:106AF00006F01EFE44F61D20012106F00DFE0120C9
:106B0000014606F0FDFD304E06F036FE4FF6FF73EF
:106B10000CA820F8303D00242C4869468DF802402E
:106B2000FCF744F830466946FCF740F828486946C7
:106B3000FCF73CF827494A6842F000754D60FFF7C2
:106B400073FF082010233061254633612249234812
:106B50000A6806AB824205D11A199179142901D12C
:106B60001020907103EBC5021859111D0135FCF777
:106B70001DF80834032DE9D101A806F073FD019B2F
:106B80001749184AB3FBF1F01749106008684FF431
:106B90007A73B0FBF3F2511E1448154AF02341609A
:106BA00082F8233000210723816003601148FBF73E
:106BB00011FDFBF701FB6420FFF77FFF0CB070BDF8
:106BC000E822010807004000000C014000080140D5
:106BD000001001400000014084010020001BB700AC
:106BE00040420F00B80E00208801002010E000E0B5
:106BF00000ED00E00058004010B540F2DB146043A7
:106C00000D4B102208215A61841E19610A48C3687D
:106C100083F01002C260C16881F00803C36020469F
:106C2000FFF74BFF0120FFF7F7FE1920FFF745FFA5
:106C30000020FFF7F1FEE9E7000C014010B1034A24
:106C4000034B1A6003480449C8607047EFBEADDECD
:106C5000F04F00200400FA0500ED00E02DE9F04FB0
:106C600089B00793754B07460692B3F90000B3F954
:106C700002200028B8BF4042002AB8BF5242002478
:106C80008242B8BF024605922546A146A04604941A
:106C9000A24626466A49CB7813B90A79002A38D029
:106CA000022E36D0674B6548EA5EDDF818B0295EE3
:106CB00002EB4100CBF100015A46FDF7DFFE6249CD
:106CC000DDF81CC06B5E3CF90520C01A8318F8790A
:106CD000FA7E584364214FF0050E90FBF1F06FF0FF
:106CE000040151430EFB02F20393FDF7C7FEDFF8E8
:106CF00078B1039B824654F80B00544942F210725B
:106D00001818FDF7BBFE7A7C44F80B0050430113C2
:106D100004914B48C3781BB102790AB9022E2FD1D6
:106D20004649502035F90180DFF828B100FB08F210
:106D3000BB5DDFF8389135F90B0092FBF3F154F8A5
:106D400009300A1AD01842494FF47A52FDF796FEDC
:106D500035F90B1049F804000029B8BF4942B1F5D4
:106D6000207F02DD002049F8040059F80420B919F9
:106D70007D23887A92FBF3FC00FB0CFE4FEAAE19F0
:106D80002F4B1A79B2B1022E14D0DDF814B0DDF811
:106D900010C00BFB08F0CBF5FA7303FB0A020BFBE8
:106DA00009F003FB0C034FF4FA7192FBF1F293FB31
:106DB000F1F308E0D97809B1022E02D14B464246E0
:106DC00001E0049B52462349DFF8A4B0695A16F843
:106DD0000BC008B20CFB00FB6FF04F0C9BFBFCFCE4
:106DE00094441D4ACDF800C035F902C0A952CCEB3D
:106DF00000001A4ADFF87CC0019054F80C10A0582B
:106E00004018019902904018A15844F80C100199BB
:106E1000A150134A0434B15C202201FB00F090FB26
:106E2000F2F1581A009B0F49C21801366A52023516
:106E3000032E7FF42FAF09B0BDE8F08F06200020AD
:106E4000DF1F00206E110020200F0020F0D8FFFF70
:106E500080C1FFFF300F0020C80E0020E40E00208C
:106E6000FB1E0020F21E0020DC0E0020BC0E0020C5
:106E7000FE1E0020D00E00202DE9F04F002485B02A
:106E8000039305468946924606462346474AD178EB
:106E900009B91079B8B1022C17D0454B454F33F9D9
:106EA000140037F91420CAF1000102EB40005246E9
:106EB000FDF7E4FD4049039F31F9143037F9142000
:106EC000C01A83180AE0022C08D1394A99F80570D3
:106ED000B2F904101B374F43791114E03348C178DD
:106EE00071B9334F99F8042037F914101B324A4313
:106EF0000079111138B16A7C5A4301EB222102E07A
:106F0000EF795F4339112D4FDFF8C4C037F9140012
:106F1000BCF800200F1A295D7A437943DFF8B4806A
:106F2000D0124FEAE11B58F82420B17A01FB00206F
:106F3000234948F824004FF400120293CDF804C00E
:106F4000FDF79CFD1F4BDDF804C053F8241043F8F7
:106F50002470791ABCF800704FF6FF723B09B2FB3F
:106F6000F3F74F43184BDFF870C048F824005CF883
:106F7000241053F82480BF1108EB010243F8247059
:106F8000337DD11959430BEB6030104A00EB2121BE
:106F90004CF8248022F8141001340136032C029B93
:106FA0007FF474AF05B0BDE8F08F00BFDF1F002095
:106FB000062000206E110020200F0020300F00203E
:106FC0000000E0FFFC0E0020080F0020F21E002051
:106FD000200D0020BC0E0020F00E0020024B5A783D
:106FE0000AB1002058707047DF1F00200023038083
:106FF00043807047024B00221A605A60704700BFFE
:10700000DC0E0020024B00221A605A609A60704722
:10701000BC0E00200128034B14BF034A034A1A6028
:10702000704700BF140000205D6C0008796E0008F6
:107030002DE9F84F384E04463768384606F044FDCF
:107040000546384606F0B4FD76688046304606F0C0
:107050003BFD8346304606F0ABFDD4F8049006466F
:1070600029464846F9F72EFEA7688246414638462B
:10707000F9F728FE01465046F9F71AFD21688246C5
:107080005846F9F71FFE414604464846F9F71AFEEE
:107090003146F9F717FE01462046F9F70BFD314658
:1070A00004463846F9F70EFE2946F9F70BFE01466D
:1070B0002046F9F7FFFC0146504606F005FE174949
:1070C000F9F700FEF9F7B2F911A3D3E90023F9F7B4
:1070D0002BFB134B044618680D46F9F7A7F9024637
:1070E0000B4620462946F9F743F800220D4BF9F7E5
:1070F0001BFBF9F789FC06F01BFD81B20A0444BFB3
:1071000000F5B47189B208B2BDE8F88FAFF3008022
:10711000182D4454FB210940280F00200000E144B1
:10712000740F00200000244010B51D4C2088F9F792
:1071300075FD1C49F9F7C6FD06F0FAFC1A4B1880DC
:107140002088F9F76BFD01461848F9F76FFE1849DA
:10715000F9F76CFE174908601748B0F87400F9F7A2
:107160005DFD01461548F9F761FEF9F75FF90AA3DD
:10717000D3E90023F9F7AEF9F9F746FC104A10609D
:10718000082002F0C7FB18B1BDE81040FFF7D8B9DE
:1071900010BD00BFAFF300803B597E90A9E781404E
:1071A00012000020C903683F240F00200AE81C4198
:1071B00000401C46181F0020C81D0020000061442C
:1071C000341F0020AFF300802DE9F0410446006831
:1071D0000D460146F9F776FDD4F80480064641468F
:1071E0004046F9F76FFD01463046F9F763FCA768A2
:1071F000064639463846F9F765FD01463046F9F747
:1072000059FC06F0F7FE00210646F9F7EFFE70B9CB
:1072100020683146F9F70AFE314628606068F9F7C0
:1072200005FE31466860A068F9F700FEA860BDE879
:10723000F0812DE9F04F0C68836889B0D0F800A088
:10724000D0F804800646204603938B4606F03CFCAB
:107250000746204606F0ACFCDBF804408146204699
:1072600006F032FC0546204606F0A2FCDBF80820BA
:1072700004461046019206F027FC8346019806F06A
:1072800097FC394602905846F9F71CFD39460490A0
:107290000298F9F717FD594605904846F9F712FD8F
:1072A000029906904846F9F70DFD29460790584681
:1072B000F9F708FD01465046F9F704FD21468346DB
:1072C0000698F9F7FFFC01460598F9F7F3FB01462C
:1072D0004046F9F7F7FC01465846F9F7EBFB214623
:1072E00083460498F9F7EEFC01460798F9F7E0FBAE
:1072F00001460398F9F7E6FC01465846F9F7DAFB30
:107300003060029905F10040F9F7DCFC0146504677
:10731000F9F7D8FC214683460798F9F7D3FC0146D4
:107320000498F9F7C5FB01464046F9F7CBFC014646
:107330005846F9F7BFFB214683460598F9F7C2FC8A
:1073400001460698F9F7B6FB01460398F9F7BAFC2F
:1073500001465846F9F7AEFB214670605046F9F7F2
:10736000B1FC2946044609F10040F9F7ABFC01469F
:107370004046F9F7A7FC01462046F9F79BFB394642
:1073800004462846F9F79EFC01460398F9F79AFC53
:1073900001462046F9F78EFBB06009B0BDE8F08FDA
:1073A00080EAE073A3EBE0738B4206DB002801DD8B
:1073B000401A704702D04018704700207047000004
:1073C0002DE9F041524B86B01A685B6802F1004229
:1073D00003F1004301934F4B0646B3F900000092BE
:1073E000F9F71CFC00F10040F9F720F846A3D3E9B7
:1073F0000023F9F76FF8F9F707FB474C0290B4F94F
:107400000000F9F70BFC0390B4F90200F9F706FC51
:107410000490B4F90400F9F701FC6946059003A84B
:10742000FFF707FF3D4B93F84430012B16D13C4842
:10743000417869B93B4C4025226892FBF5F7D01B97
:10744000F9F7ECFB0599F9F735FBF9F701FE206038
:10745000344B4021186890FBF1F001E0324B188862
:10746000F9F7DCFB01460598F9F722FB0590304659
:10747000F9F7D0FB2D490746F9F71CFB01463846C2
:10748000F9F7D4FC2A4D07462C6805982146F9F7F0
:107490000FFB01463846F9F715FC01462046F9F77F
:1074A00009FB244C28601D4D07460398D4F8008042
:1074B00006F03EFB95F83010FFF772FF08EB000274
:1074C00004982260D4F8048006F032FB95F830105E
:1074D000FFF766FF08EB000338466360D4F80880C6
:1074E00006F026FB95F82F10FFF75AFF1249134BB1
:1074F0000A684044A0601868B6180E60411C196004
:1075000006B0BDE8F08100BF399D52A246DF913F31
:10751000280F0020021F00202C1F0020C81D002063
:10752000DF1F0020700F0020120000203661823C17
:10753000180F00200C1F0020440F0020680F0020AF
:107540002DE9F04F87B0FFF7ABF8022002F0E2F927
:10755000002800F0AD81AE48FEF7CAFEFFF782FAC0
:10756000AC4C05462768C71B3846F9F753FBAA49B8
:10757000C968F9F7A7FB8346A848256090F82E80D4
:1075800000252C462E46A64A105FF9F747FB5946C0
:10759000F9F798FB03AB5851B8F1000F27D04046DC
:1075A000F9F73CFB01464FF07E50F9F73FFCDFF85E
:1075B000B092824651464FF07E50F9F779FA55F86D
:1075C0000910F9F77FFB97490346085F0193F9F724
:1075D00025FB5146F9F776FB01460198F9F76AFA5F
:1075E00049F80500F9F734FD8F4A105303E08D493F
:1075F0008D4A605AA0528C4B0435E15E0234062C51
:1076000001FB0166BFD1894A6420138846435B436E
:10761000874803A996FBF3F6FFF70BFE082002F05C
:1076200079F920B1834803A9FFF703FE07E08248F8
:1076300003A9FFF7FEFD80480146FFF7C5FD493E5F
:107640007E49B4B23B2CB1F8F00007D97B4E08203C
:10765000B6F8F25002F05EF930BB4FE0F9F7DAFA13
:107660004FF07E518046F9F725FA01464FF07E50E3
:10767000F9F7DCFB002406466D4D404655F8141022
:10768000F9F720FB81466848005FF9F7C7FA014621
:107690004846F9F70FFA3146F9F714FB45F814009C
:1076A0000234062CE8D1D1E7B6F8F200F9F7B2FAC5
:1076B00080462846F9F7AEFA4FF07E51F9F7FAF90D
:1076C00001464FF07E50F9F7B1FB00240646594DB4
:1076D000404655F81410F9F7F5FA594A8146105FFB
:1076E000F9F79CFA01464846F9F7E4F93146F9F70B
:1076F000E9FA45F814000234062CE8D1514B4C4D00
:10770000B3F90000F9F78AFAAC6801462046012671
:10771000F9F794FC00B906464B4968684E73214658
:1077200006F0D2FA494CD5F808802060286800F1AC
:10773000004668680146F9F7C5FA414605464046E5
:10774000F9F7C0FA01462846F9F7B4F906F052FCF9
:107750000146304606F0B8FA60602068F8F766FE29
:1077600029A3D3E90023F8F7B5FEF9F74DF906F0A0
:10777000DFF9374D28806068F8F758FE22A3D3E977
:107780000023F8F7A7FEF9F73FF906F0D1F9688072
:10779000082002F0BFF82F4C08B1264800E0264828
:1077A000FFF746FC1D4D20803846FFF709FE95F88F
:1077B0007620002A00F080801D4B18689C680146E6
:1077C0005F68F9F77FFA394606463846F9F77AFADC
:1077D00001463046F9F76EF9214606462046F9F78C
:1077E00071FA01463046F9F765F906F003FC0146E7
:1077F0002046F9F71BFB18490446F9F70BFC88B340
:1078000016480021018057E03B597E90A9E781404E
:10781000F21D00205C0F0020DC1E0020C81D00208F
:10782000041F00201C1F00202C1F0020120000201D
:10783000381F00204C0F002018000020181A0020CC
:10784000D41E0020240F0020DF1F0020280F00205E
:10785000200F0020021F00208FC2753C480F00201F
:10786000780F0020204606F0DFF9274B1968F9F75A
:1078700029FA06F05DF9B0F5617FA8BF4FF4617099
:10788000F8F7C2FD1EA3D3E90023F8F74DFFF9F77F
:10789000BBF806F08DF9044695F87600F9F7BEF9C5
:1078A0002146F9F70FFA06F043F9184B188003E068
:1078B000174B188058809880164A5379012B164B25
:1078C00007D0164819885A889B8801804280838097
:1078D00011E01349B3F90420B1F9000002EB4000B4
:1078E000032290FBF2F080B20C4A088019885B8872
:1078F00090801180538007B0BDE8F08FAFF3008017
:10790000A2EB0FE5DD169640341F0020480F002043
:107910001C1F0020181A0020041F0020300F002018
:10792000360F0020AFF30080044A054805490023C4
:1079300013605360936003600B6070470C1F00205E
:10794000680F0020440F0020028840F23E6302F2DC
:107950001F318AB29A4208D8408800F21F3188B29B
:1079600098428CBF00200120704700207047000023
:107970002DE9F04707462D4889469046FFF7E4FF7A
:10798000002850D02A4B2B4918680A682A49801AC7
:107990004FF4FA72FDF772F80A21FFF701FD274C48
:1079A00080262579264968434FF4967290FBF6F0BD
:1079B000FDF764F8C71BA07A20237843204990FB89
:1079C000F3F04FF49672FDF759F8217D1D4D4F43AA
:1079D0002E68082297FBF2F71B494FF44832824683
:1079E000B8192860FDF74AF806462860A07FF9F725
:1079F00015F9414604464846F9F75CF80146204629
:107A0000F9F760F94FF07251F9F75CF9F9F720FBDB
:107A10006FF095019622FDF731F84FF4806396FBE5
:107A2000F3F6301A5044BDE8F08700BF200F002065
:107A3000281F0020241F00200CFEFFFFC81D00206F
:107A4000D4FEFFFF640F002000E0FCFF2DE9F04FA3
:107A500085B0FFF707F8674B46F2A7121E68861B32
:107A6000964240F2C2801860FEF778FC30B9FEF70B
:107A70002BFD614C6149002008602060FEF7D8FCB6
:107A80005F4F604B38600546186801950097F9F71D
:107A9000C1F85D490446F9F715F95C4A82469068D9
:107AA000F9F7BCF805465A48DFF888B10068F9F7DD
:107AB000B5F801462846F9F7B9F956490546096867
:107AC000F9F700F92146F9F7FDF84FF07C510390E2
:107AD000F9F7F8F85146F9F7F5F8484C8446276865
:107AE00051463846CDF808C0F9F7ECF8DDF808A0A3
:107AF000DFF80481DBF8409001465046F8F7DAFFE2
:107B0000D8F80010F8F7D6FF4946F9F7DBF8019BE3
:107B100082461846F9F782F8494602464FF07E50F1
:107B20000192F8F7C5FF01460198F9F7CBF8014635
:107B30005046F8F7BFFFC8F80000F9F789FA364950
:107B4000086003993846F8F7B5FF2060FFF7ECFEB0
:107B5000009FD7F80080314F3B68C3EB0800F9F76E
:107B60005DF82F49F9F7AEF881463046F9F752F83B
:107B700001464846F9F75AF9F9F76AFA4FF496724E
:107B80002849C7F80080FCF779FF0A21FFF708FCB5
:107B9000DBF83C60216880463046F9F793F80746E9
:107BA0004046F9F73BF8314680464FF07E50F8F7F3
:107BB0007FFF01464046F9F785F801463846F8F759
:107BC00079FF206005F0B4FF05210646FFF7E8FBCA
:107BD000154C29462060154C30462268FFF7C8FE38
:107BE000134A25601060012000E0002005B0BDE8C8
:107BF000F08F00BF1C0F00206C0F0020840F0020AE
:107C0000700D0020440F0020BD3786350C1F00206A
:107C1000680F0020181F0020241F0020580F00208C
:107C200000247449D4FEFFFF400F0020140F0020F1
:107C3000600F0020C81D002010B5054C00202188D1
:107C4000FBF758FA61880120BDE81040FBF752BAF3
:107C50002400002010B5094C206009480160094942
:107C600009480A60094A0A491360029B039A0360A3
:107C70000848049B0A60036010BD00BF940F0020F9
:107C800064100020601000208C0F0020681000207D
:107C9000980F00205C100020094B1A6802EBC0010D
:107CA000CB79FF2B04D01BB1064830F8130004E059
:107CB0000728D4BF888840F2DC5000B2704700BF6C
:107CC000940F002036200020054B1A6802EBC000FC
:107CD00090F9063019420CBF01204FF0FF30704779
:107CE000940F002010B500244FF48040FCF780FC76
:107CF00008B1054B00E0054B1868054A8188A15280
:107D00000234182CF0D110BD641000206010002047
:107D10005C1F0020F8B53A4B3A4E0546187006EB4A
:107D2000C0000F46384C417820202160FCF760FCF1
:107D300008B101222260162D19D1002438590021E2
:107D4000F9F754F928B14FF48040FCF751FC50BBCF
:107D500025E02E4A3B1916190FCB86E80F002C4858
:107D6000103401784A1CC02C0270E7D1EBE716F8FA
:107D7000357006EBC506264BD6F804E01F70BEF141
:107D8000000FE0D00024BC42DDDA204E200136187E
:107D90000EEB00010FC9013486E80F00F3E7082D50
:107DA0001C4B23D124E01A4F3F78012FF7D91A4CEE
:107DB00000261034BE42F2DA54F8100C4FF07C5119
:107DC000F8F780FF4FF07C5144F8100C54F8140C75
:107DD000F8F778FF4FF07C5144F8140C54F80C0C71
:107DE000F8F770FF013644F80C0CE2E70E2D01D1D4
:107DF000012000E000201874BDE8F840FFF772BFD2
:107E00008A0F0020E42601086C1000209C0F00203F
:107E1000900F0020DF1F0020A40F0020F0B58C463B
:107E2000461C002300224CF803201033C02BF9D14C
:107E30000A4800EBC6014F6807B9F0BD0024074BA4
:107E400013F83620944208DA20010CEB00053918AB
:107E50000FC9013485E80F00F1E7F0BDE426010801
:107E6000284B10B5186800284AD027490A78531EB5
:107E7000142B3DD8DFE803F00B3C3C24403C3C1C79
:107E80003C3C3C3C3C2C3C3C3C3C3C242C001F48B7
:107E900001684A7832B11E4900204989BDE8104086
:107EA000FBF728B91B4B58780028F4D10146F5E7B9
:107EB000174C0020E188FBF71DF901202189EDE72F
:107EC000134C00202189FBF715F901206189E5E7B2
:107ED0000F4C0020E188FBF70DF901202189FBF709
:107EE00009F902206189FBF705F90320A189D5E78B
:107EF0002020FCF77DFB18B1BDE81040FFF79CBEC9
:107F000010BD00BF6C1000208A0F002068100020F8
:107F100024000020DF1F002010B50024064B187835
:107F2000A04208D90549204631F814100134FBF766
:107F3000D5F8E4B2F2E710BD900F0020441F0020F6
:107F4000064B1A780023D9B2914204D2044921F891
:107F500013000133F7E7FFF7DFBF00BF900F0020EA
:107F6000441F00202DE9F74FA34B187803280FD9A1
:107F7000A249A34CB1F904206FF06305002AB8BFF1
:107F80005242A91AB4F904006432FCF777FDA080CC
:107F9000994A1678012E1DD89A4E3478651E9A4C4F
:107FA000142D00F2C981DFE815F0A400C701C70154
:107FB0007B00B300C701C7015A01C701C701C70150
:107FC000C701C701D000C701C701C701C701C70169
:107FD0005F00A1018D488A4B884F0168B7F806B051
:107FE000B3F800805F88B3F904A0894C01910025A3
:107FF0001034B542D0D20FFA8BF0F8F70FFE54F8D8
:10800000101CF8F75FFE814638B2F8F707FE54F807
:10801000081CF8F757FE01464846F8F74BFD814625
:108020000FFA88F0F8F7FAFD54F80C1CF8F74AFE3E
:1080300001464846F8F73EFD019A814692F9000054
:1080400041420AFB01F0F8F7E9FD54F8041CF8F787
:1080500039FE01464846F8F72DFDF8F7F9FF6D4B5C
:1080600023F815000135C3E701210420FFF72CFE9A
:10807000634D654C6E88704387B204202781FFF7FB
:108080000BFE3818208101210520FFF71DFE2B88EB
:10809000584385B205206581FFF7FEFD2B1826E0C9
:1080A00002210420FFF710FE554C0121A6887043E1
:1080B00087B20420FFF708FE6588534C00FB057269
:1080C000042097B2FFF7E8FD38182081022105202F
:1080D000FFF7FAFD7043012186B20520FFF7F4FD9A
:1080E00000FB056105208DB2FFF7D6FD2B186381DB
:1080F00022E101210520FFF7E7FD414A424E978822
:10810000784384B20520FFF7C7FD2018708113E182
:10811000414900200D68FFF7BFFD404F95F906303B
:10812000B7F902607343322693FBF6F28018208081
:108130000120FFF7B1FD95F90E10B7F90050694322
:1081400091FBF6F3C7186780F6E03549354E4A785B
:10815000376812B9B888E08108E0284C3988B4F94A
:1081600006007A88FCF78AFC274BD881264D2E4FD3
:10817000E989284A3E681180347854B3264D02209C
:10818000FFF78AFD2B68B3F91010B3F91220FCF742
:1081900075FC2649264B0A68198854890EB2201AA4
:1081A00002B2964203DA3E683278511803E003DDEA
:1081B0003F683878091A19802D681D4F95F91630D7
:1081C000B7F90000642143430F4A93FBF1F6A41969
:1081D0009480134D0C4BAF7A67B1084801880E4A62
:1081E000D9801981868817685E814488064D9C81F4
:1081F00003241FE00248F1E7900F00200620002032
:10820000F21E00208A0F00202400002068100020A9
:108210009C0F0020441F0020940F0020200F0020FE
:10822000DF1F0020601000208C0F0020980F00201E
:10823000880F002007EBC40393F90600B5F9061078
:108240006426414391FBF6F6EE802046FFF724FDBD
:1082500001343218EA800235072CEBD16CE0A54FCF
:10826000A54B78781E6810B9B588E58108E0A34968
:108270007288B1F906003188FCF700FCA04AD08171
:108280009F4C9C4B9F48E7899E7A078001210320E1
:108290001EB1FFF719FD994D02E0FFF715FD9A4D4C
:1082A0006E880221704387B20320FFF70DFD2D88F1
:1082B00000FB05710420E1800121FFF705FD7043FB
:1082C000022186B20420FFF7FFFC00FB05620320B9
:1082D0002281FFF7E1FC8A4CE388C018E08004208B
:1082E000FFF7DAFC2789C519258125E0864A032492
:1082F000978802212046FFF7E7FC7843012186B2E8
:108300002046FFF7E1FC804DC4F10603590835F81B
:1083100011207B4D00FB026086B225F814602046D8
:10832000FFF7BAFC331825F814300134072CE0D1DC
:10833000724F744AF98811802020FCF759F90028FF
:1083400045D00020FFF7A8FC6D4F0546388001207E
:10835000FFF7A2FC6D4978800B7A002B37D06C4A6E
:108360006C4B14686C4A267806F00201CCB2D4B18A
:108370001468B3F9001094F90E2094F906404A43AA
:10838000322192FBF1F6B3F90230B2B26642734386
:108390006FF0310493FBF4F69419651993FBF1F136
:1083A0003D80561811E01168B3F9026091F906405A
:1083B0003222664396FBF2F42D193D8091F90E109E
:1083C000B3F900304B4393FBF2F680197880002616
:1083D000514F4B4D3B68A85F03EB860233F92610E3
:1083E000B2F90220FCF74AFBA8530236102EEFD157
:1083F000474C2168087800F00407FBB22BB9414ACA
:10840000464C1688277801231CE0454D2E780E2E09
:108410000AD0082E08D0434A02EBC604617800292E
:1084200014BF0225002500E0042500263E4F7019E8
:1084300007EB4603C0B219890136FAF75BFE042E3A
:10844000F4D1DCE7BB4209D22E4C36B234F913101A
:108450000133B142A8BF0E46B6B2F3E70024274667
:108460002E490878874272D2234D31B22B685A8840
:10847000914204DD2348951B235AEA1822524FF4F7
:108480008040FCF7B5F81F4DC0B1284A264B106854
:10849000B3F906104389184A9942254905DD096850
:1084A0001268285F4988528804E012680B68285FC8
:1084B00091881A88FCF7E2FA28533EE0DFF838800A
:1084C000285FD8F8003005EB040919885A88FCF7B2
:1084D000D5FA164A144913682853B1F90600998948
:1084E00088422ADA1020FCF783F8D8F8002008BB6D
:1084F000108820E0DF1F00206010002006200020F0
:1085000024000020441F0020F21E0020F01F002045
:108510005C100020200F0020940F0020900F0020FE
:108520008A0F0020E426010836200020980F002042
:10853000641000209088A9F80000064843781BB911
:1085400005490648625A22520137023488E7BDE8DD
:10855000FE8F00BFDF1F00205C1F0020441F002093
:10856000024B1868003018BF012070476C100020C3
:1085700044F25063984203DDA0F50C40A0387047E8
:1085800003498842BCBF00F50C40A030704700BFD3
:10859000B0B9FFFF10B5F8F741FB00210446F8F72A
:1085A0004DFD08B1204601E004F100400549F8F70F
:1085B0003DFC0549F8F786FB05F086FA034B186089
:1085C00010BD00BF8096184B35FA8E3C3800002055
:1085D00010B5044C002320702361FEF75DFA606142
:1085E00010BD00BF78100020F8B51D4614460E4699
:1085F000F8F714FB6968F8F765FB3146F8F762FB9A
:108600002168F8F757FA2060F8F722FDED68074671
:1086100005F10040F8F71CFD06462846F8F718FD5E
:10862000314602463846FCF729FAF8F7F7FA206097
:10863000F8F70EFDF8BD0000F8B5101A0C461F46FD
:10864000F8F7ECFA0546381BF8F7E8FA174B079EDF
:108650001968F8F737FB294604462846F8F732FB35
:10866000214607462046F8F72DFB01463846F8F725
:1086700021FA05F0BFFC0E49F8F724FBF8F70EFDD0
:1086800006990860214605F1004005F01DFB0949E7
:10869000F8F718FB0849F8F70DFAF8F7D9FC0028A5
:1086A000BCBF00F50C40A0303060F8BD38000020A1
:1086B0002C7D8E3FA00CB34500A00C4610B504469F
:1086C000002003460D49CA5CA2B12E2A04D1013311
:1086D00094B1C91800220A55084A0A21D25C4843BD
:1086E000A2F13001092901D8303880180E2B02D8A8
:1086F0000133E7E710BD002010BD00BFD2120020FB
:108700002DE9F843224B074648681D68381A0C4685
:108710009146F8F783FA2946F8F788FB1D4920614E
:108720000A6880469078F8F775FAF7F77FFE16A387
:10873000D3E90023F7F7CEFE02460B460020164988
:10874000F7F7F2FFF8F760F92946F8F7B3F90146B1
:108750002846F8F76BFBA668054631464046F8F711
:10876000A7F901462846F8F7ADFA01463046F8F772
:10877000A1F9D9F8081020616760A060F8F7A2FAA3
:10878000F8F766FCBDE8F883182D4454FB21194026
:10879000801100204C1100200000F03FAFF300805A
:1087A000014B1860704700BF4C110020F8B52D4BED
:1087B000187810B1012850D10AE02B4B2B4A587879
:1087C0002B4B02EB001149681868FEF701F941E0F4
:1087D000274D2868FEF701F900283ED0224C217869
:1087E000264601291ED1FEF757F906466069321A5E
:1087F000632A35D92169042912D81C4F286807EB50
:1088000001135968FEF7E4F8607807EB0017B968C0
:108810002868FEF7C8F822696661511C21611CE0D6
:10882000022018E022693AB96478104B286803EBFB
:1088300004114968FEF7CCF833690B4C8B2B09D82F
:108840000C4A0B48D15C0068FEF7A8F821694B1C64
:10885000236102E00320FFF7BBFE034A00205060C3
:10886000F8BD00BF6C11002078100020642B0108B7
:1088700048110020D62A010810B50B4CE37A8BB1C1
:108880000A48017804290DD9094A0A4B1068516831
:1088900018605960FFF77EFE0748084B02880121E7
:1088A0001A80217310BD00BFDF1F0020CC1F0020E5
:1088B000B41F0020981F0020021F00205411002028
:1088C000002370B51C460F48002119521420604344
:1088D0000D4A0E4E0E4D9952002232505953351802
:1088E0000C4E6960AA60325035180B4E0134696035
:1088F000AA6002333518022C32506960AA60E2D1B6
:1089000070BD00BF7C1100206E11002008110020F6
:10891000A8120020901000209411002070B5044689
:108920000079F8F777F91E49F8F780FA1D4D1E4EC9
:108930002860A07BF8F76EF91949F8F777FAEE602E
:1089400068606079F8F766F91849F8F76FFA184D1A
:108950002860E07BF8F75EF91149F8F767FA68607C
:10896000607EF8F757F91349F8F760FAEE60A860EF
:10897000A079F8F74FF90D49F8F758FA0E4D28602D
:10898000207CF8F747F90649F8F750FA6860A07EAE
:10899000F8F740F90749F8F749FAEE60A86070BDAA
:1089A0000000C842341100200000FA4400002041B9
:1089B000B012002000007A44F41000202DE9F341A9
:1089C0001A4F0E461A491B4D3A701B4A0860002088
:1089D0001360DDF82080FFF7FBFD6E70FEF75CF89A
:1089E000A860387800246C60A0420CBF01250325E4
:1089F0004046FFF793FF114B214603EB0616009408
:108A0000102072682B4602F011F90D49086030B948
:108A10004FF4807002B0BDE8F041FBF769BF012060
:108A200002B0BDE8F041FFF7D3BD00BF6C110020DC
:108A3000C4120020781000204C110020642B010883
:108A400048110020F7B5244B1D78032D3FD120207D
:108A500001F0BEFF214E044638B102F04DF93168F5
:108A60002046C968FDF7B4FF09E03268009021464E
:108A70002020D2682B4602F0D9F8044648B31848A3
:108A80000825102605610661164F3868FDF796FF28
:108A900050B1134D08266E613868FDF794FF01460A
:108AA0002046FDF77BFF2E612046FDF787FF00285B
:108AB000EAD00B4D0B4B10266E6120461F68FDF768
:108AC00082FF01463846FDF769FF2E61DCE7022090
:108AD00000E02846FEBD00BF78100020C412002030
:108AE000000C014048110020F7B50368164C174DE3
:108AF00023600968164E61600068FFF74BFD94E83B
:108B00000C0014480196009095E80300FFF794FDCF
:108B10006B68114A61683668C81A1660F8F77EF803
:108B20000E4A0F4F1168F8F7CDF8F8F791FA296857
:108B3000786020680B4A431A0B483B600168166056
:108B40000A4BCA881A80FEBD64110020B41F0020A1
:108B5000C41100207411002058110020380000209A
:108B6000C8120020D01100204C110020C01200209B
:108B7000264BF0B51D68024600F110011678144628
:108B8000AB195B78013203F00403DBB263B18A42B4
:108B9000F4D10020F0BD13B10A225343DBB210F828
:108BA000011B30395B18DBB2211A0229F3DC0021EA
:108BB000844209D911B10A225143C9B210F8012BDC
:108BC000303A8918C9B2F3E72E2E11D101340420AE
:108BD00000220A2672432678AF197F7807F004072F
:108BE000FFB217B1303A921901340138F1D100E0E7
:108BF0000022074C6420614300FB02110624054853
:108C0000B1FBF4F200FB0320F0BD00BFA401002083
:108C100040420F00809698002DE9F04F9A4B8BB0A0
:108C20001868B8B9994C21784A1E032A00F2658564
:108C3000DFE812F0F704F70442052C052068FDF781
:108C4000C2FE934904460B78012B00F0DF8008D365
:108C5000022B06D08C4C2068FDF7B0FE0028EDD129
:108C6000E0E7242C07D18B4B8B4A8C4C00211970E8
:108C700011702170C5E02C2C02D02A2C40F082808B
:108C8000854D844A2978864B157800205854854AAA
:108C9000B5B918781570472868D15978502965D129
:108CA0009878472840F01785D978472940F01385F0
:108CB0001B79412B40F00F850120107000F00BBD97
:108CC000117801293AD1022D05D11846FFF750FF3E
:108CD000754908604AE0032D07D11978532945D119
:108CE000714802685342036040E0042D05D11846E4
:108CF000FFF73EFF6C4B586038E0052D07D11B781D
:108D0000572B33D168494A68504248602EE0062DFF
:108D100007D119786548302994BF00210121C1721B
:108D200024E0072D04D1FFF7C9FC614A10701DE053
:108D3000092D1BD1FFF7C2FC5E4B16E0022915D1AD
:108D4000072D0CD10120FFF7B9FC41F21842504326
:108D50004FF47A71584BB0FBF1F0188006E0082D03
:108D600004D10120FFF7AAFC544B1880494B4A4913
:108D7000013500202A2C1D70087039D1504801247B
:108D800004703EE00D2C4E4A01D00A2C26D11478F6
:108D9000FCB1434C21786478A1F13000C3B2092BB7
:108DA00084BFA1F13703DBB2A4F1300003F00F025E
:108DB000C3B21101092B84BFA4F13703DBB2374CD6
:108DC00003F00F0289182078CBB2C21A514251EB3E
:108DD00002043B4B002018707CB912E02E490B783E
:108DE0000E2B03D82E48C45401330B70127842B9AD
:108DF0002A4B1A7854401C7003E02A4A1078012844
:108E000000D00020C00700F1338123E72D4B002262
:108E1000197808293FF61EAFDFE801F00A0511199D
:108E200027607C96A000622801D1022105E01A701B
:108E3000B52C7FF40FAF1C78611C19700AE722492A
:108E4000224A03261E7008701070214B0BE01F4E43
:108E50000421197032781E4BA1181878CAB2101864
:108E600018701C4B32701C70F4E605211970174BFA
:108E7000174E1A783078A118CAB210183070164EF2
:108E80001A703480E6E600BF4811002078100020F8
:108E90006C110020731000208C110020C8110020DC
:108EA000D212002004110020B41F0020DF1F002078
:108EB000CC1F0020861F00208A1F0020CA1100201E
:108EC000D112002051110020D411002044110020A3
:108ED0005211002074100020F21000206C49062668
:108EE0001E700A786B4BA6181878F2B2101818701A
:108EF000694B0A70198801EB0424A6B2B6F5007F0D
:108F000001D81E8003E000221A80644B1A700024EE
:108F1000634983E35E495F4E0A783078A318DAB27A
:108F2000101830705E4E0A7033885B4AC72B98BFAA
:108F30005C49108898BFCC545C1CA1B28842318037
:108F40007FF488AE072107E0514808261E70037899
:108F5000A3423FF47FAE0021504B6EE74D4E1A7096
:108F6000337883427FF476AE4F4C207806283BD08E
:108F700005D8022813D003287FF46CAE23E0122812
:108F800047D030287FF466AE464A484C1679454AA9
:108F9000102E88BF102626702178002347E0414C10
:108FA000434E6368A06821697360424B4FF47A7244
:108FB0003060414C91FBF2F6187840492680C87227
:108FC00001223F4923E037494A7912F0010004D0D9
:108FD0000E79F41E634253EB0400364908700028F2
:108FE00039D1364AD07236E02E4EF47A14F00101AF
:108FF00004D0B07AC21E534253EB02012D4E3170A1
:1090000009B92E4CE17227482E4990F82F200A709A
:1090100021E024482C498669426942F210742B4BA6
:1090200096FBF4F00A80188001222949EFE70C3200
:109030008B4210DA12F8046C264812F8034C1E54C6
:10904000254E26489C5512F8014C16781C54244C89
:109050001E550133EBE71A490A78002A3FF4FAADAE
:109060001B4B1E78002E3FF4F5AD00240C701C70D5
:109070001C4CA068E060FDF70FFDA060202000F010
:1090800053FC19490A78012A30D100232FE000BF90
:109090004411002052110020F21000205111002034
:1090A00030110020D811002074100020CD1F0020A6
:1090B000B41F002070100020861F0020DF1F00203A
:1090C00050110020CC1F00208A1F0020CA11002050
:1090D000D5110020741F0020A21F0020BC1F0020FB
:1090E000CE1F002078100020C212002001230B7038
:1090F0000C787E497E48CA7AC480002A3FF4AAAD23
:109100007C4B1C78042C7FF6A5AD4F7807B90F7304
:109110000D7B15B90FB1FFF7AFFB774E0521307806
:10912000764F421C92FBF1F301FB13243470744E12
:1091300097F800C0734D06EB840200237248734910
:109140001C58DFF814E2724E5C5094FBFEF103EB06
:10915000000A06FB01406F4F42F21074DFF8FC91E9
:10916000D95190FBF4F71668BCB253F8097010603F
:10917000C6EB07084044052643F8090090FBF6F0CB
:109180000EFB01016448BCF1010F25F8024F195094
:1091900005D1023CB4F5797F98BFCAF800100433BA
:1091A0001432082BCAD1FDF777FC5C4D5C4C2A6861
:1091B000801AF7F72FFD5B49F7F738FE2060FDF7BF
:1091C0006BFC286025684FF07E512846F7F718FFA2
:1091D00008B94FF07E55256006A907AC4A48524BA6
:1091E0000194009103C80CCBFFF726FA069A64237A
:1091F0004E49B2FBF3F00880079A3C4892FBF3F328
:109200004B4C027B23800AB90A80228049490C78A2
:10921000002C36D0424F4FF07E503968F7F706FEEB
:10922000454D394E2B6804463068C01AF7F7F6FCF6
:109230002146F7F747FDF7F70BFF726869683F4D66
:109240000746501AF7F7EAFC2968F7F73BFD214675
:10925000F7F738FDF7F7FCFE04B239480225B0F9FC
:1092600002303FB2E21892FBF5F1B0F900208BB268
:10927000B918344C91FBF5F291B2638021804380A0
:1092800001802C4B0120204C1870184B61682A4A31
:1092900020681C7A516010601CB9DA79002A3FF40A
:1092A000D9AC294E294D2A4C01960095164F94E8C9
:1092B0000C00FFF7C1F961687868264E081AF7F7C5
:1092C000ADFC1E4B1968F7F7FDFCF7F7C1FE7060A7
:1092D0000A48226890F900303C68012BC4EB020177
:1092E00031603DD0022B7FF4B5ACA0E0DF1F002041
:1092F0009E1E0020CC1F0020D012002072100020E3
:10930000C810002076110020B41F0020A0120020F9
:10931000806967FF84110020C0100020B810002071
:109320008011002000007A44981F0020941F002024
:10933000A01F002071100020BC1100203800002068
:10934000CC1100208E110020C411002074110020C7
:1093500064110020C8120020809698005C11002043
:10936000002634463546DFF818C3AF4F5CF825B009
:10937000CDF80CC05846F7F751FC3968F7F7A2FC56
:10938000F7F766FEDFF8DC92A84934F80920DFF829
:10939000DC82801A83B21FB2635238460497A44F0E
:1093A000F7F73CFC3968F7F78DFCF7F751FE4FF003
:1093B000140A0AFB058A82B29E4B0498196805922A
:1093C0003B4658445246FFF70FF90599DFF8B4B20F
:1093D000DDF80CC00A1824F80B205CF82500514673
:1093E0003A46FFF78DF994494FF4FA62FBF746FBD2
:1093F00034F809303BF80420313399B2622998BF20
:109400000020801883B22BF804308C4940F6B83223
:1094100018B2FBF733FB58F80610894A01352BF8D0
:109420000400B15002341436022D9CD112E4854F51
:109430002D683E686C08B6F90820A24228BF224673
:10944000814C97B2268839B230B2814209DD794B1E
:109450007E491868F7F736FCF7F7FAFD8719BFB2AF
:1094600027807B4A7B4E14683168661A3046FFF7C6
:109470007FF80028D8BF404241F293139842CCBFF6
:109480000020012050B33046F7F7C8FB7249F7F7C8
:1094900019FC04F08DFB06462846F7F7BBFB014696
:1094A0003046F7F70FFCF7F7D3FD6C4A634910809D
:1094B00000B240F6B832FBF7E1FA201848F6A044B3
:1094C000A04203DDA0F50C40A03804E00028BCBF9A
:1094D00000F50C40A0306249086001E0604D2C604E
:1094E0005F4B1D68C5F50C502830F7F797FB5A49BC
:1094F000F7F7E8FB064604F0E7FA0990304604F077
:1095000057FB002508902C462E4638B2F7F786FB0D
:1095100008AA52F82610F7F7D5FB80465148DFF825
:109520000C91005FF7F77AFB01464046F7F7C0FA67
:10953000F7F78EFD4FF47A7224F809004A4900B219
:10954000FBF79CFA81B20BB2DFF83C8124F80910DA
:1095500018460493F7F762FBD8F80010F7F7B2FB50
:10956000F7F776FDDFF8D8A04FF0140B0BFB06AB36
:10957000049A30491FFA80FC0968434610465A464F
:10958000CDF80CC0FFF730F842460346594639F98A
:1095900004000493FFF7B4F8049ADDF80C808018F7
:1095A00008EB000CDFF8DC801FFA8CF124F80810BF
:1095B00008B240F6B8322149FBF760FA55F80A20A4
:1095C0002A4B013628F80400EA5002341435022EE2
:1095D0009BD11C480368197931B1214A6420146871
:1095E000234A94FBF0F11180224C1B88206898429A
:1095F0000ED91749174B0A681C68101BFEF7B8FFF5
:1096000042F210710028B8BF404288427FF722AB77
:10961000194B1A4A01201C88154910700C80FFF75D
:1096200019BBFFF7C3F868E034110020BC1000201C
:10963000B01200208011002030F8FFFF48F4FFFF37
:10964000941100204C110020C01200200000C842DC
:10965000C4110020D0110020D3023739F0100020AF
:10966000581100208E11002018FCFFFF90100020E0
:10967000F01E0020741100205411002072100020F0
:10968000C8120020A8120020F41000206268607840
:10969000531C411CCAB263600523B2FBF3F003FB09
:1096A00010216170FDF7F8F9154AA06015480023F4
:1096B000C372137001200BE0FDF7EEF9A36840F6CA
:1096C000C411C01A884218D9202000F035F90420AE
:1096D000FEF77EFF11E00C498A78522A7FF446ABF0
:1096E000CB784D2B7FF442AB087943287FF43EAB17
:1096F000064A02211170FFF739BB0BB0BDE8F08FAD
:10970000CC1F0020DF1F0020D212002004110020F7
:109710003D4B2DE9F047B3F90000F7F77FFA3B49DD
:10972000F7F7D0FA044604F043FA0646204604F060
:10973000CBF9DFF8EC900546D9F80000344F90F8EB
:109740000380B8F1000F2BD0324CB7F90210B4F8F7
:1097500002A00FFA8AF2881AFEF70AFFC8F1000188
:109760004246FBF78BF9B4F8008000EB0A03B7F927
:1097700000000FFA88F7C01B6380FEF7F9FED9F8E6
:109780000010CA785142FBF779F900EB080297B252
:109790002780B4F90200F7F741FA804638B206E0B4
:1097A000B7F90200F7F73AFA8046B7F90000F7F781
:1097B00035FA294607464046F7F784FA314681468E
:1097C0003846F7F77FFA01464846F7F771F912492C
:1097D000F7F72CFBF7F73CFC104C31462080404655
:1097E000F7F770FA294606463846F7F76BFA01464E
:1097F0003046F7F75FF90849F7F718FBF7F728FC49
:109800006080BDE8F08700BF021F002035FA8E3C63
:10981000A81200207C110020000020416E110020C1
:109820004C11002038B5254CE37A2246002B3ED05F
:109830002348017804293AD92248817A79B1E1791B
:10984000002939D12048214B012221721970011DB4
:10985000E271FFF749F91E490220087038BDC37A4A
:10986000E171C3B11B4A1068408900F073F890B1F0
:10987000237A002B20D115481749037017480A682E
:109880004B680125011D026043602572FFF72CF92A
:109890000F48057038BD0D48084B02780021197239
:1098A00052B901210170BDE83840FFF709B8002323
:1098B000D3711372064A137038BD00BFDF1F00203A
:1098C000CC1F0020F01F0020981F00203400002033
:1098D000721000204C110020B41F00208C1F0020AB
:1098E000094B1A68811A00290DDB084A11780429EE
:1098F00009D900F5123000F5F8721A60044BD968E6
:1099000081F01000D8607047AC120020CC1F0020FE
:10991000000C0140034B196808420CBF00200120D5
:10992000704700BFE4120020024B1A681043186011
:10993000704700BFE4120020024B1A6822EA0000C0
:1099400018607047E4120020014B1868704700BF90
:10995000E4120020094BB3F90020002AB8BF52429C
:10996000824209DAB3F902100029B8BF49428142A4
:10997000ACBF002001207047002070470620002067
:1099800010B544780078002303FB03F119396143D3
:1099900001F6C4115943414340F6C41291FBF2F160
:1099A000034A22F813100133072BEDD110BD00BF7D
:1099B000262000202DE9F04384780A276743C678E3
:1099C000C4F1640C1A4D5FFA8CFCC6F164080023E4
:1099D0001A1B12B2002A04DCB8BF204602DB0120A9
:1099E00000E0604602FB02F9404309FB06F999FBDF
:1099F000F0F0404442434FF00A0992FBF9F2B818E4
:109A000082B26A800888B1F8029012B2C0EB0909EC
:109A100002FB09F20A334FF47A7992FBF9F29BB216
:109A20008018782B25F8020FD2D1BDE8F08300BF53
:109A30000C200020014B1860704700BF4413002029
:109A4000074B19680B7A032B09D8DFE803F00202F1
:109A5000040600F001BB00F063B900F02BBA7047B8
:109A60004413002008B5037A032B12D8DFE803F073
:109A70000202070C0A490B4A00F0F6FA08E008490E
:109A8000084A00F055F903E00549064A00F01AFAC1
:109A900028B90820FAF72CFF02480022026008BD0E
:109AA0003420002040130020174B10B518600446E6
:109AB00000236089154A98520233242BF9D11448A7
:109AC00001600820FAF794FD10B12046FFF7CAFFA5
:109AD0004FF48030FAF78CFD20B120460D490E4A34
:109AE00000F0D2F80120FAF783FD28B109480A49AD
:109AF000BDE8104000F0D4B84FF40040FAF778FD0C
:109B00000028F3D110BD00BF4413002036200020F0
:109B10003C1300203420002040130020037A032B44
:109B200009D8DFE803F00202040600F0D5BA00F01D
:109B30002DB900F0E5B90020704700002DE9F84F7D
:109B400080464FF400708B46FAF752FD20B1334B3C
:109B5000186801680A6990474FF40040FAF748FD19
:109B600040B12F4C257805F10107FBB2237003F0BB
:109B7000030A05E00120FAF73BFD0028F1D18246F7
:109B80000025284C4FEA4A0A2F462748026822B986
:109B9000B8F80A20254BEA5238E018F807905846E2
:109BA0004946904706464FF40070FAF721FD30B160
:109BB0001A490B6831461868C26948469047A6F2B0
:109BC000EE2188B240F2DC5398424FF4004088BF47
:109BD000B8F80A60FAF70CFD30B90120FAF708FD71
:109BE00010B912482E5211E024F80A6022886188C8
:109BF000A3885018E288C11888180D4983B26B52A7
:109C000018B20422094990FBF2F36B520137023576
:109C10000834082FB9D1BDE8F88F00BF3C130020ED
:109C2000F8120020FA1200204013002036200020F5
:109C3000E8120020F8B505460F46441E14F8011F2F
:109C400049B1054E304607F00BFC0028F6D0861BC4
:109C5000631BBB55F2E7F8BDB42B0108014B33F889
:109C60001100704736200020014B01221A70704706
:109C700048130020034B187810B100221A700120FD
:109C8000704700BF481300200AB1024B1360012047
:109C9000704700BF5D9C00080846F9F733BB000021
:109CA000024B0B6008210170704700BF999C0008AF
:109CB000034B53F82100410801F5777290B27047C9
:109CC0004C13002038B50446FCF7CCFE104B40F690
:109CD000C4111A68821A8A421A460E4B01D9002111
:109CE00019701B7810600BB90F2C10D10A48002195
:109CF0000170084A4BB1094D182B1D4405F8014C61
:109D000003D101230370117038BD0133137038BDC6
:109D10006C130020891300204913002070130020C9
:109D2000024B03214360836041737047A0860100AA
:109D300073B50023044600930E4605230E491546CD
:109D400008200E4A00F072FF62890D4B0D49A2F502
:109D50007774640008601C605C609C60DC601C615F
:109D60005C619C61DC610DB107492960082200300B
:109D7000327018BF01207CBDC59C0008A086010080
:109D80004C1300208C130020B19C0008254B10B50B
:109D90001A780AB9002010BD00201870224B997D56
:109DA0000A07F7D458781978204A00F0070441EAE6
:109DB00004211160997801F03F04640144EAD00065
:109DC0005060DC78A00040EA9110197901F001049C
:109DD00040EA84209060587900F00F04E40144EADE
:109DE0005101D160997901F07F04240144EA1010F7
:109DF0001061DC79600040EAD111187A00F00304A8
:109E000041EA44215161597A01F01F04A40144EA56
:109E1000900090619B7AD80040EA5111D1610120F5
:109E200010BD00BF49130020701300204C13002008
:109E3000024B53F82100C0F3CF007047AC13002051
:109E400010B50446FCF70EFE154B1A68811AB1F5E1
:109E50007A6F1A46134B01D90021197010601878D7
:109E600020B9A82C1AD1104B187006E0022802D194
:109E70000E4A147001E0142801D80D490C540B4906
:109E80000130C3B20878074A4100481D834213706D
:109E900004D100230449137001220A7010BD00BFD1
:109EA000A813002090130020A6130020A713002061
:109EB000911300204FF4E13301214360836041732B
:109EC0007047000037B5002300930D46144609493A
:109ED00008204FF4E132012300F0A8FE0649086093
:109EE0000CB1064A2260082300302B7018BF0120F5
:109EF0003EBD00BF419E0008CC130020319E0008EB
:109F0000124B10B51A780AB9002010BD1049002074
:109F100018704B78012BF7D10E480278082A01D926
:109F20000821017001780C4A0023D8B2023288421D
:109F30000AD212F8010C12F8024C40EA0424074835
:109F400040F823400133F0E7012010BDA6130020A4
:109F500091130020A713002094130020AC130020BD
:109F6000114B012210B51A700446FCF77BFD0F4A15
:109F70000146106811600B1A0D4841F288318B427E
:109F800003600C4B01D900221A7018780A49E4B218
:109F90000F280C5403D109490120087010BD054A4F
:109FA000431C137010BD00BFD2130020D413002037
:109FB0002014002024140020E0130020D1130020DE
:109FC0001E4B2DE9F0411A781AB31D4C1D4D267811
:109FD000077895F800C002231B4A03F10108D45CFE
:109FE00044FA06F404F00F04E5B2BD420BD20B2D87
:109FF00009D8D55C12F8082005EA0C0502EB052506
:10A00000124A42F824500233102BE5D10B4B0022A8
:10A010001A70007888420ED90D4A107860B10D4B45
:10A020000A481A7850F8211002B1490801F57773EF
:10A0300098B2BDE8F0810020BDE8F081D113002086
:10A04000D0130020D9130020E0130020F0130020CB
:10A05000D2130020D81300204FF4E13301214360D4
:10A06000836041737047000013B5037A14465BB1F7
:10A07000012B13D1124A03201070124A07201070CE
:10A08000114803700C2308E00D4A022010700D4A9D
:10A09000032010700C48037007230B7000210091FF
:10A0A0004FF4E13208200949012300F0BFFD084ABE
:10A0B00010600CB1074B2360003018BF01201CBD9D
:10A0C000D0130020D9130020D8130020619F00086E
:10A0D000DC130020C19F0008014B1878704700BFB7
:10A0E000D1130020014B1860704700BF28140020D6
:10A0F000034B18680178D1F1010038BF0020704788
:10A1000028140020034B186801784A1E534253EB71
:10A11000020070472814002008B54FF40060FAF7D9
:10A1200067FA20B10420BDE8084000F037BD08BD43
:10A13000084B187860B108490A68537813B1074A88
:10A14000117D01E006484178081C18BF01207047C6
:10A15000012070472514002028140020F01F002043
:10A16000DF1F002008B5FFF7C3FF18B1BDE80840A6
:10A1700000F062BAFFF7C6FF18B1BDE8084000F072
:10A180009DBB08BD08B5FFF7B3FF08B100F094F818
:10A19000FFF7B8FF18B1BDE8084000F07FBA08BD6E
:10A1A0000F4B10B51878D0B1FFF7C2FF0D49044628
:10A1B0000A78824213D070B1FFF79AFF18B10A4BA8
:10A1C000186800F091F8FFF79DFF30B1064800686D
:10A1D00000F07CFA01E0FFF7D5FF02490C7010BDDA
:10A1E0002C140020261400202814002008B501217A
:10A1F000042000F0DFFC054B1870FFF78DFF0449C9
:10A200000870BDE80840FFF7CBBF00BF2514002051
:10A210002C14002008B5094B187870B1FFF788FF9F
:10A2200058B1FFF765FF08B100F0A0F8FFF76AFF2B
:10A2300018B1BDE8084000F07DBA08BD2C1400201C
:10A2400038B5064C05465E212068FCF7A7FB206860
:10A250002946BDE83840FCF7A1BB00BF3C140020F4
:10A26000024B5E211868FCF799BB00BF3C1400202C
:10A2700010B50A4C5E280146206805D15D21FCF727
:10A280008DFB20683E2105E05D2903D1FCF786FBAC
:10A2900020683D21BDE81040FCF780BB3C14002045
:10A2A00010B50446C0B2FFF7E3FFC4F30720BDE8D2
:10A2B0001040FFF7DDBF000010B5084B084C1978BF
:10A2C0002068FCF78FFB074920680968FCF780FBD2
:10A2D00020680421BDE8104000F0AABB371400201C
:10A2E0003C1400203014002037B50546042000F04F
:10A2F0006FFB154C01462060A0B14279134B816879
:10A300001A70134A11604FF41651FCF761FB206874
:10A310000221FCF767FB2068042103B0BDE8304050
:10A3200000F074BBAB784FF4165200930420022364
:10A3300000F07CFC054942792060054B80680A707A
:10A34000186003B030BD00BF3C140020371400205B
:10A350003014002008B5044B1868FCF72FFBD0F12F
:10A36000010038BF002008BD3C1400202DE9F04159
:10A37000FFF7F0FF002800F04081FCF78DFBA04BB9
:10A380001A68811A7C2940F2388118609D48047847
:10A39000651C0570002404F12406F0B2FFF750FF9D
:10A3A000994B33F91400F6F739FC984A05461088A2
:10A3B000F6F734FC01462846F6F738FD9449F6F7DF
:10A3C00081FCF6F745FE013400B2FFF769FF032C6C
:10A3D000E1D13020FFF734FF8E49B1F90000FFF7DB
:10A3E0005FFFFFF73DFF8748067816F0030629D187
:10A3F000894D1020FFF724FF2B68642493FBF4F2AF
:10A4000010B2FFF74DFF2120FFF71AFF296891FBDB
:10A41000F4F004FB101484EAE473A3EBE47318B2C1
:10A42000FFF73EFF1420FFF70BFF7C4AB2F9000054
:10A43000FFF736FF1C20FFF703FF3046FFF730FF22
:10A44000FFF70EFF6F490878430740F0B080744D66
:10A450000220FFF7F5FEB5F900300A2593FBF5F071
:10A46000FFF71EFF0220FAF7C3F8002847D06D4F10
:10A470006D4E3878347840F63401B4FBF0F26B4C12
:10A480004A4321882A2391FBF0F800FB1810B2FB05
:10A49000F3F24FEA001399B241EA022C1FFA8CFE44
:10A4A000C2F303224EEA02080620FFF7C9FE0FFAA4
:10A4B00088F0FFF7F5FE20883F78431C9AB292FBA4
:10A4C000F7F107FB1120367820806E2474431523A2
:10A4D00094FBF3F43A206427FFF7B2FEB4FBF7F6DF
:10A4E0003046FFF7DDFE3B20FFF7AAFE07FB1642D2
:10A4F00091B24C1D94FBF5F000B2FFF7D1FE202085
:10A50000FFF708FA002850D0494C1320FFF798FEB7
:10A510002568484F002DB8BF6D4295FBF7F630B265
:10A52000FFF7BEFE1B20FFF78BFE23680A26002BD9
:10A53000B8BF5B4293FBF6F142F2107591FBF5F266
:10A5400005FB121000B2FFF7ABFE2320FFF778FEE9
:10A550002368002BACBF4E205320FFF7A1FE122032
:10A56000FFF76EFE61680029B8BF494291FBF7F220
:10A5700010B2FFF795FE1A20FFF762FE6068002810
:10A58000B8BF404290FBF6F696FBF5F305FB13616E
:10A5900008B2FFF785FE2220FFF752FE6268002A0C
:10A5A000ACBF45205720FFF77BFEFFF759FE15484B
:10A5B0000378282B21D100240470FCF76DFA4FF4A6
:10A5C0007A753C24B0FBF5F61720FFF739FEB6FB91
:10A5D000F4F5B5FBF4F104FB1152100200B2FFF7E1
:10A5E0005FFE1820FFF72CFE04FB156318B2FFF77F
:10A5F00057FEBDE8F041FFF733BEBDE8F08100BF74
:10A6000038140020361400202C1F002012000020D7
:10A6100000007A44400F0020700D0020021F00202F
:10A620009C1E002010000020141A0020341400206A
:10A63000B41F0020A08601004FF4165070470000A0
:10A64000154B2DE9F04180460F4618680221FCF7B2
:10A65000C9F900242646781E84420F4D0DDA18F8F9
:10A66000041028688E190134FCF798F94FF47A70B9
:10A67000B6B2FCF717FAE4B2EDE7F1B22868FCF7DE
:10A680008DF94FF47A70FCF70DFA28680121BDE8C6
:10A69000F041FCF7A7B900BF7014002010B5084BBB
:10A6A000084C19782068FCF79DF90749206809686B
:10A6B000FCF78EF920680421BDE8104000F0B8B91D
:10A6C000A2140020701400206C14002013B5042084
:10A6D00000F07EF9144C01462060A0B14279134B82
:10A6E00081681A70124A11604FF49641FCF770F9B4
:10A6F00020680121FCF776F92068042102B0BDE84A
:10A70000104000F083B900904FF4964201230420DA
:10A7100000F08CFA054B42792060054980681A7078
:10A72000086002B010BD00BF70140020A214002009
:10A730006C140020F8B5544C2068FCF73FF9002851
:10A7400000F0A0802068FCF73EF905460520FCF7E4
:10A75000B4F98A2D21D08E2DEDD14C4C00212E2222
:10A76000204606F025F84A4A7C2323701378E0201F
:10A770007D21E07084F82C1014204FF4FA71A37737
:10A780002375482278232076607661836570628421
:10A7900084F8243020462E2171E02020FFF7BAF8FB
:10A7A0000028C8D03B4C00212C22204606F000F89F
:10A7B000A021E170384B39497C207D22207084F83B
:10A7C0002B201878CA7A6570A076002A52D03449B6
:10A7D00034480F686625FE0F97FBF0FC6672324E18
:10A7E0005FFA8CFC06FB0C7284F8295006256A433C
:10A7F00042F21073B2FBF3FE03FB1E274968277376
:10A8000091FBF0F03F0AC0B26773CF0F06FB001157
:10A810006943B1FBF3F5642203FB1513E9B202FBB4
:10A820000010010AE0732148217401885FFA8EFE4E
:10A8300063741B0A02FB0CECA374B1FBF2F2242339
:10A840005A4390B21A4A010A1388E0712172180A19
:10A850001849207518480A8801884FEA1C2EE374AD
:10A86000130A84F80AC084F80BE0A7736275A37515
:10A87000217702E0202384F8293006482C21FFF7B5
:10A88000DFFE58E7F8BD00BF7014002074140020EC
:10A89000141A002040140020CC1F0020DF1F0020CD
:10A8A000B41F0020A08601006079FEFF8A1F0020EF
:10A8B000941F0020861F0020A01F00204FF4964008
:10A8C0007047000010B500230C245C430549DAB240
:10A8D000615C814203D00133042BF5D11A46104646
:10A8E00010BD00BF3C0000202DE9F84F0C2283462C
:10A8F0000D4622480421224B05F0F0FF00260C23D0
:10A9000073431E4A02EB030898F808101BEA010F74
:10A910002DD0D05C00241B4F2201BB5CBA46834281
:10A9200003D00134E4B2042CF5D14FEA04194020DD
:10A930000AEB0907F9F75CFE20B91AF80910881E1E
:10A94000012814D96B7B13B13A7B13420FD069688D
:10A95000786881420BD3AA68BB689A4207D80A4834
:10A9600004708760C0F80480C560BDE8F88F0136C8
:10A97000042EC4D10020BDE8F88F00BF3C000020A9
:10A980008DA90008C82B0108A4140020037A002018
:10A9900023B15A1E01301340C0B2F9E70A7A22B13E
:10A9A000511E01330A40DBB2F9E7984294BF002000
:10A9B0000120704700230549DAB2595C814203D077
:10A9C0000133092BF7D11A4610467047BD2B0108F9
:10A9D00000220D4B0C2101FB0233197A814211D068
:10A9E0000132D2B2042AF4D10022074B0C2101FB20
:10A9F0000233197A014005D10132D2B2042AF4D1CE
:10AA000008467047586870473C00002010B5002386
:10AA1000064A0C2404FB03225468844203D0013309
:10AA2000042BF5D10022517210BD00BF3C00002064
:10AA30000023074A0C2101FB03225168814203D005
:10AA40000133042BF5D1002200205072704700BF63
:10AA50003C00002038B5002205461A481101431871
:10AA6000405CA84204D00132062AF6D1002038BD4D
:10AA7000154C042D0FCB84E80F0016D007D8012DFC
:10AA80000DD0022D1BD111490B6898680AE0082DE2
:10AA900011D0202D13D10D490B68D86802E00B4866
:10AAA000026850686060A06003E0FFF75BFB6060D5
:10AAB000A060204638BD2046FEF7C2FFF9E70248F5
:10AAC00038BD00BF082C0108C8140020C4140020A1
:10AAD000214B10B518600120FFF7BCFF0146012093
:10AAE000FFF702FF08B9002010BD0220FFF7B2FFF8
:10AAF00001460220FFF7F8FE0028F4D01020FFF7EF
:10AB0000A9FF01461020FFF7EFFE04464FF48070C6
:10AB1000F9F76EFD08B1002CE5D00820FFF79AFF89
:10AB200001460820FFF7E0FE04460820F9F760FD23
:10AB300008B1002CD7D00420FFF78CFF0146042079
:10AB4000FFF7D2FE04464FF40060F9F751FD08B15B
:10AB5000002CC8D0012010BDC4140020F8B50F4649
:10AB600000240D4BE05C00230B4E1D01715D72193A
:10AB7000814203D00133062BF6D100221146FFF7A4
:10AB8000B3FE80680178B94204D01034602CE8D15B
:10AB90000020F8BD0120F8BD082C010810B50446BE
:10ABA000FFF758FF01462046FFF79EFE003018BF12
:10ABB000012010BD38B505460C46FFF74BFF014696
:10ABC0002846FFF791FE28B14368187A04420CBF6B
:10ABD0000020012038BD0000F8B505460020FFF731
:10ABE00071FE104E0C272B780F4C07FB0060E15CC8
:10ABF00001720120FFF766FE07FB00626878235CA4
:10AC000002201372FFF75EFEAA7807FB0061A05CCA
:10AC100008720320FFF756FEEB7807FB0061E25C49
:10AC20000A72F8BD3C000020BD2B01082DE9FF474A
:10AC3000814603920C461E469DF83070FFF70AFFCE
:10AC400001464846FFF750FE039A054600282ED0DD
:10AC5000836890F800A093F80080B8F1030F26D81D
:10AC6000DFE808F002050D0F0097134801E01348D4
:10AC7000009721463346F8F7DBFD04460AE0002042
:10AC800000E0012021463B46F8F7BCFB3146044674
:10AC9000FBF7A8FE5CB184F80480696808484C6042
:10ACA00040F82A4049462046FFF7B0FE00E0002465
:10ACB000204604B0BDE8F087003801400044004061
:10ACC000B414002038B5064C05462060FFF784FF19
:10ACD000284600F0FFFF2068BDE8384000F0E0BEE5
:10ACE000C4140020034B187808B100F0E1BD01F056
:10ACF0007BB800BFD814002010B504462046FBF7EF
:10AD00006CFE18B90A20FBF7D8FEF7E710BD00006B
:10AD1000232801D100F0CCBD044B19680A7D824282
:10AD200002D10120FBF78ABF704700BFC414002086
:10AD300010B5441E14F8011F21B1034B1868FBF72E
:10AD40002DFEF7E710BD00BF101500200148FFF7EA
:10AD5000EFBF00BFF02D010810B50748FFF7E8FF6F
:10AD60000024064B06481A19E15852680C34F9F7CA
:10AD7000B1FFC02CF5D110BD2E2E01080C2D0108FD
:10AD8000442E010870B5FBF787FE244C244B4FF48A
:10AD90007A71B0FBF1F11A7822482378F9F79AFF1B
:10ADA000FEF7D2FD05462048204902682048B2FB44
:10ADB000F1F1F9F78FFF00241E4B53F8241051B125
:10ADC000012000FA04F0284202D01B48F9F782FF64
:10ADD0000134E4B2F0E70220FEF79CFD68B1174AA7
:10ADE000174B1178174853F82110F9F773FF1648DD
:10ADF000017A11B11548F9F76DFF154C1548FFF7A9
:10AE000097FF2488F7F7A4FD0246134821464FF424
:10AE10006C73BDE87040F9F75DBF00BF1000002003
:10AE2000141A00204C2E01088801002040420F0017
:10AE30008A2E01088C3C0108A82E0108560D00201E
:10AE4000CC2D0108AC2E0108AC1E0020B62E010846
:10AE5000200D00201C310108BA2E010838B50C68FD
:10AE60000546204606F0D8FB024628682146BDE884
:10AE7000384006F001BC000037B5037904460D46A2
:10AE8000052B34D8DFE803F003060A0D111481689E
:10AE900009782DE0806890F9001029E0836819880E
:10AEA00026E08268B2F9001022E0816809681FE09C
:10AEB000806869460068F9F7F3FF01461148F9F721
:10AEC00009FFF5B1E068F5F7A9FE6946F9F7E8FF73
:10AED00001460D48F9F7FEFE2069F5F79FFE694629
:10AEE000F9F7DEFF01460848F9F7F4FE09E0002112
:10AEF0000648F9F7EFFE25B10548E1682269F9F740
:10AF0000E9FE3EBDB32E0108B22E0108F02E010865
:10AF1000EC2E010808B50648FFF70AFF054B186834
:10AF2000FFF7EAFE0020BDE80840FBF787BE00BF40
:10AF3000F32E01081015002008B50748FFF7F8FEAA
:10AF4000064B93F8AC03F9F7F5FAF9F703FBBDE804
:10AF50000840FFF7DFBF00BF022F0108181A0020CA
:10AF60007FB5044606F058FB082825D100231F4969
:10AF7000E25C086885186E7806F00301022908BFB4
:10AF8000203AE2540133082BF1D10025665D1848C0
:10AF9000314606F065FA28B101356019314606F0F0
:10AFA0005FFA18B11348FFF7C3FE1DE0082DEDD17D
:10AFB00020461149FEF73EFE1048FFF7B9FE002378
:10AFC0000F4A04A9981890F808218818084A995C33
:10AFD0000133082B00F80C1CF2D100208DF80C0076
:10AFE00001A90848F9F776FE7FBD00BFA401002043
:10AFF000B42B01080C2F0108201B00202C2F010866
:10B00000181A0020472E010808B5FDF71BFD02287D
:10B0100001D0032804D10348BDE80840FFF788BEEB
:10B0200008BD00BF412F01082DE9F041054606F09B
:10B03000F3FA0446F9F71CFD064694B92A48FFF7CF
:10B0400077FE2A4951F8241049B1012202FA04F28C
:10B05000324202D02648F9F73DFE0134F1E7254897
:10B0600021E028462449224606F006FB58B9234829
:10B07000FFF75EFE224C54F8041F0029EFD01C4855
:10B08000F9F728FEF7E72B782D2B04D10135013C89
:10B090004FF0010801E04FF000080026134850F877
:10B0A000267027B91748BDE8F041FFF741BE284692
:10B0B0003946224606F0E0FAA0B9012000FA06F06F
:10B0C000B8F1000F03D0F9F713FC0F4802E0F9F7CD
:10B0D00099FA0E48FFF72CFE0D483946BDE8F041BD
:10B0E000F9F7F8BD0136D9E7672F0108682C010888
:10B0F000A82E01081C310108733A01087A2F0108B3
:10B10000642C01088F2F0108A92F0108B32F010813
:10B11000472E010810B504460848FFF709FE084A03
:10B12000084809490023036013700B70FCF7DAFD2F
:10B130002046BDE81040FFF7FFBE00BFBC2F01084E
:10B14000D91400200C150020D814002008B504489C
:10B15000FFF7EEFDF9F75EFABDE80840FFF7DABE4B
:10B16000D42F01082DE9F04389B0044606F054FAC3
:10B17000C6B2002E6AD17A48FFF7DAFD794C206911
:10B180000021F5F733FF38BB013677483146F9F730
:10B19000A1FD206904A9F9F783FE01467348F9F778
:10B1A00099FD606904A9F9F77BFE01466F48F9F73C
:10B1B00091FDA06904A9F9F773FE01466B48F9F700
:10B1C00089FDE06904A9F9F76BFE01466848F9F7C3
:10B1D00081FD10340C2ED2D10025664C2F46A84696
:10B1E0004FF000091034B14514DA404654F8101CF1
:10B1F000F5F760FC54F80C1C80462846F5F75AFC1D
:10B2000054F8081C05463846F5F754FC09F10109C5
:10B210000746E7E75848CDF8048002950397FFF703
:10B2200087FD002401A82358544923F00040F5F776
:10B2300005FF5349534A0434002814BF10460846FA
:10B24000FFF776FD0C2CEDD14F4871E020464F49B9
:10B25000052206F011FA38B9424B0022C11810300D
:10B26000C0280A61F8D177E020464949042206F057
:10B2700003FA054620460DBB202106F0F1F8002810
:10B280006AD0461C304606F0C7F92C4607464148AE
:10B2900050F824500DB940484AE030462946FAB2E9
:10B2A00006F0EAF940B920463C49FCF7B7FD3C48B6
:10B2B0002946F9F70FFD47E00134E8E705F02EF9DC
:10B2C000461E0B2E074643DC2046202106F0C8F818
:10B2D000054640B1451C2846F9F74AFE214B3F017F
:10B2E000D851012400E004462846202106F0B8F891
:10B2F000054640B1451C2846F9F73AFE1949013484
:10B3000001EB061250612846202106F0A9F80546F7
:10B3100040B1451C2846F9F72BFE124B013403EBD4
:10B32000061188612846202106F09AF818B91D48B0
:10B33000FFF7FEFC10E00130F9F71AFE094A032C72
:10B3400002EB0616F061F2D11748FFF70BFF03E09E
:10B3500016480C21F9F7BEFC09B0BDE8F08300BF28
:10B36000F52F0108181A00202030010826300108A6
:10B37000472E01082C1A00202A3001080AD7233C46
:10B38000F12F0108ED2F01081C31010839300108A7
:10B390003F300108B02C010844300108281A002071
:10B3A0005C3001086F3001085B330108A9300108E7
:10B3B000F8B5074606F030F9044638B91A491B4B70
:10B3C0004A791B48511E53F8211028E03846194984
:10B3D000224606F051F960B91748FFF7A9FC174C4F
:10B3E00054F8041F19B11648F9F774FCF8E715482A
:10B3F00005E000250D4B53F8256026B91248BDE83D
:10B40000F840FFF795BC38463146224606F034F93D
:10B4100001350028EED10448314645710B48BDE89E
:10B42000F840F9F757BC00BF181A0020B02C0108EB
:10B43000D1300108733A0108E5300108AC2C01084D
:10B44000A82E01081C31010844300108F830010819
:10B450002DE9F047064606F0DFF8054620B1012841
:10B4600019D133782A2B16D14748FFF761FC002405
:10B4700014266643454F4648F159F9F72BFCB81995
:10B480002946FFF7F9FC01344248FFF751FC722CC2
:10B49000EED1BDE8F08730463D2105F0E1FF002800
:10B4A00057D0441C204605F039F882462046F9F76B
:10B4B0005FFD0027054614247C43DFF8D09054F844
:10B4C0000980404606F0A8F841460246304606F09C
:10B4D000D3F8002835D14C44E068F5F79FFB0146CE
:10B4E0002846F5F7A1FD002829D02069F5F796FB3D
:10B4F00001462846F5F78EFD002820D020792279D4
:10B50000052818BF5546052A0FD8DFE802F00303C7
:10B510000606090CA1680D7007E0A268158004E01A
:10B52000A068056001E0A1680D6041461A48F9F77E
:10B53000D1FB20460021BDE8F047FFF79DBC17482E
:10B5400003E00137722FB6D11548BDE8F047FFF789
:10B55000EFBB0446142565430C4F314655F8078070
:10B56000404606F05BFB50B109484146F9F7B2FB93
:10B5700078190021FFF780FC0648F9F7ABFB01348E
:10B58000722CE7D1BDE8F0870A310108AC3C010814
:10B59000E43201081C3101081F3101082A31010879
:10B5A0004F31010810B50446204606F035F810F07A
:10B5B000FF0F07D10B490C4891F8AC13BDE81040C0
:10B5C000F9F788BB204604F0A9FF022808D8054BEC
:10B5D000064C83F8AC03F8F7BDFFF9F705FAE3E78B
:10B5E00010BD00BF181A00206C3101085B33010840
:10B5F00070B5044606F010F808B9204830E020463F
:10B600001F4906F081FC00242646254678B12CB15E
:10B61000012C06D104F082FF064602E004F07EFF12
:10B62000054600201649013406F06EFCEEE70B2DAE
:10B6300005D914480C21BDE87040F9F74BBB012C2B
:10B6400008DC114A114832F915202946BDE870403E
:10B65000F9F740BBA6F57A73B3F57A7F04D90C48A5
:10B66000BDE87040F9F736BB0A4829463246F9F77B
:10B6700031FB054820F8156070BD00BF823101081C
:10B6800025330108BC3101085C1F0020E2310108AC
:10B69000FA3101081C32010838B5054605F0BCFF37
:10B6A000C0B268B904461249124801EB4402B2F82C
:10B6B000462021460134F9F70DFB152CF3D138BD96
:10B6C000284604F02BFF142804460BDC20212846D2
:10B6D00005F0C6FE04F022FF054B03EB4404A4F87A
:10B6E000460038BD04481521BDE83840F9F7F2BAE4
:10B6F000C81D002035320108413201082DE9F04310
:10B70000584885B0584CF9F7E5FA5848FFF7C4FF98
:10B710006279574B511E574853F82110F9F7DAFA5E
:10B7200020690021F5F762FC002858D10025266920
:10B7300000213046F5F75AFC00284CD101354E481F
:10B740002946D4F81490D4F81880E769F9F7C2FABA
:10B7500030460021F5F754FC10B14848F9F7BAFA21
:10B7600069463046F9F79CFB01464548F9F7B2FABD
:10B7700048460021F5F744FC10B14048F9F7AAFA11
:10B7800069464846F9F78CFB01463D48F9F7A2FAAD
:10B7900040460021F5F734FC10B13848F9F79AFA21
:10B7A00069464046F9F77CFB01463548F9F792FABD
:10B7B00038460021F5F724FC10B13048F9F78AFA31
:10B7C00069463846F9F76CFB01462E48F9F782FACC
:10B7D00010340C2DABD12C48691CF9F77BFAF9F722
:10B7E00047F92A4C064654F8041F19B12848F9F7BE
:10B7F00071FAF8E70D46274850F8251049B10122A3
:10B8000002FA05F2324202D02348F9F763FA013511
:10B81000F1E7154B214ACE1896F808418B5C04A835
:10B8200001310519082905F8103CF2D100241C4803
:10B8300069468DF80840F9F74DFA14256543194E0D
:10B840001948A959F9F746FA00217019FFF714FBB6
:10B8500001341648FFF76CFA722CEED105B0BDE842
:10B86000F08300BF67320108181A00205B3301081B
:10B87000B02C010897320108A232010825330108D3
:10B88000B32E0108472E0108AA320108642C0108D2
:10B89000BC320108682C0108CA320108B42B010827
:10B8A000D7320108AC3C0108E03201081C31010824
:10B8B000F0B56D4B87B01A787AB96C4C01201870CE
:10B8C00002212068FFF7A2F82068F9F72DFA6848EE
:10B8D000FFF72EFA6748FFF72BFA644C2068FBF756
:10B8E0006DF8002800F0BD802068FBF76CF809288F
:10B8F0000146614A01D03F2851D1002517685F4CAD
:10B900002E462FB15E4821683A4605F0B5FE10B9C3
:10B91000254606B926465B490C348C42F1D3C6B1A4
:10B920003468D5F800E03B46E05C1EF80310814225
:10B930000DD1534A41B92D2B06D820244E48D4545A
:10B9400001330360D15404E0D0540133ECE74A4999
:10B950000B60494A14681CB1AE4201D13C4612E06A
:10B960004948FFF7E5F9AE4209D856F80C0BFFF746
:10B97000DFF93E4B09211868FBF710F8F3E73D4863
:10B98000FFF7D6F900243C4B18688442A5D237490A
:10B990003B4A0868115DFBF701F80134F3E71368CF
:10B9A0002BB9042838D13648FFF7B4FB59E00C28EE
:10B9B00001D136488CE70A2901D00D2948D12E4DF6
:10B9C0003348FFF7B5F92E4C2A6832480023A354B8
:10B9D00004930090294903A810220C23039404F037
:10B9E000A1FD054638B1006805F016FE411CAA68A5
:10B9F0006018904702E02848FFF79AF900213022AA
:10BA00001F4804F0D5FE18491B4B0A780020186027
:10BA1000002A7FF45FAF24E00C28CAD07F2903D12D
:10BA20005BE72F2B3FF659AF1F297FF656AF7E29D4
:10BA30003FF653AF13B920293FF44FAF104C581CB9
:10BA4000E1540A4A0C4B18601068FAF7A7FF44E764
:10BA50007F29E6D10A4C581E0021106021540F485E
:10BA600039E707B0F0BD00BFD81400201015002042
:10BA7000EA320108223301080C1500200C2D0108C0
:10BA8000D9140020CC2D0108273301082C330108DC
:10BA90001C3101085DAE0008373301085833010836
:10BAA00037B505460220FEF793FF064C014620609D
:10BAB00030B90090AA6802200323FFF7B7F820608E
:10BAC0003EBD00BF10150020F8B5174E174C184D9D
:10BAD0000746C1B230682170FAF760FF22782B78F0
:10BAE000C7F3072182EA0300287030682170FAF753
:10BAF00055FF21782A78306881EA0203C7F30741AD
:10BB00002B702170FAF74AFF2078297880EA010229
:10BB1000390E306821702A70FAF740FF2B782078B0
:10BB200080EA03012970F8BD1C15002017150020BC
:10BB300014150020F8B50D4E0D4D0E4CC1B2074640
:10BB400030682970FAF72AFF2A782378391282EAB6
:10BB50000300207029703068C9B2FAF71FFF2378FC
:10BB60002A7882EA03002070F8BD00BF1C1500206F
:10BB70001915002014150020054B10B50446214668
:10BB80001868FAF70BFF034802785440047010BDA0
:10BB90001C15002014150020034B04491A78885CFA
:10BBA00001321A70704700BF1515002038150020AB
:10BBB00010B5FFF7F1FF0446FFF7EEFF04EB00209E
:10BBC00080B210BD10B5FFF7F3FF0446FFF7F0FF9A
:10BBD00004EB004010BD000038B5044624200D469B
:10BBE000FFF7CAFF4D20FFF7C7FF002C0CBF3E2018
:10BBF0002120FFF7C1FF064B002228461A70FFF7ED
:10BC0000BBFF04480078BDE83840FFF7B5BF00BF70
:10BC1000141500202115002001460020FFF7DCBF8D
:10BC200001460120FFF7D8BF014B1878FFF7A4BFEA
:10BC30001415002070B5054608460E46FFF7ECFFC8
:10BC40002C467219D0B2E3B2984204D014F8010B1A
:10BC5000FFF792FFF5E770BD10B5441E14F8010F11
:10BC600010B1FFF789FFF9E710BD00002DE9F84397
:10BC7000002701240025144B187885421CDA13494B
:10BC8000134B15F801800C2202FB0830406805F0C8
:10BC9000C3FC81460CB13F180CE026464E4509DA3C
:10BCA0000B4A0C2101FB08235868805DFFF764FFF5
:10BCB0000136F3E70135DEE724B1F8B2FFF7ACFF58
:10BCC0000024D7E7BDE8F8832015002022150020C6
:10BCD0006C000020F7B5404DFF211522074628468D
:10BCE00004F066FD002302202B70FDF713FE0124F3
:10BCF00018B102206C70A87003240420FDF70AFE1E
:10BD000068B1354E03214FF400503155651CF8F7EA
:10BD10006FFC18B104227255023400E02C46022058
:10BD2000FDF7F8FD48B12C4B05201E19062107250B
:10BD300018557170B570033404E00820FDF7EAFD72
:10BD40000028F0D12020F8F753FC18B1224B08222C
:10BD50001A5501344FF48070F8F74AFC30B11E4890
:10BD60000A2601190B2506554D7002341B4A1A4B41
:10BD70005079082801D00E2802D10C261E55013416
:10BD80000D2104201955651CF8F732FC18B1124832
:10BD900011224255A51C1149132391F839210E4E49
:10BDA0006C1C101C18BF01207355F8F721FC10B152
:10BDB00014203055AC1C0A4B01201C70FEF708FE05
:10BDC000084C0146206030B900907A6801200323B6
:10BDD000FEF72CFF2060FEBD22150020181A00205F
:10BDE000201500201C150020F8B5B54C2068FAF786
:10BDF000E5FD002800F033852068FAF7E4FDB14A3C
:10BE00000346117871B9B0F12404634253EB040185
:10BE100011700029E9D1AC4A5478002CE5D1FEF725
:10BE200077FFE2E7012904D14D280CBF022300234C
:10BE300021E0022904D13C280CBF032300231AE08F
:10BE400003290FD140284FF0000101D91170CCE730
:10BE50009E489F4C03709F48217001709E490B7053
:10BE6000042308E0042908D19B499C480C780370FE
:10BE700063400B7005231370B7E70529B5D19448CB
:10BE8000924C017822788A42934A07D914785C4010
:10BE90001470934A53544B1C0370A6E710789842D1
:10BEA00040F0D8848D4B19787B2900F01F8300F275
:10BEB000C5806E2900F0698360D8682900F032835C
:10BEC00025D8652900F0068219D8642940F0BD8480
:10BED0000720844CFFF7A0FEE620FFF74DFE6079B7
:10BEE000FFF74AFE0020FFF747FE94F819017E4B4A
:10BEF0007E4A00280CBF1046184600F059BC66293F
:10BF000000F06682672940F0A08479480BE36B2932
:10BF100000F0198323D8692900F009836A2940F0C9
:10BF200094841020FFF778FE6748724CC07AFFF7C0
:10BF300023FE71490878FFF71FFE2068FFF7C4FD54
:10BF40006068FFF7C1FD6D4AB2F90000FFF7F2FD2E
:10BF50006B4BB3F90000FFF7EDFD6A4A12E36C2961
:10BF600000F003836D2940F070840620FFF754FE33
:10BF700065490868FFF7A8FD644A03E3732900F0E8
:10BF800071833CD8702900F02F83C0F00F83712992
:10BF900000F03D83722940F05884524C1620FFF780
:10BFA0003BFE0020FFF7C6FDB4F9D000FFF7C2FD4D
:10BFB000574DB4F9D200FFF7BDFDB4F9D400FFF737
:10BFC000B9FDB5F9BA00FFF7B5FD0020FFF7B2FDE6
:10BFD0000020FFF779FDB5F928000A2390FBF3F064
:10BFE000FFF7A8FD94F80401FFF7C6FD94F80601D9
:10BFF000FFF7C2FD94F80501FFF7BEFD61E3762966
:10C0000000F03B830DD8742900F01983752940F0A6
:10C010001C842F20FFF700FE3E48FFF71DFE00F0B6
:10C0200017BC772900F00E83782940F00E84384C35
:10C030003820FFF7F1FD04F1400507E2D02900F0B8
:10C04000758300F2CA80CA2900F005816CD8A42942
:10C0500000F0DA8310D8A02940F0F7830C20FFF716
:10C06000DBFD2D492D4C0868FFF72EFD2C4A10688A
:10C07000FFF72AFD20689BE3C82900F0DE80C9296C
:10C0800040F0E383FFF788FD0F4B1A4CD872FFF79F
:10C0900083FD19490870FFF795FD2060FFF792FDB9
:10C0A0006060FFF785FD154A1080FFF781FD144B96
:10C0B00018801C48017841F002040470DAE000BFE7
:10C0C0001C15002016150020DF1F00201815002069
:10C0D000371500201515002014150020211500200B
:10C0E00038150020181A00201C0000801400008061
:10C0F00024000020B41F0020CC1F0020861F002039
:10C100008A1F0020CA110020241F0020400F002099
:10C11000C81D002094450108E8F7FF1FF0F7FF1F36
:10C12000ECF7FF1FC2120020CD2900F0098322D8AE
:10C13000CB2900F0A180CC2940F08783FFF72CFDAC
:10C14000CC4CE077FFF728FD84F82000FFF724FDB2
:10C1500084F82300FFF720FD84F82400FFF71CFD7E
:10C1600084F82500FFF718FD84F82100FFF714FD7F
:10C1700084F822007EE0CE2900F0EC82CF2940F046
:10C180006483FFF715FDFFF713FDBB4CB94DA4F811
:10C19000D000FFF70DFDA4F8D200FFF709FDA4F8C9
:10C1A000D400FFF705FDA5F8BA00FFF701FDFFF782
:10C1B00009FDFFF7FDFC0A2358432885FFF7ECFC37
:10C1C00084F80401FFF7E8FC84F80601FFF7E4FCBB
:10C1D00084F80501FFF7E0FC4CE0D52900F09481DC
:10C1E0000FD8D22961D0C0F07082D3296DD0D42964
:10C1F00040F02B839F4C0020FFF70EFD04F140051B
:10C2000056E1F02900F0C7820CD8D62944D0EF2996
:10C2100040F01B83FFF7CCFC964CA085FFF7C8FCD1
:10C22000608527E0FA2900F09D82FE2940F00D8309
:10C230000820FFF7F1FC0024A5E20024FFF7B8FC7A
:10C240008E4A10530234102CF8D10020FFF7E4FC82
:10C25000FDF70AFDFCE28A4C04F10A05FFF79CFC9D
:10C2600001346070FFF798FCE072FFF795FCAC4278
:10C270006075F3D1002083E20024824801788C426B
:10C28000F8D2814D655DFFF793FC7A4A013402EBE9
:10C290004505A5F84600F0E70024FFF789FC7B4A36
:10C2A00010530234102CF8D1E4E7794C6478002C58
:10C2B000E0D1FFF771FC7049022881F8AC0388BF18
:10C2C00081F8AC43F8F746F937E2FFF771FC714BA0
:10C2D0001880CFE7704D0B20FFF79EFCB5F90000EA
:10C2E000FFF728FCF6F734FB00B2FFF723FC02202F
:10C2F000FDF710FB05460420FDF70CFB0446082063
:10C30000FDF708FB820042EA4401294320208CB259
:10C31000FDF700FB44EAC00084B21020FDF7FAFAF2
:10C3200044EA001318B2FFF705FC594A1079D17896
:10C3300084005378907944EA4101194341EAC004EA
:10C340005179537A44EA411040EA83145348C17941
:10C3500044EAC113047A417A43EA042343EA4124BC
:10C36000D379117A44EA8324927A44EAC123417B47
:10C3700043EA0234827B44EA4133017C43EA82345B
:10C38000027944EA0143417C43EA0214827C44EA94
:10C390004143C17C43EA8244007D44EAC142394BB7
:10C3A00042EA00540020197803468B420AD2364DE7
:10C3B00001225D5D02FA05F525421CBF9A4010433B
:10C3C0000133F2E72C4CFFF77FFB94F8AC0379E1E3
:10C3D0001220FFF721FC32490C88B4F5806F314CF4
:10C3E000B4F9000008D8FFF7A5FBB4F90200FFF785
:10C3F000A1FBB4F904000EE0082590FBF5F0FFF76F
:10C4000099FBB4F9020090FBF5F0FFF793FBB4F948
:10C41000043093FBF5F0244CFFF78CFBB4F90000DB
:10C42000FFF788FBB4F90200FFF784FBB4F90400BE
:10C430001E4CFFF77FFBB4F90000FFF77BFBB4F95C
:10C440000200FFF777FBB4F90400AEE1B4F978001D
:10C45000FFF770FBB4F97A00FFF76CFBB4F97C00CE
:10C46000FFF768FB94F87E000834FFF785FBAC42C9
:10C47000ECD1EDE1C81D0020181A00203620002064
:10C48000C71D002020150020221500205C1F002061
:10C49000DF1F0020F01E0020200D0020F01F0020D4
:10C4A000120000202C1F0020300F0020D41E00207E
:10C4B000FFF77EFBA4F87800FFF77AFBA4F87A0078
:10C4C000FFF776FBA0F57A7107288AB298BF84F847
:10C4D0007F00B2F57A7F98BFA4F87C00FFF75CFB81
:10C4E00084F87E000834AC42E2D1B1E10820FFF7C5
:10C4F00093FB0024B04AA31893F87F000834FFF799
:10C500003BFB402CF6D1A3E10020FFF785FB002484
:10C51000FFF742FBA84AA3180834402C83F87F0099
:10C52000F6D195E1A5481021FFF784FB90E110209A
:10C53000FFF772FB0024A248005F0234FFF7FAFA0B
:10C54000102CF8D184E10520FFF766FB9D4BB3F971
:10C550000000FFF7EFFA9C48B0F90000FFF7EAFA95
:10C560009A490A7802F00100ACE0994C0620FFF7E6
:10C5700053FBB4F90000FFF7DDFAB4F90200FFF74E
:10C58000D9FA944AB2F900000FE10720FFF744FB03
:10C5900091480078FFF7F0FA0020FFF7CBFA8F4BB5
:10C5A000B3F90000FFF7C6FA0020FEE0824C072036
:10C5B000FFF732FBE07FFFF7DFFA94F82000FFF788
:10C5C000DBFA94F82300FFF7D7FA94F82400FFF77A
:10C5D000D3FA94F82500FFF7CFFA94F82100FFF77B
:10C5E000CBFA94F822006DE01E20FFF715FB7C4C7F
:10C5F00004F10A0501346078FFF7BEFAE07AFFF72C
:10C60000BBFA607DFFF7B8FAAC42F3D120E175497F
:10C610000A78540004F0FE00FFF7FEFA0024714887
:10C6200003789C4280F014816F496348625C013456
:10C6300000EB4203B3F94600FFF77CFAEFE7FFF7A0
:10C6400015FB05E1674900240878FFF7E5FA654A1C
:10C650001078844280F0FC80634B185DFFF78CFA01
:10C660000134F4E70820FFF7D7FA0124E0B20134DF
:10C67000FFF782FA092CF9D1EAE0FFF78DFA0646B6
:10C680001220FFF7C9FA0EB9584902E0102E03D163
:10C6900057490D684C6801E0002425463046FFF7F5
:10C6A0006BFA2846FFF710FA2046FFF70DFA514AB9
:10C6B0001068FFF709FA0020FFF73CFA0020FFF7A7
:10C6C00039FA0020FFF758FAC2E0FFF765FA05468D
:10C6D000FFF778FA0746FFF775FA0646FFF772FA92
:10C6E0000446FFF765FAFFF763FAFFF755FA65B9F5
:10C6F0003E484149012207604660CD710A73002C13
:10C700003FF4B8AD3B4B1C60B4E5102D7FF4B2ADE7
:10C710003748076046600CB136490C603448374BE7
:10C720000222011D1A70FCF7DFF9A3E532484178B7
:10C7300000297FF49FADF7F76DFFF8F755F999E5FC
:10C740002D4C6378002B7FF495AD4FF4C870F9F74A
:10C75000E7FC8FE52848417800297FF48BAD012262
:10C76000827387E5244B5C78002C6ED1244991F8C4
:10C77000AC03F7F7DFFEF7F7EDFEF8F735F92046E3
:10C78000FFF74AFA64E01F48005F0234FFF7D2F96E
:10C79000082CF8D15CE0084C0420FFF73DFAB4F90E
:10C7A0002C00FFF7C7F9B4F92A00FFF7C3F94FE0EF
:10C7B000FFF78AF94CE000BFC81D0020441F00208D
:10C7C00036200020941F0020A01F0020C21200204D
:10C7D000200F0020021F0020141A0020A61E002097
:10C7E000C71D00202015002022150020981F0020C2
:10C7F0008C1F0020281F0020DF1F00207210002047
:10C80000181A00209E1E0020154C23789800411C09
:10C81000C8B2FFF701FA2078FFF7AEF90024104AFA
:10C8200013789C4214D20F48005DFFF7A5F90E491A
:10C83000085DFFF7A1F90D4A105DFFF79DF90C4B5C
:10C84000185DFFF799F90134E9E70020FFF7E8F9EF
:10C85000FFF7EAF9074900200870FFF7C6BAF8BDEC
:10C86000CD1F0020741F0020A21F0020BC1F00202D
:10C87000CE1F0020161500202DE9F04107468846FE
:10C8800016460024B44219D00025BD4210D00C4BEE
:10C890000135DA68EDB282F00800D8600120FAF7BD
:10C8A000BBF84046FAF709F90020FAF7B5F8ECE7CB
:10C8B0003C200134FAF701F9E4B2E3E7BDE8F08186
:10C8C000000C01400F4B1A6842F0010018605968D3
:10C8D0000D4A0A405A60186820F0847121F48032B1
:10C8E0001A60186820F4802119605A684FF41F01FB
:10C8F00022F4FE0058609960044B4FF000629A6089
:10C90000704700BF001002400000FFF800ED00E09B
:10C91000164A174B516801F00C00042803D0082870
:10C9200005D0144801E014490868186011E0516806
:10C930005068C1F383410231C00301D40F4A06E0BD
:10C9400052680D4812F4003F026818BF5208514364
:10C950001960064B0A485A68054BC2F30311415C43
:10C960001A6822FA01F21A60704700BF00100240F4
:10C970008801002000127A008401002000093D0097
:10C98000740100201FB50023574C4FF4E0110093B1
:10C99000019302930391226842F480332360A169DA
:10C9A00041F01002A261504C236803F40031019160
:10C9B000009A531C0093019919B9009AB2F5A06F1F
:10C9C000F1D12168484B11F4003401D0022416E063
:10C9D0001A6842F0010119600094434B1C6804F08E
:10C9E0000202019200994C1C0094019A1AB9009914
:10C9F000B1F5A06FF1D11B6899073BD501243B49E4
:10CA000002940A6842F010030B600C6824F00302E1
:10CA10000A600B6843F002040C60A1F5805359686A
:10CA200059605A685A605C68314A44F480615960C0
:10CA3000146824F0704111602E4C2F490C605C6822
:10CA400024F47C145C60146844F00044146094681E
:10CA500024F400449460043A9268120449BF274ABF
:10CA60004FF4E0120A604FF48012039202990129F8
:10CA700001D119E0FEE702291AD168B10398B0F597
:10CA8000801F02D14FF4A01205E0039BB3F5E01F15
:10CA900002D14FF400120392134B5968039841EAF4
:10CAA000000242F4803002E0596841F4601058609E
:10CAB0000D4B1A68184642F08071196002680A4BE3
:10CAC0009201FBD5596821F0030058605A6842F082
:10CAD00002015960044B586800F00C02082AF9D191
:10CAE000FFF716FF1FBD00BF0010024000200240EC
:10CAF0000410014000127A0084010020001BB700DE
:10CB0000837910B5002B29D01A4B01681C68CA43E1
:10CB100014401C605C6822405A60027902F1804433
:10CB200004F5823214682143116002689C68D14385
:10CB30000C409C60DC68407921401028D96006D107
:10CB4000986810439860D9680A43DA6010BD00F114
:10CB5000804303F5823319680A4308E001790068CD
:10CB600001F1804202F582331A6822EA00021A605B
:10CB700010BD00BF00040140064B1A68596910EA55
:10CB8000010304D010420CBF00200120704718465A
:10CB9000704700BF00040140014B5861704700BF5F
:10CBA0000004014008B5154B98420BD101214FF408
:10CBB000805000F0C9FD4FF480500021BDE80840CE
:10CBC00000F0C2BD0E49884207D14FF480400121D8
:10CBD00000F0C6FD4FF4804009E00A4A90420BD1B4
:10CBE0004FF40040012100F0BBFD4FF40040002154
:10CBF000BDE8084000F0B4BD08BD00BF00300140F2
:10CC000000380040003C00400B8810B54C8802887A
:10CC100023438C8802F441522343CC8823430C895C
:10CC200023434C8923438C892343CC89098A23439A
:10CC30001A4393B20380828B22F400631A04130C0C
:10CC40008383018210BD038819B199B241F040037A
:10CC500003E023F040010A04130C03807047818134
:10CC60007047808980B27047038919420CBF002049
:10CC700001207047426810B522F470230A6823F43B
:10CC8000807444EA02030C7943EA04224260CB68D0
:10CC90008A6884681A43084B234013434A7943EA5D
:10CCA00042038360097CC26A4B1E22F47002D9B22F
:10CCB00042EA0152C26210BDFDF7F1FF836811B173
:10CCC00043F0010101E023F00101816070478368B6
:10CCD00011B143F4807101E023F4807181607047E9
:10CCE000836843F00801816070478068C0F3C0002A
:10CCF0007047836843F00401816070478068C0F327
:10CD000080007047836811B143F4A00101E023F46F
:10CD1000A00181607047092970B54FF003040CD958
:10CD20004C4307251E3C05FA04F503FA04F3C668D4
:10CD300026EA05052B43C3600BE04C43072505FAA3
:10CD400004F503FA04F3066926EA050545EA030437
:10CD50000461062A4FF005030DD8013A53431F2200
:10CD600002FA03F201FA03F1446B24EA020242EAF6
:10CD70000103436370BD0C2A0DD853431F22233B8C
:10CD800002FA03F201FA03F1046B24EA020242EA16
:10CD90000103036370BD53431F22413B02FA03F2B8
:10CDA00001FA03F1C46A24EA02021143C16270BDB0
:10CDB00040F0BF60024B40F40031D960704700BFC3
:10CDC00000ED00E0C37810B503B3164CE168CB4327
:10CDD000C3F302244178C4F1040201FA02F10F22E4
:10CDE00022FA04F28478037822400A43110103F105
:10CDF0006043CAB203F5614181F800230078012243
:10CE000000F01F03410902FA03F007E00078012255
:10CE100000F01F03410902FA03F02031024B43F8EE
:10CE2000210010BD00ED00E000E100E030B5048C11
:10CE300024F001052C04250C0584048BA5B225F0F3
:10CE4000F3052A4342EA0313114A048C9042A4B228
:10CE50009DB215D002F50063984211D0B0F1804F19
:10CE60000ED0A3F5983290420AD002F58063984222
:10CE700006D003F58062904218BF24F00A0401D165
:10CE800024F0020444F0010421430583018430BDF1
:10CE9000002C014030B5048C24F010052C04250C26
:10CEA0000584048B058C24F440742405240D44EA85
:10CEB000022242EA0333144AADB290429BB212D02E
:10CEC00002F5006290420ED0B0F1804F0BD0A2F577
:10CED0009832904207D002F58062904203D002F56A
:10CEE0008062904207D125F0200242F0100545EA09
:10CEF000011189B204E025F0A00545F01005294391
:10CF00000383018430BD00BF002C0140224A038806
:10CF100090429BB212D002F5006290420ED0B0F166
:10CF2000804F0BD0A2F59832904207D002F5806274
:10CF3000904203D002F58062904203D14A8823F0E8
:10CF400070031343154A904208D002F58062904264
:10CF500004D023F44073CA889BB2134303808B88A8
:10CF60000A8883850C4B028598420FD003F5006236
:10CF700090420BD002F54063984207D003F58062DF
:10CF8000904203D002F58063984201D1097A01866C
:10CF900001228282704700BF002C01400010004037
:10CFA000038C70B523F001021404250C0584068C53
:10CFB0008388028B9CB222F073052B040D881A0C17
:10CFC00026F0020633042A434E880D891B0C354394
:10CFD000ADB22B43134DA8420FD005F50065A84212
:10CFE0000BD005F54065A84207D005F58065A8423D
:10CFF00003D005F58065A8420ED123F008064B89C1
:10D000008D881E4326F004032B43CE898D8924F49A
:10D0100040743543ADB22C43C98884800283818635
:10D02000038470BD002C0140038C30B523F0100246
:10D030001404250C0584038C8288048B23F02003C0
:10D0400024F4E6452C040D88240C44EA05241D0430
:10D050002B0C0D8992B243EA05134D88A4B243EA22
:10D060000513124D9BB2A84203D005F50065A842F6
:10D0700015D14D8923F080039BB243EA05134FF687
:10D08000BF751D408B8822F4406245EA0315ABB2A0
:10D090008D8942EA8502CD8942EA850292B2C98829
:10D0A000828004830187038430BD00BF002C0140CF
:10D0B000038C30B523F480721404250C0584038C92
:10D0C0008288848B23F4007324F073052C040D886C
:10D0D000240C2C431D042B0C0D8992B243EA05232A
:10D0E0004D8843EA0523124D9BB2A84203D005F5B3
:10D0F0000065A84215D14D8923F400639BB243EA31
:10D1000005234FF6FF351D408B8822F4405245EA37
:10D110000325ABB28D8942EA0512CD8942EA051298
:10D1200092B2C988828084838187038430BD00BF26
:10D13000002C0140038C30B523F480521404250CDC
:10D140000584038C8288858B94B225F4E64215040D
:10D150002A0C0D8823F4005342EA05221D042B0CEF
:10D160000D8992B243EA05334D8843EA05330A4DEF
:10D170009BB2A84203D005F50065A84205D18D8970
:10D1800024F4804444EA8514A4B2C988848082834C
:10D19000A0F84010038430BD002C014000214FF660
:10D1A000FF7383800180C18041800172704700233A
:10D1B000038043808380C380038143818381C38153
:10D1C000704700230122038043808280C380038153
:10D1D0007047038819B199B241F0010303E023F0CD
:10D1E00001010A04130C03807047B0F8443029B1E0
:10D1F0006FEA43436FEA53418AB201E059044A0C93
:10D20000A0F84420704783899BB20AB1194301E01A
:10D2100023EA010181817047038B23F00802130484
:10D220001A0C114301837047038B23F4006213042B
:10D230001A0C42EA01218BB203837047838B23F0DF
:10D24000080213041A0C114381837047838B23F463
:10D25000006213041A0C42EA01218BB283837047E7
:10D2600081847047038B23F00C0213041A0C028391
:10D27000038B9AB2114301837047038B23F44062FE
:10D2800013041A0C0283038B9AB242EA01218BB277
:10D2900003837047838B23F00C0213041A0C8283E0
:10D2A000838B9AB2114381837047838B23F440624E
:10D2B00013041A0C8283838B9AB242EA01218BB247
:10D2C00083837047F8B50B880D4604464988AA88C1
:10D2D00043B92B89FFF7AAFDE9882046BDE8F8404D
:10D2E000FFF7C0BF042B08D12B89FFF7D3FDE988D6
:10D2F0002046BDE8F840FFF7C0BF082B0E462F8937
:10D30000008C3BD120F480731804030C2384A08B81
:10D3100083B223F0F30343EA0717374B208CBFB2E5
:10D320009C4280B247EA020212D003F500639C429D
:10D330000ED0B4F1804F0BD0A3F598339C4207D0A8
:10D3400003F580639C4203D003F580639C4207D1C0
:10D3500020F4007040EA06218BB243F4807305E0AC
:10D3600020F4206041F4807140EA0103E9882046FE
:10D37000A2832384BDE8F840FFF78CBF20F48053DC
:10D380001804030C2384A38B208C23F440731B0507
:10D390001B0D43EA022242EA0733174A80B2944245
:10D3A0009BB212D002F5006294420ED0B4F1804FCD
:10D3B0000BD0A2F59832944207D002F580629442D5
:10D3C00003D002F58062944207D120F4005040EA75
:10D3D000063291B241F4805205E047F6FF52024016
:10D3E00041F480510A43E9882046A3832284BDE8A2
:10D3F000F840FFF75ABF00BF002C0140808E80B27A
:10D400007047008F80B27047808F80B27047B0F84D
:10D41000400080B27047038A828911EA030092B209
:10D4200003D011420CBF002001207047C9438AB2CB
:10D4300002827047038A30B50D460446EA8898B2E6
:10D4400020F4405111432182A3892889A98823F41B
:10D45000B05340EA0102688923F00C01024308043A
:10D46000030C1A4391B2A181A08AAA8983B223F442
:10D47000407187B01143A18201A800F0F3F8184869
:10D48000A38984420CBF0498039819B200294FF075
:10D4900019032A6803FB00F001DA510000E0910053
:10D4A000B0FBF1F16423B1FBF3F21201100903FBAD
:10D4B0001011A08900B2002806DAC9003231B1FB90
:10D4C000F3F303F0070005E009013231B1FBF3F398
:10D4D00003F00F00024390B2208107B030BD00BFBF
:10D4E00000380140838919B199B241F4005303E037
:10D4F00023F400510A04130C83817047C1F34213D3
:10D5000010B5012401F01F01A34204FA01F101D179
:10D510000C3004E0022B01D1103000E0143003681D
:10D5200012B143EA010201E023EA0102026010BDE8
:10D53000838A9BB20AB1194301E023EA0101818287
:10D540007047090A012303FA01F3DA4391B201801B
:10D5500070470000034A044B02F188305A6058605B
:10D56000704700BF2301674500200240024B1A6943
:10D5700042F080001861704700200240014BD860E3
:10D58000704700BF00200240084BDA68D20709D478
:10D59000D868400708D4D96811F0100F0CBF0420D8
:10D5A000032070470120704702207047002002408E
:10D5B00010B50446FFF7E8FF012806D11CB1FFF7BC
:10D5C000E3FF013CF8E7052010BD002C08BF052053
:10D5D00010BD000073B5002306464FF400500D4601
:10D5E0000193FFF7E5FF04281AD10E4CAAB2206977
:10D5F00040F0010121614FF400503280FFF7D8FF65
:10D60000042808D102360196019B2D0C1D804FF491
:10D610000050FFF7CDFF216941F6FE720A402261FA
:10D620007CBD00BF0020024038B505464FF43020D5
:10D63000FFF7BEFF042812D1094C236943F0020012
:10D640002061656121694FF4302041F04002226180
:10D65000FFF7AEFF216941F6FD730B40236138BD32
:10D6600000200240204B10B55A6802F00C0104293A
:10D6700003D0082905D01D4B01E01D4C2368036031
:10D6800011E05C685968C4F38342941CC90301D457
:10D69000184A06E016495B680A6813F4003F18BF91
:10D6A000520854430460104B5968C1F303121249E5
:10D6B0008C5C026822FA04F242605C68C4F30224C3
:10D6C0000C5D22FA04F484605C68C4F3C224095D32
:10D6D00022FA01F2C2605B680849C3F38133CB5C74
:10D6E000B2FBF3F2026110BD0010024000127A009A
:10D6F0008401002000093D00900100208C010020E1
:10D70000044B5A6909B1104301E022EA0000586154
:10D71000704700BF00100240044B9A6909B11043E2
:10D7200001E022EA00009861704700BF001002404B
:10D73000044BDA6909B1104301E022EA0000D86124
:10D74000704700BF00100240044BDA6809B1104373
:10D7500001E022EA0000D860704700BF00100240DC
:10D76000044B1A6909B1104301E022EA0000186174
:10D77000704700BF00100240024B5A6A42F08070AE
:10D78000586270470010024008B50B4B984207D111
:10D790004FF400100121FFF7E3FF4FF4001006E003
:10D7A0004FF480000121FFF7DBFF4FF480000021E0
:10D7B000BDE80840FFF7D4BF00540040F0B58688AC
:10D7C000044687B026F03F000D46010401A80E0C68
:10D7D000FFF748FF2C4A0399B1FBF2F087B23E43B2
:10D7E000A680238823F0010213041A0C22802B68E0
:10D7F000264A93420AD85B00B1FBF3F0013783B2AB
:10D80000BFB22784032B98BF042320E0EE884BF699
:10D81000FF72964204D103225343B1FBF3F305E0B8
:10D8200019225343B1FBF3F141F4804399B20A0545
:10D830004FF4967208BF41F00101504341F4004398
:10D840004FF47A7190FBF1F0421C91B22184A383D2
:10D85000228891B241F001032380208820F4816264
:10D8600022F002010B04AA886989180C41EA02031C
:10D870002989AA89184380B241EA0203208098B21C
:10D88000208107B0F0BD00BF40420F00A08601001C
:10D8900041F28833002103604BF6FF724FF480435E
:10D8A0008180C2800181418183817047038819B1E1
:10D8B00099B241F0010303E023F001010A04130CC3
:10D8C00003807047038819B199B241F4807303E073
:10D8D00023F480710A04130C03807047038819B184
:10D8E00099B241F4007303E023F400710A04130CAD
:10D8F00003807047038819B199B241F4806303E053
:10D9000023F480610A04130C0380704783889BB260
:10D910000AB1194301E023EA0101818070470182C5
:10D920007047008AC0B2704712B141F0010101E0B6
:10D9300001F0FE010182704702684FF6FE7313404A
:10D9400003602D4B00219842016041608160C160FD
:10D9500022D02A49884229D0294B984230D02949DF
:10D96000884237D0284B98423ED0284B984206D167
:10D9700053F8681C41F4700043F8680C7047244960
:10D98000884206D151F87C0C40F0706241F87C2C42
:10D990007047204B984206D153F8042C42F00F01F7
:10D9A00043F8041C70471C49884206D151F8183CC2
:10D9B00043F0F00041F8180C7047184B984206D11C
:10D9C00053F82C2C42F4706143F82C1C7047144916
:10D9D000884206D151F8403C43F4704041F8400C75
:10D9E0007047104B984205D153F8542C42F47021E3
:10D9F00043F8541C704700BF080002401C0002405E
:10DA00003000024044000240580002406C000240D6
:10DA100080000240080402401C040240300402401E
:10DA2000440402405804024070B506688C680D6AD0
:10DA300026F4FF4222F070060A6945EA04034C69A5
:10DA400013438A692343CC6913431C434B6A44EA5A
:10DA500003028B6A1A4332430260CB680A68496842
:10DA600043608260C16070BD0023036043608360D7
:10DA7000C360036143618361C36103624362836284
:10DA8000704719B1016841F0010303E002684FF6E5
:10DA9000FE7313400360704703680AB1194301E045
:10DAA00023EA01010160704741607047406880B21D
:10DAB00070470000C3004CBF014B024B58607047D9
:10DAC000000402400000024000B540F6D87320F088
:10DAD0000042C3F649739A4283B0014615DDB2F1A4
:10DAE000FF4F03DBF2F7E4FF03B000BD694601F02E
:10DAF000C9F800F00302012A009801990ED0022A09
:10DB000007D082B901F0D4FAEEE7002101F0D0FA93
:10DB1000EAE701F0CDFA00F10040E5E702F074F920
:10DB200000F10040E0E7012202F06EF9DCE700BFFF
:10DB300030B5C0F3C754A4F17F031E2B83B0014658
:10DB400021DC581C1DDBCD0F162B0CDD21F07F4393
:10DB500023F4000040F40000963C00FA04F005B104
:10DB6000404203B030BD114850F825402046F2F73E
:10DB7000A1FF019021460198F2F79AFF20F00041A1
:10DB800021B90020EDE7F3F763FAEAE720F07F42DE
:10DB900022F40003C0F3C75043F40001C0F1960221
:10DBA00021FA02F0002DDCD0DAE700BF744601084C
:10DBB00000B540F6D87320F00042C3F649739A428C
:10DBC00083B0014616DDB2F1FF4F03DBF2F770FFC1
:10DBD00003B000BD694601F055F800F003000128CC
:10DBE00015D002280BD0B8B900980199012202F093
:10DBF0000BF9EDE70021002202F006F9E8E70098B2
:10DC00000199012202F000F900F10040E0E70098DC
:10DC1000019901F04DFADBE70098019901F048FA0B
:10DC200000F10040D4E700BF70B58AB0064600F0AE
:10DC30002FFA224C054694F90030013303D03046C8
:10DC400002F080FB10B928460AB070BD304602F0E1
:10DC500023FB4FF07E51F3F7F1F90028F3D0184A77
:10DC6000012100253046019200910895F2F7DEFB74
:10DC700002460B461348CDE90423CDE9022302F006
:10DC800045F994F90030CDE90601022B0BD0684626
:10DC900002F03AF938B1089850B9DDE90601F2F717
:10DCA000B3FE0546CFE702F05DFC21210160F2E7FB
:10DCB00002F058FC089A0260EFE700BFA0010020C4
:10DCC0007C4601088846010800F096BB2DE9F0412A
:10DCD0008AB007460D4600F035FC854E044696F99D
:10DCE0000030013303D0284602F02CFB18B920463F
:10DCF0000AB0BDE8F081384602F024FB80460028D7
:10DD000033D128460021F3F771F90028EFD0794A82
:10DD10000121384601920091CDF82080F2F786FB70
:10DD2000CDE902012846F2F781FB002396F9004075
:10DD30000022C3F6F073CDE90623631CCDE904018C
:10DD40000DD0022C0BD0684602F0DEF8002800F05F
:10DD50009A80089818B102F005FC08990160DDE985
:10DD60000601F2F751FE0446C1E738460021F3F7F9
:10DD70003DF920B328460021F3F738F9002855D0A3
:10DD80005C4B012200243846009201930894F2F77C
:10DD90004DFBCDE902012846F2F748FB96F9004019
:10DDA00000220023CDE90401CDE90623002CCAD0CE
:10DDB00000230022C3F6F073CDE90623CFE7204607
:10DDC00002F06EFA8046002862D020460021F3F768
:10DDD0000DF900288BD0384602F062FA002886D070
:10DDE000284602F05DFA002881D0424A042100242E
:10DDF0003846019208940091F2F718FBCDE9020130
:10DE00002846F2F713FB96F9004000220023022C6B
:10DE1000CDE90401CDE9062365D0684602F074F827
:10DE2000002860D00898002899D094E7284602F08E
:10DE300037FA00283FF45BAF28460021F3F7E0F8FB
:10DE400000283FF454AF2B4A0023012138460192A9
:10DE500008930091F2F7EAFACDE902012846F2F7B9
:10DE6000E5FA3478CDE9040100220023002C32D0F9
:10DE7000CFF6F073022CCDE906232ED102F072FB0F
:10DE800021210160CEE702F06DFB2123036060E7F2
:10DE9000384602F005FA002897D0284602F000FA2A
:10DEA000002892D0204602F04DFA0146384619BBB0
:10DEB000104B0122009201930891F2F7B7FACDE9D5
:10DEC00002012846F2F7B2FA3478CDE90401002CB9
:10DED00065D100220023CDE90623684602F014F83C
:10DEE00000289FD1CAE702F03DFB2223036099E797
:10DEF000A0010020844601083D4C032200920194B9
:10DF0000CDF82080F2F792FACDE902012846F2F727
:10DF10008DFA96F90030CDE9040138460021D3B9D5
:10DF20004FF6FF734FF06042C4F2EF73CDE9062362
:10DF3000F3F766F800283ED196F90000022805D0D4
:10DF4000684601F0E1FF00287FF403AF02F00AFB0E
:10DF500022210160FDE600230022C7F6F073CDE91F
:10DF60000623F3F74DF80028E6D04FF07C51284601
:10DF7000F2F7A8FEF2F75AFA04460D4601F0CCFF7C
:10DF800002460B4620462946F2F70CFD0028D3D165
:10DF900000230022CFF6F073CDE90623CCE7002062
:10DFA000002102460B46F2F7BFFB022CCDE9060129
:10DFB0003FF464AF91E74FF07C512846F2F782FEC0
:10DFC000F2F734FA04460D4601F0A6FF02460B466E
:10DFD00020462946F2F7E6FC0028ADD14FF6FF7344
:10DFE0004FF06042CCF2EF73CDE90623A4E700BF07
:10DFF0008446010870B58AB0054600F0EFFF224C58
:10E00000064694F90030013308D0284602F09AF908
:10E0100020B128460021F2F7F3FF10B930460AB0CC
:10E0200070BD1A4A012128460026009101920896E7
:10E03000F2F7FCF92478CDE90401CDE902017CB9BD
:10E0400000220023CDE90623684601F05DFF88B178
:10E050000898A0B9DDE90601F2F7D6FC0646DDE72F
:10E060000020002102460B46F2F75EFB022CCDE9B0
:10E070000601E9D102F076FA21230360E8E702F015
:10E0800071FA08990160E5E7A00100208C460108BB
:10E09000F8B520F00043B3F17E5F044613D00BDCEB
:10E0A000B3F17C5F14DAB3F10C5F00F3A48040F6A7
:10E0B000DB70C3F6C970F8BD0146F2F7F9FC014602
:10E0C000F2F7B4FEF8BD002840F30E810020F8BD41
:10E0D0000028C0F20E8101464FF07E50F2F7E8FCB6
:10E0E0004FF07C51F2F7EEFD044600F077FF4EF65C
:10E0F0000871064620F47F65C3F611012046F2F749
:10E10000E1FD47F60471C3F64F21F2F7D3FC214637
:10E11000F2F7D8FD41F24611C3F62451F2F7C8FCDC
:10E120002146F2F7CFFD40F6A821C3F64E61F2F783
:10E13000C1FC2146F2F7C6FD4BF29001C3F6A66181
:10E14000F2F7B6FC2146F2F7BDFD4AF6AB21C3F665
:10E150002A61F2F7AFFC2146F2F7B4FD4CF22E61D2
:10E160000746C3F69D512046F2F7ACFD43F26131FC
:10E17000C3F63071F2F79CFC2146F2F7A3FD45F29D
:10E180002D71C4F20101F2F795FC2146F2F79AFDD8
:10E190004DF23911C4F21901F2F78AFC2146F2F767
:10E1A00091FD4FF07E51F2F785FC01463846F2F7BB
:10E1B0003DFE3146F2F786FD25F00F05074629465C
:10E1C0002846F2F77FFD01462046F2F771FC29460A
:10E1D00004463046F2F76EFC01462046F2F726FE72
:10E1E00001463846F2F766FC2946F2F763FC014621
:10E1F000F2F760FCF8BD0146F2F764FD4EF60871D7
:10E20000C3F611010546F2F75DFD47F60471C3F64A
:10E210004F21F2F74FFC2946F2F754FD41F2461127
:10E22000C3F62451F2F744FC2946F2F74BFD40F6C1
:10E23000A821C3F64E61F2F73DFC2946F2F742FDF4
:10E240004BF29001C3F6A661F2F732FC2946F2F7D1
:10E2500039FD4AF6AB21C3F62A61F2F72BFC2946B9
:10E26000F2F730FD4CF22E610646C3F69D5128466A
:10E27000F2F728FD43F26131C3F63071F2F718FC72
:10E280002946F2F71FFD45F22D71C4F20101F2F7A4
:10E2900011FC2946F2F716FD4DF23911C4F21901AD
:10E2A000F2F706FC2946F2F70DFD4FF07E51F2F72A
:10E2B00001FC01463046F2F7B9FD01462046F2F76F
:10E2C00001FD014642F26810C3F2A230F2F7F0FB02
:10E2D00001462046F2F7ECFB014640F6DA70C3F641
:10E2E000C970F2F7E5FBF8BD40F6DB70C4F24900F7
:10E2F000F8BD4FF07E51F2F7DDFB4FF07C51F2F7A5
:10E30000E1FC4EF60871C3F611010446F2F7DAFC9F
:10E3100047F60471C3F64F21F2F7CCFB2146F2F722
:10E32000D1FC41F24611C3F62451F2F7C1FB21465C
:10E33000F2F7C8FC40F6A821C3F64E61F2F7BAFB2B
:10E340002146F2F7BFFC4BF29001C3F6A661F2F74B
:10E35000AFFB2146F2F7B6FC4AF6AB21C3F62A61C1
:10E36000F2F7A8FB2146F2F7ADFC0646204600F086
:10E3700035FE4CF22E610546C3F69D512046F2F75C
:10E38000A1FC43F26131C3F63071F2F791FB2146F3
:10E39000F2F798FC45F22D71C4F20101F2F78AFB05
:10E3A0002146F2F78FFC4DF23911C4F21901F2F750
:10E3B0007FFB2146F2F786FC4FF07E51F2F77AFBA5
:10E3C00001463046F2F732FD2946F2F77BFC42F275
:10E3D0006811C3F2A231F2F76BFB01462846F2F74F
:10E3E00069FB0146F2F766FB014640F6DA70C4F2BB
:10E3F0004900F2F75DFBF8BDF8B521F00044B4F137
:10E40000FF4F034617DC20F00045B5F1FF4F0646ED
:10E4100011DCB1F17E5F42D08F1707F0020040EAB5
:10E42000D37775B9022F35D0032F08D140F6DB73AF
:10E43000CCF2490303E01846F2F73CFB03461846CA
:10E44000F8BDD4B1B4F1FF4F2DD0B5F1FF4F14D0CA
:10E450002C1BE4153C2C18DC002952DB1846F2F783
:10E46000E5FC01F019FF01F0EBFD012F46D0022F72
:10E4700035D0002F25D10346E1E7002E40F6DB73AF
:10E480001CDBC3F6C9731846F8BD40F6DB70C3F653
:10E49000C970EAE740F6DB73C4F24903CFE7BDE891
:10E4A000F84001F0CDBDB5F1FF4F2FD0022FF1D0D4
:10E4B000032FBBD0012F34D00023C0E7CBF6C973A4
:10E4C000BDE74BF62E51C3F2BB31F2F7F3FA40F63B
:10E4D000DB71C4F24901F2F7EBFA0346AFE74BF602
:10E4E0002E51C3F2BB31F2F7E5FA014640F6DB707C
:10E4F000C4F24900F2F7DCFA0346A0E700F100435A
:10E500009DE714F13C0FA9DA0020AEE7022F13D0EB
:10E51000032F0CD0012F40F6DB7305D0C3F64973EF
:10E520008DE74FF000438AE7CBF6497387E74CF657
:10E53000E433CCF2160382E74CF6E433C4F216035C
:10E540007DE700BF2DE9F04F31F0004987B00C4660
:10E550000D46074611D020F0004ABAF1FF4F804621
:10E5600005DD544807B0BDE8F04F01F017BFB9F121
:10E57000FF4F08DDBAF17E5FF3D14FF07E542046A5
:10E5800007B0BDE8F08F002854DB0026B9F1FF4F3B
:10E5900049D0B9F17E5F64D0B5F1804F38463ED0A6
:10E5A000B5F17C5F1FD001F077FEBAF1FF4F014655
:10E5B00021D0BAF1000F1ED0BAF17E5F1BD04FEA16
:10E5C000D87808F1FF3856EA08015FD0B9F19A4FC0
:10E5D00072DD4FF6F771C3F67F718A4513DC002DAB
:10E5E00019DB0024CBE7B8F1000FDCDB07B0BDE896
:10E5F000F04F00F0F3BC002D50DB0846B8F1000FDF
:10E600003ADB0446BBE70723C3F680739A4540F321
:10E61000E982002DE5DD4FF2CA20C7F2491001461C
:10E62000F2F750FBEDE7BAF17E5FA6D01FDD002DBB
:10E63000A5DAD6E7B9F1974F17DAB9F17E5F09DBB2
:10E640004FEAE953C3F1960049FA00F202FA00F1E9
:10E65000494501D000269CE702F00106C6F10206FA
:10E6600097E7002D1FDB3C4689E702268EE7002D49
:10E67000B7DA04F1004482E7AAF17E5156EA010AB2
:10E6800005D0012EBDD100F1004478E7384601469F
:10E69000F2F70EFA0146F2F7C9FBB2E74FF07E50EF
:10E6A000F2F7C4FBAAE74FF07E503946F2F7BEFB03
:10E6B000044664E788460108BAF5000F80F222821A
:10E6C0004FF09741F2F7FEFA6FF0170782462AF0F3
:10E6D0007F434CF2714223F400014FEAEA50C0F24A
:10E6E0001C027F38914200EB070C41F07E5740F34B
:10E6F00006824BF2D630C0F25D00814240F3B88210
:10E7000000220CF1010CA7F5000705920599A94814
:10E71000CDF804C050F821303846194604930392CE
:10E72000F2F7C6F9394681460498F2F7C3F9014673
:10E730004FF07E50F2F77AFB0246114648460292AD
:10E74000F2F7C0FABB467F10039A47F000518246A9
:10E7500001F5802320F47F60D31820F00F071946BD
:10E7600038460393F2F7AEFA01464846F2F7A0F9AD
:10E770000399814608460499F2F79AF901465846EA
:10E78000F2F796F93946F2F79DFA01464846F2F754
:10E790008FF9029A1146F2F795FA51468346504690
:10E7A000F2F790FA01468146F2F78CFA4FF24211E5
:10E7B0000346C3F6536148460293F2F783FA43F2E5
:10E7C0005521C3F66C61F2F775F94946F2F77AFA0A
:10E7D0004AF20531C3F68B61F2F76CF94946F2F75C
:10E7E00071FA4AF6AB21C3F6AA61F2F763F949461A
:10E7F000F2F768FA46F6B751C3F6DB61F2F75AF959
:10E800004946F2F75FFA49F69A11C3F61971F2F721
:10E8100051F901460298F2F755FA394681465046B9
:10E82000F2F748F95946F2F74DFA4946F2F742F93C
:10E83000394604903846F2F745FA0021C4F2400107
:10E840000390F2F737F90499F2F734F920F47F6175
:10E8500021F00F0949463846F2F734FA494607468F
:10E860005846F2F72FFA00218346C4F24001484689
:10E87000F2F71EF9039B1946F2F71AF901460498BC
:10E88000F2F716F95146F2F71DFA01465846F2F72B
:10E8900011F9834659463846F2F70CF920F47F6C9B
:10E8A0002CF00F0A4FF46051C3F676715046F2F720
:10E8B00009FA4CF2A0318146C3F29D615046F2F74D
:10E8C00001FA3946024650460292F2F7F1F8014643
:10E8D0005846F2F7EDF843F64F01C3F67671F2F7BA
:10E8E000F1F901460298F2F7E5F8059F324951F82F
:10E8F0002710F2F7DFF8DDF804B007465846F2F7C4
:10E900008DF92E4B059A049053F822B039464846AB
:10E91000F2F7D0F85946F2F7CDF80499F2F7CAF8B1
:10E9200020F47F6C2CF00F0A04995046F2F7C0F8DF
:10E930005946F2F7BDF84946F2F7BAF801463846AB
:10E94000F2F7B6F8013E56EA0806814640F0D48058
:10E950000027CBF6807725F47F6525F00F05294643
:10E960002046F2F7A5F85146F2F7ACF949460646BB
:10E970002046F2F7A7F901463046F2F79BF8294600
:10E9800080465046F2F79EF9014604464046F2F7AB
:10E9900091F8002806460546A246014620F00049A7
:10E9A00040F30181B9F1864F00F3BF8000F0AC80E5
:10E9B00006E000BFA44601089C46010894460108F1
:10E9C000B9F17C5F00F3C0804FF0000BD94621F411
:10E9D0007F6525F00F044FF4E4412046C3F6317102
:10E9E000F2F770F9514605462046F2F761F8014604
:10E9F0004046F2F75DF847F21821C3F63171F2F79D
:10EA000061F94BF68C610646C3F2BF512046F2F71E
:10EA100059F901463046F2F74DF806463146284688
:10EA2000F2F748F829460446F2F742F80146304624
:10EA3000F2F73EF8214606462046F2F743F94BF638
:10EA40004C31C3F231310546F2F73CF94EF60E2156
:10EA5000C3F2DD51F2F72CF82946F2F733F94BF205
:10EA60005531C3F68A01F2F725F82946F2F72AF95B
:10EA700040F66131C3F63631F2F71AF82946F2F75B
:10EA800021F94AF6AB21C3F62A61F2F713F82946B9
:10EA9000F2F718F901462046F2F70AF8054629462A
:10EAA0002046F2F70FF94FF0804180462846F1F7F3
:10EAB000FFFF01464046F2F7B9F9314605462046C8
:10EAC000F2F700F93146F1F7F5FF01462846F1F774
:10EAD000EFFF2146F1F7ECFF01464FF07E50F1F7D2
:10EAE000E7FF8344BBF5000FC0F2C78059463846A4
:10EAF000F2F7E8F8044642E54FF07E572BE7002294
:10EB0000059203E60027E2E54AF63C21C3F23831DC
:10EB10004046F1F7CFFF214682463046F1F7C8FF65
:10EB200001465046F2F78AFA70B14FF2CA21C7F295
:10EB300049113846F2F7C6F84FF2CA21C7F2491117
:10EB4000F2F7C0F804461AE54FEAE953A3F17E0054
:10EB50004FF4000646FA00F14B19C3F3C75223F0F5
:10EB60007F4E4FF6FF76A2F17F002EF4000CC0F22C
:10EB70007F064CF4000AC2F1960246FA00F64AFA01
:10EB800002F923EA0601002D2046B8BFC9F10009A9
:10EB9000F1F78EFF824651464046F1F78BFF4FEA70
:10EBA000C95B014613E70022C4F2163291450ADC24
:10EBB0007FF406AF2146F1F77BFF01464046F2F7AE
:10EBC00029FA0028C0D044F26021C0F6A25138468C
:10EBD000F2F778F844F26021C0F6A251F2F772F829
:10EBE0000446CCE44FF07E51F1F762FF4FF42A4126
:10EBF000C3F6B8710746F2F765F84AF270518146DC
:10EC0000C3F2EC613846F2F75DF839468246384681
:10EC1000F2F758F84FF07A5183463846F2F752F837
:10EC200001464AF6AB20C3F6AA60F1F741FF394628
:10EC3000F2F748F801464FF07C50F1F739FF0146F2
:10EC40005846F2F73FF84AF63B21C3F6B871F2F79F
:10EC500039F801465046F1F72BFF0746394648463A
:10EC6000F1F728FF20F47F6020F00F0A504662E69B
:10EC700001234FF40012059348E5494601F092FB49
:10EC8000014634E72DE9F04F40F6D87320F00044F8
:10EC9000C3F649739C4289B006460D4640F38B800B
:10ECA0004CF6E331C4F216018C4226DC4FF4786155
:10ECB0000028C3F6C97140F32B81F1F7F9FE4FF438
:10ECC0007D6224F00F04C3F6C9729442064600F038
:10ECD000818044F24341C3F23571F1F7E9FE014608
:10ECE00028603046F1F7E4FE44F24341C3F2357147
:10ECF000F1F7DEFE0127686061E04FF47867C4F247
:10ED00004937BC4240F38180B4F1FF4F5BDA4FEAF0
:10ED1000E459A9F18609A4EBC9542046F2F798F901
:10ED2000F1F77CFF0246014620460592F1F7C0FE4E
:10ED30004FF08741F1F7C6FF0746F2F789F9F1F77F
:10ED40006DFF0146044638460694F1F7B1FE4FF0D8
:10ED50008741F1F7B7FF00210790F2F747F9002844
:10ED600000F0F6800327204600210DF11808013F2E
:10ED7000F2F73CF940B158F8044D00212046013F1C
:10ED8000F2F734F90028F6D1924B0220009001935B
:10ED900005A83B4629464A4600F066FA002E07467B
:10EDA0000DDA95E80C0002F1004103F10042296000
:10EDB0006A60474203E00023286000274B60384622
:10EDC00009B0BDE8F08F0146F1F772FE00276860D8
:10EDD0002860F4E74FF48841C3F23571F1F768FE1B
:10EDE0004AF20831C2F685610446F1F761FE014638
:10EDF00028602046F1F75CFE4AF20831C2F68561D0
:10EE0000F1F756FE01276860D9E701F045FA4FF6A1
:10EE10008411C3F622718046F1F754FF4FF07C5104
:10EE2000F1F748FEF2F714F90746F1F7F7FE4FF451
:10EE30007861C3F6C9718346F1F744FF0146404645
:10EE4000F1F736FE44F243418146C3F2357158462C
:10EE5000F1F738FF1F2F8246514648461FDC5E4BB4
:10EE60007A1E53F8223024F0FF029A4217D0F1F7AD
:10EE70001FFE8046C5F8008041464846F1F718FE5F
:10EE80005146F1F715FE002E686098DA08F1004847
:10EE900000F10041C5F8008069607F428FE7F1F71B
:10EEA00007FEE3158046C0F3C750191A0829E1DDB3
:10EEB0004FF48841C3F2357158460393F1F702FFCE
:10EEC000824651464846F1F7F3FD0446214648463E
:10EED000F1F7EEFD5146F1F7EBFD4AF208318146BC
:10EEE000C2F685615846F1F7EDFE4946F1F7E0FDBF
:10EEF000824651462046F1F7DBFD039BC0F3C75223
:10EF00008046981A192841DCC5F80080A146B3E76D
:10EF1000F1F7D0FD4FF47D6724F00F04C3F6C977F5
:10EF2000BC42064616D044F24341C3F23571F1F7B4
:10EF3000C1FD014628603046F1F7BAFD44F2434175
:10EF4000C3F23571F1F7B6FD4FF0FF37686036E771
:10EF5000032719E74FF48841C3F23571F1F7AAFD91
:10EF60004AF20831C2F685610446F1F7A3FD014675
:10EF700028602046F1F79CFD4AF20831C2F685610F
:10EF8000F1F798FD4FF0FF37686018E74FF4234121
:10EF9000C2F685615846F1F795FE80464146204607
:10EFA000F1F786FD814649462046F1F781FD41464D
:10EFB000F1F77EFD43F232110446C2F28D4158460C
:10EFC000F1F780FE2146F1F773FD8246514648462F
:10EFD0004DE700BF2C470108AC46010820F0004275
:10EFE000B2F1FF4FF8B50446034646D2002A42D09C
:10EFF000002852DBC415B2F5000F09D210F4000549
:10F0000053D15B0001351902FBD5C5F1010024186D
:10F0100023F07F417F3C21F40006E20746F4000024
:10F0200048BF400043004FF08072002760109A42B2
:10F030003C462CDD5B004FF400021825A618510851
:10F040009E4205F1FF3502DCB4189B1BBF185B0024
:10F0500062189A4202DC9B1A54187F185B004A0817
:10F06000013DEBD113B107F001017F187C1004F1D1
:10F070007C5303EBC0542046F8BD0146F1F722FE55
:10F0800001462046F1F716FD04462046F8BD4FF034
:10F09000007403F17F431746CCE70146F1F708FD02
:10F0A0000146F1F7C3FE0446E5E70120AFE700BFE4
:10F0B0002DE9F84320F00046B6F1485F05460F46BB
:10F0C0005BDAF1F7C5FF002800F0CA802946284620
:10F0D000F1F7F8FD4DF24E71CAF647510446F1F7CB
:10F0E000F1FD47F2F641C3F20F11F1F7E3FC2146BF
:10F0F000F1F7E8FD4FF27C21C3F29341F1F7D8FC20
:10F100002146F1F7DFFD40F60151C3F2D071F1F76E
:10F11000D1FC2146F1F7D6FD40F66131C3F6B621A8
:10F12000F1F7C6FC2146F1F7CDFD4AF6AB21C3F657
:10F130002A51F1F7BFFC2146F1F7C4FD8046204675
:10F140004FF07C51F1F7BEFD414606462046F1F7EF
:10F15000B9FD394604462846F1F7B4FD014620467C
:10F16000F1F7A6FC01463046F1F7A2FC01464FF04C
:10F170007E50F1F79DFCBDE8F8830146F1F7A2FD52
:10F180004DF24E71CAF647510446F1F79BFD47F226
:10F19000F641C3F20F11F1F78DFC2146F1F792FD14
:10F1A0004FF27C21C3F29341F1F782FC2146F1F743
:10F1B00089FD40F60151C3F2D071F1F77BFC214685
:10F1C000F1F780FD40F66131C3F6B621F1F770FC2E
:10F1D0002146F1F777FD4AF6AB21C3F62A51F1F744
:10F1E00069FC2146F1F76EFD49F69913C3F6996360
:10F1F0009E428046A3DD0020C3F64870864227DC8D
:10F2000006F17F464FF07E503146F1F751FC8146C2
:10F2100020464FF07C51F1F755FD3146F1F748FC9F
:10F22000414606462046F1F74DFD3946044628463C
:10F23000F1F748FD01462046F1F73AFC0146304619
:10F24000F1F736FC01464846F1F732FCBDE8F88399
:10F250004FF000090026C3F63879C3F69066D7E769
:10F260004FF07E50BDE8F8832DE9F04FDFB00C93EE
:10F270000C9D224B689C0A91691ED61E48BF161D24
:10F28000834653F82400F71027EAE77308900491A7
:10F2900004980D93089DDC43DDF834C002EBC402F2
:10F2A00041190792C0EB0C0750D47E18699BC7EB3D
:10F2B00006090136002F03EB870522AC09F0010A8D
:10F2C000C0F2FE822868F1F7A9FC0137B74220603E
:10F2D0004FF004083AD0BAF1000F26D0002FC0F248
:10F2E000F18255F80800F1F799FC0137B74244F86C
:10F2F000080008F1040818D128E000BF444A0108BA
:10F3000055F80800F1F78AFC013708F1040944F8C0
:10F31000080013D455F80900F1F780FC0137B74213
:10F3200044F8090009F1040810D0002FE8DA0020A1
:10F33000013708F1040944F80800EBD50137002033
:10F34000B74244F8090009F10408EED1089A002AEE
:10F35000C0F2458508990C9E8D004AAB5C19039557
:10F3600049AF02944FEA860A049A002AC0F29682B4
:10F370000DF1880808EB860555F8041CAAF1040372
:10F38000DBF80000C3F38009F1F79CFC0146002084
:10F39000F1F790FB0424043D544580462BD0B9F18D
:10F3A000000F0DD055F8041DDBF80400F1F78AFCBE
:10F3B00001464046F1F77EFB0824544580461AD0AA
:10F3C00055F8041C5BF80400F1F77CFC014640464C
:10F3D000F1F770FB0434804655F8081C5BF8040014
:10F3E000F1F770FC01464046F1F764FB0434083D38
:10F3F00054458046E4D1029847F8048F013687428D
:10F40000B2D1039F0EA9CE190996089EB2005EAB39
:10F410009D18002E029255F8509C7DDD0DF5947CD0
:10F420004FF06E5148460DACA7180CEB0205F1F7F2
:10F4300049FCF1F70DFEF1F7F1FB4FF08741019028
:10F44000F1F740FC01464846F1F732FBF1F700FEC8
:10F450000EAC20600198014655F8040DF1F72AFB27
:10F46000BC428146C7F3800156D0E9B14FF06E51DE
:10F47000F1F728FCF1F7ECFDF1F7D0FB4FF08741F5
:10F480000190F1F71FFC01464846F1F711FBF1F737
:10F49000DFFD019A0FAC2060114655F8040DF1F71D
:10F4A00009FBBC42814637D04FF06E514846F1F718
:10F4B00009FCF1F7CDFDF1F7B1FB4FF08741804634
:10F4C000F1F700FC01464846F1F7F2FAF1F7C0FD0A
:10F4D0004146606055F8040DF1F7ECFA4FF06E51BB
:10F4E0008146F1F7EFFBF1F7B3FDF1F797FB4FF032
:10F4F00087418046F1F7E6FB01464846F1F7D8FA26
:10F50000F1F7A6FD4146A06055F8040DF1F7D2FAD7
:10F510000834BC428146C7D10799484600F042FFF3
:10F520004FF078510546F1F7CDFB00F0C1FE4FF0EA
:10F530008241F1F7C7FB01462846F1F7B9FA0746C1
:10F54000F1F786FD8146F1F769FB01463846F1F790
:10F55000AFFA07990746002940F33981721E0EACB5
:10F56000079D54F82230C5F1080043FA00F101FA72
:10F5700000F0C5F107041B1A43FA04F40DF1380C2E
:10F5800089444CF82230002C55DD002E09F1010988
:10F5900040F39481029D0EABDDF808C053F8042BB4
:10F5A000281F0DF1380E00250EEB0C01C0F3800072
:10F5B00022B1C2F5807243F8042C01258B4226D07B
:10F5C00060B10F9A0433002D40F0F38022B1C2F5F0
:10F5D000807543F8045C01258B4218D053F8042B46
:10F5E000002D40F0EC80C2F5807012B143F8040C9D
:10F5F000012553F8042B002D40F0DB80C2F580700C
:10F60000002AE9D001258B4243F8040CE6D1079982
:10F6100000290DDD012900F0E280022908D1701EC9
:10F620000DF1380E5EF8202002F03F034EF8203036
:10F63000022C00F0E08038460021F1F7D7FC0028CA
:10F6400000F0F3800898751EA84225DC029B0DF19E
:10F65000380E0EEB03010B46DDF824C053F8042DE1
:10F66000CCEB0100011F6345C1F3800011D030B124
:10F6700053F8041DDDF824E00A43734509D0099FBF
:10F6800053F8040D53F8041D0243BB4242EA010241
:10F69000F6D1002A40F01A81089F0EAD781E55F869
:10F6A0002020002A40F0108105EB8004012354F84B
:10F6B000041D01330029FAD0F018771C87420B9003
:10F6C00075DCDDF810E00D9D0B9B0C9C0EEB07022A
:10F6D000DDF808C0699F991B06EB05094AA8A61921
:10F6E00022AB07EB890900EB0C05571C8A0003EBE2
:10F6F0008601029506920591002659F8040FF1F74C
:10F700008DFA059CA051049800285EDB22AD05EB24
:10F710008702AAF10403C3F3800452F8041CDBF847
:10F7200000000394141FF1F7CDFA01460020F1F711
:10F73000C1F94FF00408D04505462DD0039971B1A9
:10F7400054F8041DDBF80400F1F7BCFA0146284622
:10F75000F1F7B0F94FF00808D04505461CD054F831
:10F76000041C5BF80800F1F7ADFA01462846F1F7F2
:10F77000A1F908F10408054654F8081C5BF80800D4
:10F78000F1F7A0FA01462846F1F794F908F10408C8
:10F79000083CD0450546E2D1DDF808E0069804367D
:10F7A0004EF8045F01378642CDF808E0A5D10B9EE4
:10F7B0002CE6C2F1FF0243F8042C01250CE7C2F14C
:10F7C000FF0543F8045C012513E70025E4E75ED15B
:10F7D000701E0DF1380E5EF820301C12D3E6711E3B
:10F7E0000DF1380C5CF82100022C00F07F024CF87F
:10F7F00021207FF420AF39464FF07E50F1F758F9C1
:10F800000746002D3FF417AF07994FF07E5000F0E8
:10F81000C9FD01463846F1F74BF907463846002145
:10F82000F1F7E4FB00287FF40DAF0294079C384603
:10F830006142CDF8109000F0B5FD4FF087410546CC
:10F84000F1F7F2FB002800F0D2824FF06E5128460B
:10F85000F1F738FAF1F7FCFBF1F7E0F94FF08741E7
:10F860000746F1F72FFA01462846F1F721F9F1F79B
:10F87000EFFB0EA941F826003846F1F7E9FB079A9D
:10F88000013608320EAC079244F8260034E04FF0FF
:10F890007C51F1F7C9FB58B90024CCE64FF00008C1
:10F8A000029847F8048F013687427FF45DADA8E5E2
:10F8B0000224002E09F101093FF76CAE0025A6E6EF
:10F8C000002002E5002010E50123F5E6079A0EAEC0
:10F8D00056F82530083ACDF8109002940792002B84
:10F8E00040F08E8206EB85042E4654F8045D013EFE
:10F8F000083A002DF9D007924FF07E50079900F09A
:10F9000051FD002E0446C0F2AC804FEA860AC6EBD9
:10F91000867B0EAF4FEA8B095744C9F100034AA911
:10F92000386801EB0A08C3F3800BF1F777F9214639
:10F93000F1F7C8F94FF06E51C8F800002046F1F712
:10F94000C1F9A9F104096FF0030ACA45054631D08F
:10F95000BBF1000F0BD057F8040CF1F75FF9294603
:10F96000F1F7B0F96FF0070A48F8040C1AE057F8FD
:10F970000A00F1F753F92946F1F7A4F94FF06E5157
:10F9800048F80A002846F1F79DF9AAF10404054653
:10F990003859F1F743F92946F1F794F9AAF1080A21
:10F9A00048F8040028464FF06E51F1F78BF9CA452C
:10F9B0000546DCD1701CDFF84C94DDF820A00390E4
:10F9C00000270596BAF1000FC0F20582002FC0F2A1
:10F9D0000282002600241AF0010F354620D0D8F804
:10F9E0000010D9F80000F1F76DF901462046F1F753
:10F9F00061F80125AA45044626DB0426BD420FDD39
:10FA000022E0BB4520DC58F8021059F80200F1F75B
:10FA100059F901462046F1F74DF8BD42044613DC82
:10FA200058F8061059F80600F1F74CF9014620463F
:10FA3000F1F740F805F1010B06F104020235DA4551
:10FA4000044602F10406DCDA5EABDDF80CC003EB21
:10FA500087010137674541F8A04CA8F10408B1D1EE
:10FA6000059E689C032C16D8DFE814F085011F0161
:10FA70001F011B0000230299002900F00B81379C15
:10FA8000369804F100420A9C00F1004503F100435E
:10FA900025606260A360049D05F007005FB0BDE8CB
:10FAA000F08F002EE6DD06F1FF3836AF07EB880950
:10FAB0004D4655F804290DF1D40AD5F808B0104682
:10FAC00059460192F0F7F6FF804641460198F0F75B
:10FAD000EFFF01465846F0F7EDFF5545C9F38003A7
:10FAE000A860C5F8048044D0BBB155F80429D5F806
:10FAF00008B0104659460192F0F7DCFF01998046A4
:10FB000008464146F0F7D4FF01465846F0F7D2FFC9
:10FB10005545C5F80480A8602BD02C4654F804390C
:10FB2000D4F808B0184659460193F0F7C3FF804651
:10FB300041460198F0F7BCFF01465846F0F7BAFF7E
:10FB4000C4F80480A06055F804BC251FD5F80880CF
:10FB500058464146F0F7AEFF044621465846F0F7B6
:10FB6000A7FF01464046F0F7A5FF55456C60A86029
:10FB7000D3D1012E7FF77EAF4D4655F804B9C7EBC0
:10FB8000090ED5F808A058465146AEF10409F0F721
:10FB900091FF804641465846F0F78AFF014650469D
:10FBA000F0F788FFBD42C9F38009C5F80480A8605A
:10FBB00043D0B9F1000F15D055F804A9D5F8089035
:10FBC00050464946F0F776FF804641465046F0F7EA
:10FBD0006FFF01464846F0F76DFFBD42C5F804804F
:10FBE000A8602AD02C4654F804A9D4F808905046AE
:10FBF0004946F0F75FFF804641465046F0F758FF10
:10FC000001464846F0F756FFC4F80480A06055F856
:10FC1000049C251FD5F8088048464146F0F74AFF66
:10FC2000044621464846F0F743FF01464046F0F7B8
:10FC300041FFBD426C60A860D4D1013607EB860756
:10FC400008353E467A1B131F56F8041D0020C3F3E7
:10FC50008007F0F72FFFAE4203463FF40CAF3FB1F1
:10FC600056F8041DF0F726FFAE4203463FF403AFFB
:10FC7000184656F8041C341FF0F71CFF083E54F8D1
:10FC8000041CF0F717FFAE42F3D102990346002996
:10FC90007FF4F5AEDDF828C036993798CCF800101F
:10FCA000CCF80400CCF80830F5E60023002E29DB60
:10FCB00036AF751C07EB85042546E21B55F8041D7D
:10FCC000A2F1040E0020CEF38008F0F7F3FEBD424F
:10FCD000034617D0B8F1000F06D055F8041DF0F711
:10FCE000E9FEBD4203460DD0184655F8041C2C1FF2
:10FCF000F0F7E0FE083D54F8041CF0F7DBFEBD42CF
:10FD0000F3D103460299002967D003F10040DDF8E2
:10FD100028C01946CCF800003698F0F7C9FE002E2E
:10FD2000034621DD36AF07EB8606F51B2A1F379900
:10FD3000C2F38007F0F7BEFE37ACB442034613D0DF
:10FD400037B16168F0F7B6FE38ACB44203460BD069
:10FD5000184654F8041FF0F7ADFE54F8041FF0F7EE
:10FD6000A9FEB442F5D10346029909B103F100435B
:10FD70000A9C63608FE6002E40DB36AF013607EB4E
:10FD800086000546C21B55F8041D0020141FF0F71D
:10FD900091FEBD42C4F38006034615D036B155F836
:10FDA000041DF0F787FEBD4203460DD0184655F8F6
:10FDB000041C2C1FF0F77EFE083D54F8041CF0F7DD
:10FDC00079FEBD42F3D10346029909B103F1004324
:10FDD0000A9C23605FE6002436E6184697E7DDF8C4
:10FDE00030E0900003904FEA8E0AFFF70ABB2846E6
:10FDF000F1F72EF90EAB43F826007DE50023E3E78B
:10FE00002E4679E5504A01082DE9F84320F00043D9
:10FE1000B3F1485F04460F46904603DAF1F718F94C
:10FE2000002859D021462046F0F74CFF21460546D0
:10FE3000F0F748FF4CF6D311C2F62E71064628465D
:10FE4000F0F740FF42F63471C3F2D721F0F730FEED
:10FE50002946F0F737FF4EF61B71C3F23861F0F711
:10FE600029FE2946F0F72EFF40F60151C3F6501146
:10FE7000F0F71EFE2946F0F725FF48F68901C3F684
:10FE80000841F0F717FE8146B8F1000F27D04FF078
:10FE90007C513846F0F716FF494680463046F0F769
:10FEA00011FF01464046F0F703FE2946F0F70AFF2E
:10FEB0003946F0F7FDFD4AF6AB210546C3F62A6147
:10FEC0003046F0F7FFFE01462846F0F7F3FD014605
:10FED0002046F0F7EDFD04462046BDE8F8830146D4
:10FEE0002846F0F7EFFE4AF6AB21C3F62A61F0F799
:10FEF000DFFD3146F0F7E6FE01462046F0F7DAFD79
:10FF000004462046BDE8F883002070470021002009
:10FF1000C7F6F871704700BF2DE9F041C1F30A58E8
:10FF2000A8F2FF37132F82B002460B4604460D4657
:10FF30008C464FEAD17635DC002F51DB4FF6FF714E
:10FF4000C0F20F0141FA07F101EA0300104324D087
:10FF50004A0813401C430BD04FF4802141FA07F1AB
:10FF600025EA0205132F0CBF4FF0004400240D4377
:10FF70002246324C2B4604EBC606D6E90045204605
:10FF80002946F0F7F5F8CDE90001DDE90001224648
:10FF90002B46F0F7EBF802460B461046194602B026
:10FFA000BDE8F081332F07DDB7F5806FF5D1F0F7AD
:10FFB000DFF802460B46F0E7A8F213484FF0FF3196
:10FFC00021FA08F01042E8D042082242D0D04FF087
:10FFD000804343FA08F824EA020444EA0804C7E725
:10FFE00021F0004050EA0201D7D023F07F4525F4EC
:10FFF000700343EA0204614241EA04000F4C050B1E
:020000040801F1
:100000004FEA5C4E05F4002304EBC601D1E900453C
:1000100043EA4E4320462946F0F7AAF8CDE900010D
:10002000DDE9000122462B46F0F7A0F8044602461F
:1000300021F000400D4640EAC673AEE7804A010851
:100040002DE9F04120F00045B5F1A14F04460646E8
:100050000DDBB5F1FF4F00F39C80002840F6DB7408
:1000600040F3D480C3F6C9742046BDE8F0814FF652
:10007000FF73C3F6DF639D4200F3A280B5F1445FD6
:10008000C0F28E804FF0FF3721462046F0F71AFE6F
:1000900001468046F0F716FE46F6D711C3F68541B5
:1000A0000546F0F70FFE4DF65921C3F64B51F0F718
:1000B00001FD2946F0F706FE46F63531C3F68851B4
:1000C000F0F7F8FC2946F0F7FDFD42F66E61C3F645
:1000D000BA51F0F7EFFC2946F0F7F4FD44F625118C
:1000E000C3F61261F0F7E6FC2946F0F7EBFD4AF69D
:1000F000AB21C3F6AA61F0F7DDFC4146F0F7E2FD63
:100100004AF221218046CBF615512846F0F7DAFD58
:100110004FF26B11C3F66E51F0F7CAFC2946F0F7A7
:10012000D1FD48F29571C3F69D51F0F7C1FC294607
:10013000F0F7C8FD48F63861C3F6E351F0F7B8FCB4
:100140002946F0F7BFFD4CF6CD41C3F64C61F0F700
:10015000AFFC2946F0F7B6FD7B1C0146404658D05F
:10016000F0F7A8FC2146F0F7ADFD494B53F82710F6
:10017000F0F79EFC2146F0F79BFC0146454850F8FD
:100180002700F0F795FC002E3DDB04462046BDE835
:10019000F0810146F0F78EFC04462046BDE8F08170
:1001A0004FF2CA21C7F24911F0F784FC4FF07E519B
:1001B000F0F744FF00283FF465AF2046BDE8F0812A
:1001C00000F06AF84FF6FF71C3F697718D4204464E
:1001D0004FF6FF7228DCC3F62F72954246DC0146CB
:1001E000F0F768FC4FF07E51F0F762FC4FF0804171
:1001F00005462046F0F75EFC01462846F0F716FE5D
:100200000027044640E700F100442DE7CBF6C9740F
:100210002AE7F0F74FFC2146F0F754FD014620464F
:10022000F0F746FC04461FE7C4F21B02954214DCBB
:100230004FF07F51F0F73CFC4FF07F5105462046D0
:10024000F0F740FD4FF07E51F0F734FC01462846B0
:10025000F0F7ECFD0227044616E700202146CBF616
:100260008070F0F7E3FD032704460DE74FF07E5161
:10027000F0F71EFC4FF07E5107462046F0F71AFCBF
:1002800001463846F0F7D2FD01270446FCE600BFE0
:10029000904A0108A04A010820F00040704700BFC2
:1002A00020F00040B0F1FF4FACBF002001207047AC
:1002B000F8B520F00046F50D7F3D162D01460446A9
:1002C0001BDC002D074620DB4FF6FF73C0F27F03D7
:1002D00043FA05F606420ED04FF2CA21C7F2491181
:1002E000F0F7E8FB0021F0F7A9FE18B1002C1BDBAA
:1002F00027EA060421460846F8BDB6F1FF4FFAD3B7
:10030000F0F7D8FB01460846F8BD4FF2CA21C7F204
:100310004911F0F7CFFB0021F0F790FE0028E9D05B
:10032000002C07DB0024E5E74FF4000040FA05F558
:100330006719DDE70021CBF68071002E18BF0C464F
:10034000D8E700BF08B902207047B0F1004FFAD0DB
:10035000A0F500026FF001439A4201D804207047D3
:1003600000F1FF419942F9D94FF6FE73421EC0F2E7
:100370007F039A4201D80320704700F100414A1ED2
:100380009A42F8D9B0F1FF4F05D010F5000F14BF15
:100390000020012070470120704700BF0020C7F6F1
:1003A000C070704738B530F00044034602460D4631
:1003B0000FD0B4F1FF4F0ED2B4F5000F11D3E40DFE
:1003C0006419FE2C33DC002C1BDD22F0FF4141EAD6
:1003D000C453184638BD0146F0F76CFB0346184677
:1003E00038BD4FF09841F0F76DFC43F6B041CFF6C1
:1003F000FF718D42034612DBC0F3C7540246193C1D
:10040000DEE714F1160F21DA4CF25032954219460C
:100410000EDC44F26020C0F6A25000F023F844F253
:100420006021C0F6A251F0F74DFC0346D1E7194612
:100430004FF2CA20C7F2491000F014F84FF2CA2157
:10044000C7F24911F0F73EFC0346C2E722F0FF4332
:1004500004F1190043EAC0504FF04C51F0F732FC60
:100460000346B6E701F0004120F000400843704722
:100470002DE9F041274C84B025680746D5F848415E
:10048000002C41D066681F2E1CDD234810B94FF0A8
:10049000FF301FE04FF4C870039102920193AFF355
:1004A000008003990446029A019B0028EFD0D5F8FA
:1004B0004861002060602660C5F84841C4F88801A2
:1004C000C4F88C01656847B9A81C013544F82010B0
:1004D0006560002004B0BDE8F081012000FA05F05D
:1004E000D4F8886104EB85080643022FC8F88820F9
:1004F000C4F88861C8F80831E6D1D4F88C3143EAF1
:100500000002C4F88C21DFE705F5A674C5F8484160
:10051000B8E700BFB84B01080000000000210A2224
:1005200001F0C4BD2DE9F84FDDF828B081468A46B8
:1005300098469AB193B11646002503E00FD0651C8A
:10054000AE420BD97419640808FB04A74846394623
:10055000D8470028F2DA2646AE42F3D800273846BC
:10056000BDE8F88F40F2D053C2F20003186870471C
:10057000114B124A70B5981A831018D0591E02EB0D
:1005800083040D4654F8042D01F00106904775B11F
:1005900026B154F8040D8047013D08D054F8043DBD
:1005A0009847013D54F8041D8847013DF6D1BDE848
:1005B000704004F009BB00BFE04B0108DC4B0108B0
:1005C000F8B5204F204C381B871017D07A1E2368AF
:1005D000012502F001069847AF420FD02EB154F822
:1005E000041F02258847AF4208D060688047023563
:1005F000A268261D90470834AF42F6D1134F144C21
:1006000004F0DCFA3B1B9F1018D07D1E216805F01A
:10061000010601258847AF4211D02EB154F8040FCE
:1006200002258047AF420BD0626890470235A3682D
:10063000261D98470834AF42F6D1F8BDF8BDF8BD85
:10064000F8BD00BFD44B0108D44B0108DC4B0108B6
:10065000D44B01080F2A2DE9F00340F2A18041EAB2
:1006600000039B0740F09E800C68A2F11005046017
:100670004B68AC4643608C68BCF10F0F8460CC685B
:10068000C5F30015C46000F1100301F110042BD96B
:1006900075B12568ACF1100C1D6065685D60A568DA
:1006A0009D60E5681034DD601033BCF10F0F1BD97D
:1006B000276804F110061F60676803F110055F608A
:1006C000A768ACF1200C9F60E768DF6024691C61BB
:1006D000776806F110046F60B7682033AF60F66882
:1006E000BCF10F0FEE60E3D8A2F1100828F00F0361
:1006F00002F00F0403F1100C032C00EB0C0301EBD0
:100700000C0851D9211F4FEA9109444608EB890C86
:1007100054F8046BC8EB0C010CF1040C1D46644545
:1007200045F8046BC1F3800112D029B154F8041BC1
:10073000644545F8041B0BD0274657F8041B2E468A
:1007400046F8041B64686C603C1D351D6445F3D19C
:1007500009F1010C4FEA8C0902F0030208EB0901D0
:100760004B44D2B10D789A18DC4303F8015B14199D
:10077000934204F0010410D02CB111F8014F03F89A
:10078000014B934209D04D781C4604F8015B8D78EB
:1007900002315D70631C9342F5D1BDE8F0037047F0
:1007A0000346DEE70346DDE741462246D9E700BFC0
:1007B000F0B48407034600F08D80541E002A00F038
:1007C0008780E507CEB211D41A4602F8016B1346B2
:1007D0001546920710D0621E002C79D003F8016BE9
:1007E00014469A071D4607D0013CEDE7034603F87F
:1007F000016B9A071D46F7D1032C52D9CEB246EAB7
:1008000006270F2C47EA07432DD9A4F110021746FB
:100810000F2FC2F300162B606B60AB60EB6005F12D
:10082000100216D93EB1103F136053609360D3603D
:1008300010320F2F0DD9203F02F1100613605360C4
:100840009360D360136153619361D36120320F2FA2
:10085000F1D8A4F1100222F00F0204F00F041032BC
:10086000032C15441DD9271F3E462A46032E42F865
:10087000043BC7F380070DD927B1043E032E42F88D
:10088000043B07D9174647F8043B083E53603A1D1E
:10089000032EF7D8231F23F00302131D04F00304D3
:1008A000ED18ACB1C9B2EA432C1905F8011BA31825
:1008B000A54203F001020BD01AB105F8011BA542B5
:1008C00006D02B4603F8011B69705D1CA542F8D1C8
:1008D000F0BC7047054614468EE700BF2DE9F04F87
:1008E00089B014468046019202EB4202A5085000EE
:1008F00004F0030418F0030F02919946039506943F
:10090000079040F0D6800699002940F05A82019A5B
:10091000151F18BF01250095029D062D40F2CF80BE
:10092000DDF808C0019F64464FEA5C06072C07FB10
:10093000068A40F0E281DDF81CC008EB0C06009B43
:10094000002B40F0FB81D8F80010DAF80030C8F82E
:100950000030CAF800100198DDF804A008EB00058B
:100960004946002205952F4604953446CAF1000AEF
:1009700091460D46A74240F213812B464D469946BB
:10098000002D00F0C183DDF810B00299CBEB070A0F
:10099000C8EB0B025245A8BF5246DDF804C0002A3E
:1009A0000CFB018B3ADD009BB91A022B404640F04C
:1009B000D28210F8015B91F800C0029500F801CCDA
:1009C000DDF808C00B468A18CD4303F801CBAD18FB
:1009D0000130934205F0010520D04DB110F8015CC3
:1009E000497800F8011C03F8015B0130934215D0EF
:1009F000014611F8015C93F800C0184601F801CCDB
:100A000000F8015B11F8015B93F801C0034601F89F
:100A100001CC03F8015B01319342EAD10199C6EBA5
:100A20000B03341B581AA04228BF204600282FDD94
:100A3000009DC0EB0B02022D40F053821578FB4362
:100A40003978381807F8015B874203EB0005134635
:100A500003F8011B05F001011AD039B155783A7835
:100A600007F8015B874203F8012B11D03D781E780F
:100A70001A46394601F8016B02F8015B5B787D7814
:100A80000F4607F8013B8742134603F8015BEDD19F
:100A9000019D5545C0F08C81DDF804C0A4457CD291
:100AA000C4EB0B0818F0030FB4FBFCF402943FF402
:100AB0002AAF029D0223062D00933FF631AFDDF8E9
:100AC00004C00CFB058A08EB0C01514565D2019C62
:100AD000DDF804B065420434009E02940091CDF824
:100AE00010A04F46DDF80090C14509D84DE0D9F877
:100AF00000002168C9F8001020604445A14644D98F
:100B000009EB050420464946B84700283DDD002E84
:100B1000EDD0012E00F0A7831BF804E094F80090BC
:100B20000BF1FF310BEB04000246234601F0010CF0
:100B3000002902F8019B03F801EBDEDDBCF1000F98
:100B400009D0407894F801E00139002902F801EB5E
:100B500003F8010BD1DD93F800A092F800909446C1
:100B600018460CF801AB00F8019B92F801E093F8ED
:100B700001A0023962460346002902F801AB03F8DE
:100B800001EBE8DC4445A146BAD8DDF800C0049B7F
:100B9000DC449C45CDF800C0A4D309B0BDE8F08F7B
:100BA00038464146A84700280BDC8CE020683268B4
:100BB0002260306056444FF001095444A7423FF68A
:100BC000DCAE20464146A8470028C0F29A83F4D103
:100BD000009B002BEAD00099012935D0DDF804E014
:100BE000207896F800C00EF1FF312246334601F01E
:100BF0000109002902F801CB03F8010BDADDB9F194
:100C0000000F09D0107893F800C00139002902F8CC
:100C100001CB03F8010BCDDD93F800B092F800E0B2
:100C2000944618460CF801BB00F801EB92F80190CD
:100C300093F801B0023962460346002902F801BB6D
:100C400003F8019BE8DCB5E721463346DDF80CE00C
:100C500053F8042B51F8040B0EF1FF3C41F8042C1F
:100C60000CF0010243F8040C04310433BCF1000F12
:100C7000A0DD72B151F8040C53F8042C0CF1FF3CC8
:100C800041F8042C43F8040C04310433BCF1000F88
:100C900090DD53F8042C51F8049C084641F8042CCC
:100CA0001A4643F8049C50F8043B52F8041BACF17C
:100CB000020C40F8041C011D42F8043C131DBCF159
:100CC000000FE6DC76E714D1009A002A7CD1049864
:100CD0003B680268DDF810C0CCF800303A60DDF8FF
:100CE00010E0DDF804900EEB090CCDF810C04FF0C9
:100CF0000109DDF804E077443CE602980199431EBF
:100D0000282801FB038600F2AB8034464546514655
:100D10002846C847002821465046C0F29580C8475B
:100D200000283FF70CAE28462146C847009B34EA0E
:100D3000200A28BFAA46002B3FF405AE0099424680
:100D4000012900F04781DDF804C012F8015B9AF830
:100D500000400CF1FF3102F8014C574601F0010050
:100D60000132002907F8015B7FF7F5AD58B13D78F6
:100D700012F8013C013902F8015C0132002907F840
:100D8000013B7FF7E8AD12F8014C3B78384602F89A
:100D9000013C00F8014B12F8014B7D78023902F852
:100DA000015C07460132002907F8014BEBDCD2E574
:100DB000019D4046BAFBF5F12A464B46FFF78EFDF2
:100DC0006AE602240094A7E50098012800F03B8120
:100DD000DDF810E0DDF804B039789EF800000BF182
:100DE000FF3B724602F8011B3B460BF00101BBF1D1
:100DF000000F03F8010B7FF772AF59B11178187823
:100E00000BF1FF3BBBF1000F02F8010B03F8011BD4
:100E10007FF765AF92F800C093F80090104619462E
:100E200000F8019B01F801CB92F801E093F801C0B2
:100E3000ABF1020B02460B46BBF1000F02F801CBEF
:100E400003F801EBE6DC4AE7C8470028FFF677AD78
:100E500028462146C84735EA200A28BFA2466EE543
:100E6000019AC40802FB04F408EB04054FEA440BA2
:100E700029464046CDF810B0C84708EB0B070028BC
:100E800039462846C0F23481C847002840F33182F1
:100E9000C4F1000B0AEB0B0751463846C8475444CF
:100EA000002821465046C0F21781C847002840F369
:100EB0001882049806EB0B04371A21463846C847B7
:100EC000002831462046C0F2FB80C84700283FF783
:100ED0001EAF38463146C84736EA200428BF3C4694
:100EE00015E73946134653F8042B51F8045B800884
:100EF000013841F8042C00F0010243F8045C04318D
:100F0000043300287FF7C4AD6AB151F8045C53F88C
:100F1000042C013841F8042C43F8045C04310433F8
:100F200000287FF7B5AD51F8046C53F8042C0D463A
:100F300041F8042C43F8046C1A4652F8041B55F887
:100F4000046B023845F8041C131D291D002842F8C3
:100F5000046CE8DC9CE50B4653F8045B50F8041B7A
:100F6000920802F1FF3C40F8045C021D0CF0010500
:100F700043F8041C0433BCF1000F7FF74FAD7DB183
:100F800052F8041C53F8040C0CF1FF3C42F8040C1A
:100F900043F8041C04320433BCF1000F7FF73EAD6C
:100FA00052F8045C53F8040C114642F8040C43F860
:100FB000045C184650F8042B51F8045BACF1020CA9
:100FC00041F8042C031D0A1DBCF1000F40F8045C1D
:100FD000E6DC23E55746039952F8043B57F8040B27
:100FE000013942F8040C01F0010447F8043C0432D2
:100FF0003B1D00297FF7AFAC6CB152F8045C53F88D
:10100000047C013942F8047C43F8045C0432043364
:1010100000297FF7A0AC52F8045C53F8040C144686
:1010200042F8040C1F4643F8045C57F8042B54F8AC
:10103000045B023944F8042C3B1D221D002947F8AB
:10104000045CE8DC87E404993B46DDF80C9053F837
:10105000042B51F804EB09F1FF3041F8042C00F0A7
:10106000010243F804EC0431043300287FF737AE63
:101070006AB151F804CC53F8042C013841F8042C1F
:1010800043F804CC0431043300287FF728AE53F82A
:10109000042C51F804EC894641F8042C1A4643F814
:1010A00004EC59F8043B52F8041B023849F8041CBC
:1010B00042F8043C131D002809F10401E7DC0EE6A8
:1010C000C8470028FFF623AE38463146C84737EAFE
:1010D000200428BF34461AE6C8470028FFF6E9AEC8
:1010E00038462146C84737EA200A28BFA246E0E62C
:1010F000C8470028FFF6CCAE40463946C84738EA14
:10110000200528BF3D46C3E60298019C059D04FBCF
:10111000008A5545BFF441AD019FDDF814B03C1D78
:10112000009ECDF800B0DDF804B07D420494CDF807
:1011300008A01F46DDF80090C84509D34CE0D9F857
:1011400000002168C9F8001020604445A14643D939
:1011500009EB050420464946B84700283CDD002E2F
:10116000EDD0012E41D01BF804E094F800900BF173
:10117000FF310BEB04000246234601F0010C00296D
:1011800002F8019B03F801EBDFDDBCF1000F09D091
:10119000407894F801E00139002902F801EB03F8E6
:1011A000010BD2DD93F800A092F800909446184607
:1011B0000CF801AB00F8019B92F801E093F801A054
:1011C000023962460346002902F801AB03F801EB3D
:1011D000E8DC4445A146BBD8DDF800C0029BDC44F6
:1011E0009C45CDF800C0A5D3D7E4DDF81090234688
:1011F00009EB0402DDF80CE053F8041B52F804CCB0
:101200000EF1FF3042F8041C00F0010143F804CC59
:1012100004320433002898DD61B152F8049C53F87D
:10122000041C013842F8041C43F8049C04320433C3
:1012300000288ADD53F8041C52F804EC944642F866
:10124000041C194643F804EC5CF8043B51F8042BE9
:1012500002384CF8042C41F8043C0B1D00280CF11A
:101260000402E7DC71E7029A23461219DDF80C90BC
:1012700053F8041B52F804CC09F1FF3042F8041C67
:1012800000F0010143F804CC0432043300287FF756
:1012900034AC69B152F804EC53F8041C013842F83C
:1012A000041C43F804EC0432043300287FF725AC17
:1012B00053F8041C52F8049C944642F8041C194646
:1012C00043F8049C5CF8043B51F8042B02384CF8BA
:1012D000042C41F8043C0B1D00280CF10402E7DC4F
:1012E0000BE438462146C84734EA200A28BFBA46EC
:1012F000DFE540463946C84737EA200528BF45465E
:10130000C6E5A7423FF639AB009B63B9386822684F
:101310003A602060DDF804E04FF001097744CEEB3D
:101320000404FFF727BB0098012833D0DDF80490B0
:10133000207897F800E009F1FF313A4602F8010BF6
:10134000234601F00100002903F801EBE2DD48B17A
:10135000107893F800C00139002902F801CB03F896
:10136000010BD7DD93F800B092F800E094461846E0
:101370000CF801BB00F801EB92F8019093F801B072
:10138000023962460346002902F801BB03F8019BBB
:10139000E8DCBFE739462346DDF80CE053F8042BC0
:1013A00051F8040B0EF1FF3C41F8042C0CF0010243
:1013B00043F8040C04310433BCF1000FAADD72B110
:1013C00051F8040C53F8042C0CF1FF3C41F8042CA8
:1013D00043F8040C04310433BCF1000F9ADD53F8D8
:1013E000042C51F8049C084641F8042C1A4643F892
:1013F000049C50F8043B52F8041BACF1020C40F87A
:10140000041C011D42F8043C131DBCF1000FE6DC76
:1014100080E700BF830770B5064614D10368A3F1C7
:10142000013222EA030010F0803F0CD1331D1A462E
:1014300053F8044BA4F1013525EA040414F0803F6D
:10144000F5D0104600E0304603782BB1421C1478EA
:1014500010460132002CFAD100F080F8304670BD01
:10146000C9B2F0B400294BD082070FD00278002A0D
:1014700071D0914242D0431C05E013F8012B002AA1
:101480003BD091423AD09A071846F6D1036841EA18
:101490000127A3F1013222EA030212F0803F47EA5A
:1014A00007471CD17B40A3F1013222EA030313F06A
:1014B000803F14D1021D02E014F0803F0FD110468E
:1014C00052F8043BA3F1013687EA030426EA03033A
:1014D000A4F1013513F0803F25EA0404ECD0027832
:1014E000002A38D0914209D0431C01E0914205D036
:1014F000184613F8012B002AF8D11046F0BC7047AB
:1015000083070BD00278002AF8D0431C03E001784F
:1015100001330029F2D099071846F8D10168A1F1EA
:10152000013323EA010212F0803F0AD1031D18465D
:1015300053F8041BA1F1013424EA010212F0803FA8
:10154000F5D00378002BD9D0421C11781046013217
:101550000029FAD1D2E71046D0E700BF80EA0102A5
:10156000844612F0030F4FD111F0030F32D14DF822
:10157000044D11F0040F51F8043B0BD0A3F10132DC
:101580009A4312F0803F04BF4CF8043B51F8043BEF
:1015900016D100BF51F8044BA3F101329A4312F067
:1015A000803FA4F101320BD14CF8043BA24312F06E
:1015B000803F04BF51F8043B4CF8044BEAD023466B
:1015C0000CF8013B13F0FF0F4FEA3323F8D15DF81D
:1015D000044B704711F0010F06D011F8012B0CF8E5
:1015E000012B002A08BF704711F0020FBFD031F85D
:1015F000022B12F0FF0F16BF2CF8022B8CF80020E4
:1016000012F47F4FB3D1704711F8012B0CF8012B66
:10161000002AF9D1704700BF20F0030110F0030049
:10162000C0F1000051F8043B00F1040C4FEACC0C6F
:101630006FF000021CBF22FA0CF213434FF0010CB2
:101640004CEA0C2C4CEA0C4CA3EB0C0222EA0302F1
:1016500012EACC1204BF51F8043B0430F4D013F06A
:10166000FF0F1FBF013013F47F4F013013F47F0FC2
:1016700018BF0130704700BFF0B4002A63D0344B6C
:1016800004461B6814F8010B571E1D186E7807F0EE
:10169000010706F00305012D58D011F8015B5E1912
:1016A000767806F00306012E08BF2035401B4BD18B
:1016B000002D49D0013A47D02FB314F8010B1D1863
:1016C0006E7806F00305012D11F8015B08BF20308C
:1016D0005E19767806F00306012E08BF2035401B00
:1016E00032D18DB3013A0ED12EE011F8012B9E18A4
:1016F000767806F00306012E08BF2032801A23D127
:1017000012B36A1E20D014F8010B1D186E7806F073
:101710000305012D11F8015B08BF20305E197678B2
:1017200006F00306012E08BF2035401B0CD15DB129
:1017300014F8010B551E1A18567806F00302012AF8
:10174000D3D12030D1E71046F0BC70472030A4E759
:10175000A401002041EA00039B07F0B474D1032ADE
:1017600072D90C4654F8045B161FA5F1013727EA1D
:10177000050717F0803F0346C6F3800C31D10346BE
:10178000032E324643F8045B2AD9BCF1000F0AD07D
:10179000214654F8045BA5F1013626EA050616F049
:1017A000803F18D01DE0264656F8045B2146A5F17F
:1017B000013727EA050717F0803F12D143F8045B91
:1017C00065683146A5F1013626EA0506043A0C1D86
:1017D00016F0803F05D1043A032A43F8045BE2D8AF
:1017E00021467AB30D78013A03F8015B9DB112F0FE
:1017F000010F1C462AD1234622B311F8015F013A9A
:1018000003F8015B3DB111F8015F013A65705C1CA2
:101810002346002DEFD1AAB100219C18DA4303F82A
:10182000011BA218A34202F001020BD01AB103F867
:10183000011BA34206D01A4602F8011B5970531C23
:10184000A342F8D1F0BC70470346CAE711F8015F24
:101850001C4604F8015B013A2346002DCBD1DAE7A0
:101860002DE9F00701273C4600254FF0FF366319AC
:101870008B4200EB060C0DD21CF804A010F803807C
:10188000D0452ED201241D469F1B63198B4200EBCD
:10189000060CF1D34FF0010A1760544600254FF0B3
:1018A000FF3C6319994200EB0C080ED918F804802C
:1018B00010F80390C1451AD901241D46CCEB030A48
:1018C0006319994200EB0C08F0D80CF101000136C5
:1018D000B0423CBFBA463046C2F800A0BDE8F007AF
:1018E00070470BD001272E463C46ED19BFE709D0C3
:1018F0004FF0010AAC4654465544D2E7BC4205D0ED
:101900000134B4E7544505D00134CAE727461D46E3
:101910000124ACE7A2461D460124C2E72DE9F04FA1
:10192000ADF2244D1546064689461046194607AACB
:101930001C46FFF795FF07AB82460DF21C411A1DAE
:101940005C6008338B425460F9D114B301232F78C3
:10195000611E08A8A34240F8271001EA030218D02C
:1019600032B16A7802234F1EA34240F8227010D091
:10197000B046A4465C1C15F803E0CE1A2A5D02337B
:101980000F1B634540F82E6040F82270F2D14646A6
:101990006446079928466918524600F045FC00281D
:1019A00040F0B6800AF1FF3E05EB0E0CCDF808E0E2
:1019B000CAF1010E834604F1FF38CDF80CC0CDF812
:1019C00014E00746CDF810A04A460095019408E0BF
:1019D00027B1079FBB4201D20199CB1B9B44002733
:1019E0002246019CB0185C440021A21A00F07CFB46
:1019F000002840F08780002C00F08480301910F817
:101A0000013C08A951F82330002BE1D1049B9F42EF
:101A100028BF3B46434527D2DDF8009006EB0B017B
:101A200019F80350CA5C09EB0300954266D1DD4307
:101A3000454415F0010F024613D00133434513D23C
:101A40004078CD5C013285420BD057E012F8010F8F
:101A5000CD5C854252D1013312F8010FCD5C854235
:101A60004CD101334345F1D3DDF81090029B4F4533
:101A700028BF4B4639D2DDF808C0DDF8009006EBF0
:101A80000B0519F80C1015F80C00814240F0C080CD
:101A9000DDF80CE009EB070ACAEB0E01C807724635
:101AA0001ED5DDF8089009F1FF31DDF80C90685C77
:101AB00019F801CC09F1FF32844516D10B460FE02D
:101AC00012F8019C15F800E04A1EF1450DD10346BD
:101AD000013815F800C011F8011C614505D1034615
:101AE000581E524502F1FF31EAD101379F4200F200
:101AF0009180079F019ABB44D71B71E7DDF814E082
:101B0000F3446BE7002009B00DF5806DBDE8F08F60
:101B1000CAEB0400504538BF5046CAF10102431CCD
:101B20000AF1FF3C05EB0A0704F1FF3B0192009428
:101B30004A460793B1464FF0000864463E46009976
:101B400009EB020008EB0107BA1A002100F0CCFAF9
:101B50000028D7D1002FD5D009EB070010F8013CA1
:101B600008AA52F8230000284AD1DA4509EB0800F8
:101B70002AD210F80A303178994218BF534642D120
:101B80006FEA0A0303EB0B01C9073246534618D527
:101B90000AF101035B4517D2324612F8011F10F813
:101BA00003E08E450DD02EE012F8011F10F803C09F
:101BB0008C4528D1013312F8011F10F803E08E453F
:101BC00021D101335B45EFD3621C23469BD0295DB5
:101BD000025D914213D1E10709D5631EE95CC25C45
:101BE000914204D00BE0E95CC25C914207D15A1EDD
:101BF000002B88D0A95C825C023B9142F3D007980D
